:020000040800F2
:1000000000040020B9010008BB010008BB01000882
:10001000BB010008BB010008BB010008BB010008D0
:10002000BB010008BB010008BB01000895BC00082B
:10003000BB010008BB010008BB010008CDCE0008D1
:10004000BB010008BB010008BB010008BB010008A0
:10005000BB010008BB010008C9300008F5300008EA
:10006000213100084D31000879310008BB0100083A
:10007000BB010008BB01000809D50008BB0100084E
:10008000A5310008BB010008BB010008BB01000846
:10009000BB010008BB010008BB010008BB01000850
:1000A000BB010008BB010008BDD00008BB0100086F
:1000B000BB010008BB010008EDCE0008BB01000831
:1000C000BB01000831320008BB010008BB01000879
:1000D000BB010008BB010008BB010008BB01000810
:1000E00072B6264880F30888254880F30988254899
:1000F00025490860022080F31488BFF36F8F0BF04E
:1001000041FB0BF01BF94FF0553020491B4A91423F
:100110003CBF41F8040BFAE71D49194A91423CBF24
:1001200041F8040BFAE71B491B4A1C4B9A423EBF9D
:1001300051F8040B42F8040BF8E700201849194A5B
:1001400091423CBF41F8040BFAE70BF01FFB0BF0A8
:100150001AFB154C154DAC4203DA54F8041B8847C2
:10016000F9E705F0F7FF124C124DAC4203DA54F8F0
:10017000041B8847F9E70BF007BB000000040020D0
:10018000000C00200000000808ED00E00000002046
:100190000004002080F20008000C00204011002024
:1001A000401100209C330020E0000008E00000081F
:1001B000E0000008E000000892E700F000F8FEE729
:1001C0002DE9F04FC1F80CD0C3689D46BDE8F08F13
:1001D000002383F311882846A04700200BF0DAFCA7
:1001E000FEE70BF00DFC00DFFEE7000053B94AB953
:1001F000002908BF00281CBF4FF0FF314FF0FF302F
:1002000000F074B9ADF1080C6DE904CE00F006F809
:10021000DDF804E0DDE9022304B070472DE9F04782
:100220008C460446089E002B40F086808A42154684
:1002300048D9B2FA82F24AB1C2F1200701FA02F3B8
:1002400020FA07F7954047EA030C94404FEA154E11
:10025000BCFBFEF71FFA85F80EFB17C307FB08F976
:10026000210C41EA0343994509D9EB1807F1FF3105
:1002700080F0E180994540F2DE80023F2B44A3EB01
:100280000903B3FBFEF00EFB103300FB08F1A4B230
:1002900044EA0344A14209D92C1900F1FF3380F04C
:1002A000C880A14240F2C58002382C4440EA074091
:1002B0000027641A1EB10023D440C6E90043394622
:1002C000BDE8F087002A54D0B2FA82F2002A40F04A
:1002D000B4800127491B4FEA15481FFA85F9B1FB85
:1002E000F8FE08FB1E1109FB0EF04FEA144C4CEA15
:1002F0000143984207D9EB180EF1FF3102D2984220
:1003000000F2EB808E461B1AB3FBF8F008FB1033AB
:1003100009FB00F9A4B244EA0344A14507D92C190A
:1003200000F1FF3302D2A14500F2DB801846A4EBB6
:10033000090440EA0E40BDE78B4208D9002E75D073
:100340000027C6E9000138463946BDE8F087B3FA10
:1003500083F77FB98B4202D3824200F2BC80841AB9
:1003600061EB030301209C46002EA8D0C6E9004C97
:10037000A5E7FFDEC7F12005BB4022FA05FC4CEAE9
:10038000030C21FA05F44FEA1C4EB4FBFEF91FFAE8
:100390008CF80EFB194420FA05F3B94009FB08FA62
:1003A00019430B0C43EA0444A24502FA07F200FA8F
:1003B00007F30BD91CEB040409F1FF3080F08980AE
:1003C000A24540F28680A9F102096444A4EB0A0424
:1003D000B4FBFEF00EFB104400FB08FA89B241EAC0
:1003E0000444A24508D91CEB040400F1FF316CD28F
:1003F000A2456AD90238644440EA0940A0FB028958
:10040000A4EB0A044C454146CE4655D352D0002EAB
:100410006AD05A1A64EB0E0404FA05F522FA07F3BF
:10042000FC401D43C6E90054002748E737463046E4
:1004300045E718463AE70F4621E79540C2F1200309
:1004400021FA03F04FEA1548B0FBF8F71FFA85F9D7
:1004500008FB170E24FA03FC914007FB09FA4CEA4B
:100460000101080C40EA0E40824504FA02F407D963
:10047000281807F1FF332AD2824528D9023F2844A1
:10048000A0EB0A00B0FBF8FC08FB1C000CFB09F316
:1004900089B241EA00418B4208D969180CF1FF305A
:1004A00011D28B420FD9ACF1020C2944C91A4CEA83
:1004B000074714E74345AAD2B8EB020169EB0C02E7
:1004C00001389646A3E78446F0E7084694E71F46BE
:1004D000D6E781467AE7384646E7AEF1020E2B446E
:1004E00011E702382C4422E73746E8E6704700BFA0
:1004F00008B5062000F0FAF901200CF00FFB00BF50
:10050000032A70B412D940EA0105AD0704460B4630
:1005100020D11946204653F8045B54F8046BAE42D0
:1005200018D1043A032A20461946F2D8541E72B153
:1005300003780A789A4208BF241806D00CE010F815
:10054000013F11F8012F934206D1A042F7D10020BC
:1005500070BC7047541EEBE7981A70BC704700BF20
:10056000844641EA000313F0030349D1403A23D300
:100570000B6803604B6843608B688360CB68C36023
:100580000B6903614B6943618B698361CB69C3610B
:100590000B6A03624B6A43628B6A8362CB6AC362F3
:1005A0000B6B03634B6B43638B6B8363CB6BC363DB
:1005B00040304031403ADBD230320BD30B6803601D
:1005C0004B6843608B688360CB68C3601030103128
:1005D000103AF3D20C3205D351F8043B40F8043BF7
:1005E000043AF9D2043208D0D2071CBF11F8013BFB
:1005F00000F8013B01D30B8803806046704700BFC1
:10060000082A13D38B07B1D010F00303AED0C3F187
:100610000403D21ADB071CBF11F8013B00F8013BB1
:10062000A4D331F8023B20F8023B9FE7043AD9D328
:10063000013A11F8013B00F8013BF9D20B78037045
:100640004B7843708B78837060467047F0B48607B0
:1006500046D0541E002A3CD0CAB2034602E014F130
:10066000FF3436D303F8012B9D07F8D1032C29D989
:10067000CDB245EA05250F2C45EA054533D9A4F14D
:100680001006360903F1200707EB061703F11002E5
:1006900042E9045542E902551032BA42F8D1721CBF
:1006A00014F00C0F03EB021204F00F0613D0331FEB
:1006B00023F003030433134442F8045B9342FBD159
:1006C00006F003042CB1C9B21C4403F8011B9C4280
:1006D000FBD1F0BC704734461346002CF3D1F8E749
:1006E00014460346C2E71A462646E0E738B5124BE1
:1006F00005461C68A06B18B10023C0E9045338BD3F
:10070000182000F0A1F9A06378B101220023C0E90C
:1007100004230A4B0B24836000230949094A84817E
:10072000C0E90012C0E9045338BD0246064B42211D
:10073000064800F041F900BF000C0020ECDE050087
:100740000E33CDAB34126DE6B0F10008C8F10008ED
:1007500038B51A4B1C68A26B92B1146918495369D9
:1007600001FB04F1174800FB0313A4FB0045611CC7
:100770001D4445F1000323F00040C2E9041338BDD5
:10078000182000F061F90246A06388B10124002519
:100790000B21C0E904450C4B0948136003460B4D7F
:1007A0000B4C91810B49C2E90154C2E9041338BDD5
:1007B000094B4E21094800F0FFF800BF000C002053
:1007C0002DF451582D7F954C0E33CDAB34126DE680
:1007D000ECDE05002E7F954CB0F10008C8F1000852
:1007E00010B58021044600F093F9606440B1002206
:1007F000031F7C3043F8042F8342FBD1002010BD3F
:100800004FF0FF3010BD00BF436C0BB100207047AC
:10081000E6E700BF1F2970B5054608D8436C1646A9
:100820000C464BB153F8240043F8246070BD1622E7
:100830004FF0FF302A6070BDFFF7D2FF08B96B6C34
:10084000F0E74FF0FF3070BD1F2938B5054620D8BE
:10085000426C0C466AB152F8213053B1012B16D0CC
:10086000591C10D00025204642F8245098472846AD
:1008700038BD284600F070F8224601462846BDE8FB
:10088000384000F055B8162301202B6038BD0020F9
:1008900038BD16234FF0FF302B6038BD1F2921D8FB
:1008A00038B5436C05460C4683B153F8242003EB5E
:1008B00084034AB1511C10D0012A0CD000252046D7
:1008C0001D609047284638BD012038BDFFF788FFDE
:1008D00028B96B6CE9E7032038BD022038BD4FF022
:1008E000FF3038BD4FF0FF30704700BF024B01466C
:1008F0001868FFF7A9BF00BF000C0020024B0A4692
:1009000001461868FFF786BF000C0020034B1868EB
:10091000436C0BB10020704762E700BF000C002061
:10092000024B01461868FFF7B9BF00BF000C00205A
:1009300070B50D460023074C064611462846236035
:100940000CF0F4F8431C00D070BD2368002BFBD0E2
:10095000336070BD743300200CF0F0B820F0030158
:1009600010F00300C0F1000051F8043B00F1040C4A
:100970004FEACC0C6FF000021CBF22FA0CF21343BA
:100980004FF0010C4CEA0C2C4CEA0C4CA3EB0C0283
:1009900022EA030212EACC1204BF51F8043B0430ED
:1009A000F4D0C2F1000102EA0102B2FA82F2C2F10D
:1009B0001F0200EBD200704700B50A4C05462068C4
:1009C00085B01C46C06852B1074BCDE90132009199
:1009D0002B462246054900F023F8FFF789FD044B1A
:1009E0001A46F2E7000C0020FCF100080CF20008A7
:1009F00008F2000808B513460022FFF7DDFF00BF2C
:100A00000CB410B582B004AC54F8042B2346019406
:100A100000F024F902B0BDE8104002B0704700BFFA
:100A20000EB430B582B005AC54F8042B054D014628
:100A300023462868019400F011F902B0BDE8304067
:100A400003B07047000C0020024B0146186800F00C
:100A50005FB800BF000C0020024B0146186800F090
:100A600003B800BF000C002000293AD038B551F877
:100A7000043C0C1F002BB8BFE418054601F088FAAF
:100A8000224B1A682AB1A2420DD92168601882420D
:100A900021D0626028461C60BDE8384001F07EBA73
:100AA000A34203D81A465368002BF9D11168501895
:100AB000A04217D022D821686018834203BFD3E92F
:100AC00000030918C4E90013636054602846BDE8B8
:100AD000384001F063BAD2E900020144C4E90012CF
:100AE000D8E7704720680144501883421160EDD167
:100AF000D3E900030144C2E90013E7E70C232846C9
:100B00002B60BDE8384001F049BA00BF4011002019
:100B1000F8B5CD1C25F0030508350C2D38BF0C2584
:100B2000002D064633DBA94231D82A4F01F030FAB6
:100B30003A6852B113685B1B04D43FE023685B1B27
:100B400029D522465468002CF8D1796800293BD079
:100B5000294630460BF0C6FF431C28D0C41C24F0A5
:100B60000304A04205D0211A30460BF0BBFF013030
:100B70001DD02560304601F011FA04F10B0020F081
:100B80000700231DC21A01D01B1AA350F8BD0C2266
:100B900000203260F8BD0B2B05D8A242636811D04B
:100BA0005360E7E7144623601C442560E2E70C230A
:100BB0003046336001F0F2F90020F8BD0B2BF1D87C
:100BC000144653683B60D5E730460BF08BFF7860E6
:100BD000BEE700BF401100209368013B002B9360EB
:100BE0000FDA10B49469A34208DB0A2906D013680F
:100BF000581C10601970084610BC704710BC00F0FB
:100C00009FBB1368581C106019700846704700BFDE
:100C10009BB1F8B513440F4606465D1E541E01E015
:100C2000AC4208D03A4614F8011F3046FFF7D4FF13
:100C3000431CF5D1F8BD0020F8BD0020704700BF6F
:100C4000936810B5144613B95360184610BD00F0F0
:100C50009BFE0023C4E9013310BD00BF2DE9F04F16
:100C60009FB08B4690461C46039018B18369002BB9
:100C700000F0C880AE4B9B4500F0CA80AD4B9B4551
:100C800000F0CA80AC4B9B4504BF039BD3F80CB06B
:100C9000DBF86430BBF80C20DB0702D4970540F189
:100CA0005781160740F12B81DBF81030002B00F044
:100CB000268100202021302298F800300127059459
:100CC0000B908DF831109D4E8DF83220002B00F0E6
:100CD0008880252B00F01181454603E0252B00F08C
:100CE0009F8025466B786C1C002BF7D1B4EB080A6B
:100CF00077D04246534659460398FFF789FF0130A3
:100D00006FD00B9B6A7853440B93002A69D0002361
:100D10004FF0FF3201340693CDE908338DF85B3094
:100D20001C93079206E02C46069B801B07FA00F0F6
:100D3000184306902546052215F8011B304601F0A0
:100D40007BF8AA460028EED1069BD80644BF202295
:100D50008DF85B20190748BF2B22217848BF8DF8FA
:100D60005B202A2961D1059A116804320029059275
:100D7000C0F2988009916178A51C2E296ED0704C24
:100D80000322204601F058F8002800F0818040221C
:100D9000069B001B02FA00F00343069305F10108CD
:100DA0002B780622194667488DF8303001F044F858
:100DB00000287DD0644B002B6DD005AB00935A46C4
:100DC000624B06A90398AFF300808146B9F1FF3F5B
:100DD00007D00B9B4B440B9398F80030002B7FF40B
:100DE00078AFDBF8643013F0010FBBF80C3002D1A0
:100DF0009A0540F1B4805B0600F194800B981FB017
:100E0000BDE8F08F00F0A8FC494B9B457FF436AF5E
:100E1000039BD3F804B03BE7039BD3F808B037E754
:100E2000B4EB080A3FF473AF63E7A1F13002092A7B
:100E300088BFA246A1D8099B01E02C46013529783C
:100E400003EB830302EB4303A1F13002092AAA4614
:100E5000F3D92E2904F10205099390D19AF80110D3
:100E60002A292FD1059B0AF102001A680433002AAF
:100E7000079205939AF802100AF1030538DB304C0B
:100E800082460322204600F0D7FF00287FF47FAF80
:100E9000A846554684E7059B073323F0070308332C
:100EA000059396E7494243F002030991069362E7EE
:100EB00005AB00935A46254B06A9039800F0F6F8B7
:100EC000814683E70023A1F13002092A079301D963
:100ED0002BE05546697803EB830302EB4303A1F152
:100EE0003002092A05F1010AF3D90235079346E7D2
:100EF0004FF0FF338246079341E7444607E75946E0
:100F0000039800F07DFA00283FF4D3AEDBF864309C
:100F1000DD0707D4BBF80C309C0503D4DBF8580080
:100F200000F010FF4FF0FF3069E7AA46013526E7D1
:100F3000F8E50008D8E50008B8E500083CF200082C
:100F400044F2000848F2000800000000110C0008FC
:100F5000DBF8580000F0EEFEBBF80C20A1E6DBF851
:100F6000580000F0EFFEBBF80C3044E710B4044C1E
:100F700013460A460146206810BCFFF76FBE00BF4B
:100F8000000C00202DE9F0470C460969A568914640
:100F90008D42B8BF0D46156094F8431006461F46B3
:100FA000DDF8208011B16A1CC9F800202368990679
:100FB0005CD5D9F800200232C9F80020236813F06C
:100FC000060F19461DD1E1688A1A002AD8BF1946B2
:100FD00017DD002504F1190A05E0E368D9F80020BF
:100FE0009B1AAB420CDD0123524639463046C047BE
:100FF000013005F10105F0D14FF0FF30BDE8F08779
:10100000216894F84330003318BF01238A060AD5BB
:101010003021E21882F8431094F845105A1C2244FB
:1010200082F84310023304F1430239463046C04788
:101030000130E1D02368A26803F00603042B216984
:101040001DD08A4226DD4FF00009521A9144002536
:101050001A3401E04D451DDA012322463946304657
:10106000C047013005F10105F4D1C5E713F0060FC3
:1010700013D094F84330003318BF0123D3E7D9F8D5
:101080000000E3688A42A3EB000323EAE379DCDC97
:10109000002BDCDC0020BDE8F087E168D9F80020F7
:1010A0008A1A002AD8BF194693DCAAE72DE9F04333
:1010B0000C46097E85B06E2906461746984604F10F
:1010C000430C0C986DD039D9732900F0F48044D9C1
:1010D000752900F00281782940F00F817823226879
:1010E000DFF854E284F845300168150651F8043BF6
:1010F000016040F1A180D10744BF42F0200222608C
:10110000002B00F093801022002184F843106068C7
:101110000028A060C0F2C680216821F0040121608F
:10112000002B40F0A280002840F0BE806546082ACF
:1011300000F0AB80ACEB0503236141E0632900F0D4
:10114000E3801AD8002938D0582940F0D68084F896
:1011500045102268DFF8E4E1C6E76F2900F0BD80A2
:10116000702940F0CA8078232268DFF8CCE142F091
:101170002002226084F84530B6E7642902D069294C
:1011800040F0BB8022680368110603F1040557D5BF
:10119000196805600B46002959DB0A22DFF89CE13B
:1011A000B5E7036822681D1D6169056015061B68A7
:1011B00002D4500600F1BB8019600023654623610C
:1011C000CDF800803B4603AA21463046FFF7DAFE01
:1011D000013020D02A46236939463046C0470130C5
:1011E00019D0226803989207E36819D51A1A002AC1
:1011F00016DD002504F1190904E0E36803981A1AC2
:10120000AA420DDD01234A4639463046C047013027
:1012100005F10105F1D14FF0FF3005B0BDE8F083D5
:101220009842B8BF184605B0BDE8F0832168102287
:1012300021F02001216067E7500648BF9BB25AE7C2
:101240005106A5D5B3F9003005601946A3E72D2056
:1012500061685B42002984F84300A16002DB22F050
:10126000040222600A22DFF8D4E0654600E00B4663
:10127000B3FBF2F102FB11301EF80000934205F8B7
:10128000010DF4D2082A7FF455AF2368DB077FF500
:1012900051AF626823699A423FF74CAF3023013D5A
:1012A0002B7047E7002BE0D19EF8003004F1420597
:1012B00084F842303BE703686268191D01601D68CD
:1012C0000021284600F0B8FD002832D0401B6060A5
:1012D0002061002384F8433072E72268036812F02B
:1012E000800F03F104051AD01B6805606F290CBF3D
:1012F00008220A22DFF844E006E7012384F84210BE
:10130000236104F14205E4E70122036804F1420588
:10131000191D1B68016084F842302261D9E712F080
:10132000400F0DBF1B6805601B880560DEE7198054
:1013300043E76068CCE700BF64F2000850F20008A1
:10134000F8B50D461446064608B1836943B3254BEC
:101350009C422AD0244B9C4229D0244B9C4208BF5B
:10136000F468A269A389A2601A0722D5236903B38E
:1013700022686169D31AEDB299422F4629DD013303
:10138000A168501C0139A1602060157062699A4201
:1013900016D0A389DB0701D50A2D11D03846F8BD38
:1013A00000F0DAF90F4B9C42D4D17468D9E7B468E5
:1013B000D7E72146304600F023F838B92369D7E74C
:1013C0002146304600F032F90028E7D04FF0FF37D1
:1013D000E4E72146304600F029F90028F6D1012340
:1013E0002268CDE7F8E50008D8E50008B8E5000870
:1013F000024B0A4601461868FFF7A2BF000C002006
:101400003B4B70B51D6806460C460DB1AB69DBB1B0
:10141000384B9C421ED0384B9C424AD0374B9C42A2
:1014200008BFEC68B4F90C2093B2190718D52069ED
:1014300008B313F001022CD000226369A2605B4262
:10144000A36160B3002070BD284600F085F9294BE8
:101450009C42E0D16C68B4F90C2093B21907E6D431
:10146000DD063CD5580726D4206942F00803A38145
:101470009BB20028DDD103F42072B2F5007FD8D0F2
:101480003046214600F08EFCA389206913F001024A
:10149000D2D1990758BF6269A2600028D2D1B4F9AD
:1014A0000C301A06CFD543F04003A3814FF0FF3034
:1014B00070BDAC68B6E7616B51B104F14403994269
:1014C00004D03046FFF7D0FAB4F90C200023636350
:1014D0000023206922F02402C4E90003C5E70923A0
:1014E00042F0400233604FF0FF30A28170BD00BF78
:1014F000000C0020F8E50008D8E50008B8E5000871
:101500002DE9F0418F890C463A07804641D44B685B
:10151000002B59DDE66A002E53D0002317F48052C9
:10152000D8F80050216AC8F8003051D10123404654
:10153000B047431C5FD0A789E66A216A7F0705D5BB
:101540006268636B801A0BB1236CC01A02460023D9
:101550004046B047461C45D1D8F80030B4F90C20BD
:10156000002B55D01D2B01D0162B5AD100222369F8
:10157000C4E90032616BC8F8005011B304F14403B0
:10158000994202D04046FFF76FFA00206063BDE841
:10159000F0810E69AEB10D680E60B90714BF00236B
:1015A0006369AD1BA3600AE02B463246A76A216A35
:1015B0004046B8470028A5EB000506440ADD002D8B
:1015C000F2DC0020BDE8F0810B6C002BA2DCF8E718
:1015D000606DB3E7A3894FF0FF3043F04003A38170
:1015E000BDE8F081002322696360A3892260DA04E8
:1015F000C0D56065BEE7D8F80030002B9BD01D2B0E
:101600000CD0162B0AD0A38943F04003A381D9E75D
:101610002169C4E90013D304ACD5EAE7C8F8005047
:10162000CFE742F04002A281CCE700BF38B50B699A
:101630001BB30C46054608B183691BB3184B9C428B
:101640001ED0184B9C4220D0174B9C4208BFEC6820
:10165000B4F90C308BB1626ED00701D4990516D560
:1016600028462146FFF74CFF636E0546DA0702D491
:10167000A3899B050FD5284638BD0025284638BDCF
:101680006C68E5E700F068F8D8E7AC68E0E7A06DC3
:1016900000F050FBE4E7A06D00F054FBEBE700BF67
:1016A000F8E50008D8E50008B8E5000820B1054BCA
:1016B00001461868FFF7BABF034B0449186800F0E9
:1016C00007BB00BF000C0020B4E500082D16000881
:1016D000014900F0FDBA00BF2D16000808B5436EA1
:1016E000DA0702D483899B0501D5002008BD806DEF
:1016F00000F020FB002008BD08B5436EDA0702D4D5
:1017000083899B0501D5002008BD806D00F01AFB80
:10171000002008BD70B568254A1E05FB02F50E467F
:1017200005F17401FFF7F4F9044640B100210C30D3
:10173000666005F168022160A060FEF787FF204621
:1017400070BD00BF024B0349186800F0C1BA00BF6A
:10175000B4E500082D1600082DE9F84F05463A4873
:1017600000F0E8FAAB69002B69D1384AC5E91233B9
:1017700012682B65AA4208BF0123354908BFAB6137
:10178000A962284600F072F86860284600F06EF8FA
:10179000A8602846002400F069F804236E68E86019
:1017A00021467466C6E90044B460C6E90444B461E5
:1017B000F36006F15C000822FEF748FFDFF89CB0FA
:1017C000AF68DFF89CA0DFF89C90DFF89C80214B8D
:1017D000C6E9086BC6E90AA9C6F830802146FB6055
:1017E0007C66C7E90044BC60C7E90444BC6107F1FA
:1017F0005C000822FEF72AFFEE68174BC7E9087B5A
:10180000C7E90AA9C7F830802146F3607466C6E9C3
:101810000044B460C6E90444B46106F15C000822E7
:10182000FEF714FF0123C6E9086BC6E90AA9C6F84A
:1018300030800548AB61BDE8F84F00F083BA02483C
:10184000BDE8F84F00F07EBA84330020B4E500080C
:10185000D11600080900010012000200F51F00085F
:101860001D2000085D2000087D20000870B5064698
:10187000244800F05FFA244B1D68AB697BB3483500
:10188000D5E90134013B05D525E0013B5A1C04F1A3
:10189000680420D0B4F90C20002AF6D100251B4B97
:1018A00004F15800E360656600F03CFA154800F06A
:1018B00049FA2560C4E90155C4E90455A5612946E2
:1018C000082204F15C00FEF7C1FEC4E90D55C4E92D
:1018D0001255204670BD2C682CB12546D0E728460D
:1018E000FFF73AFFCBE704213046FFF713FF04462A
:1018F00028600028F1D1034800F024FA0C2333605B
:10190000E7E700BF98330020B4E500080100FFFFBF
:10191000014800F00FBA00BF98330020014800F0E2
:1019200011BA00BF98330020014800F003BA00BF8D
:1019300084330020014800F005BA00BF8433002042
:1019400008B5054800F0F6F9044B05491868BDE8EC
:10195000084000F099B900BF98330020000C002027
:10196000DD16000808B5054B0549186800F08CF92C
:10197000BDE80840034800F0E5B900BF000C0020B6
:10198000F9160008983300209368002B00F0FC80C3
:101990002DE9F04FB1F90C300C469BB2190783B01A
:1019A000824690462BD522694AB313F00202D8F83A
:1019B000006033D000273D46D4F828B0216ADFF814
:1019C000C492C5B14D452B463A4628BF4B465046BA
:1019D000D847002840F3CE80D8F8083007441B1AB7
:1019E0002D1AC8F80830002B00F0B380D4F828B0C6
:1019F000216A002DE6D1D6E900750836E1E72146D7
:101A00005046FFF7FDFC002840F03781B4F90C3058
:101A1000D8F800609BB213F00202CBD113F0010999
:101A200040F0B4804D46A7682068002D55D09A0537
:101A300040F1C080AF42BB4600F2EE8013F4906FDD
:101A40002FD0D4E9041707EB4707A0EB010B07EBF6
:101A5000D777681C7F105844B8423A4684BF07467F
:101A60003A465B0540F1F08011465046FFF750F8CA
:101A7000002800F0FC805A4621690190FEF770FDB5
:101A8000A289019B22F4906242F08002A281A7EB1E
:101A90000B0203EB0B006761AB462F46236120600E
:101AA000A2605A46494600F00DFA2368A2685B44DA
:101AB000AB460025D71BA7602360D8F80870D9442F
:101AC000A7EB0B07C8F80870002F42D0B4F90C3010
:101AD000A7689BB22068002DA9D1D6E900950836E9
:101AE000A3E70BF1080353F8047C9B4653F8086CFA
:101AF0000833002FF7D03A460A21304600F09CF90F
:101B0000002854D00130A0EB06094B46206821691B
:101B1000BB4228BF3B468842626903D9A568154489
:101B2000AB421ADC9A4200F381801346A56A324622
:101B3000216A5046A847051E1CDDB9EB05096ED089
:101B40000120D8F808302E445B1B7F1BC8F80830F2
:101B500013BB002003B0BDE8F08F31462A4600F0E9
:101B6000B1F9236821462B4423605046FFF75EFD00
:101B70000028E2D0B4F90C304FF0FF3043F04003BE
:101B8000A38103B0BDE8F08F002070473346914633
:101B9000104617464E469B46002FA2D00028B4D1CF
:101BA0003A460A21304600F047F90028AAD17B1CAA
:101BB0009946ABE72369834217D36269AA4214D8D6
:101BC0002F4BA76A9D4294BF2B466FF0004393FBB7
:101BD000F2F3216A02FB03F350464A46B847B0F1DC
:101BE000000BC7DDA5EB0B0567E7AF4228BF2F460B
:101BF00049463A4600F066F9A3682268DB1B3A447E
:101C0000BB46A3602260002BECD121465046FFF773
:101C10000DFD0028E6D0ADE72F46AB4641E7214653
:101C20005046FFF703FD00288BD0A3E71A46314644
:101C30001D46019300F046F9A1682268019BC91A6C
:101C40001344A160236078E7504600F0ADF90346E5
:101C500000287FF41CAF21695046FEF705FF0C22D7
:101C6000B4F90C30CAF8002023F0800384E70C227A
:101C7000B4F90C30CAF800207EE74FF0FF3069E776
:101C8000FEFFFF7F00FCFF7F2DE9F04110F14807C8
:101C90001AD088460026D7E90154013D0ED4A38905
:101CA000013D012B06D9B4F90E30013302D0204694
:101CB000C04706436B1C04F16804F0D13F68002F55
:101CC000E9D13046BDE8F0813E463046BDE8F081BE
:101CD0002DE9F84310F148061ED0884607464FF01C
:101CE0000009D6E90154013D10D4A389013D012B1F
:101CF00008D9B4F90E30013304D021463846C04724
:101D000049EA00096B1C04F16804EED13668002E24
:101D1000E7D14846BDE8F883B1464846BDE8F883B8
:101D2000704700BF704700BF704700BF704700BFDB
:101D3000704700BF704700BF012070470120704707
:101D4000704700BF704700BF70B50C46B1F90E1068
:101D500096B0002916461D4613DB6A460AF0CFFEF0
:101D600000280EDB019A4FF4806302F47042A2F562
:101D70000052B2FA82F2002052092A60336016B093
:101D800070BD0022A3892A601B0604D540230020D1
:101D9000336016B070BD4FF480630020336016B01E
:101DA00070BD00BF8A890B46920706D5012103F159
:101DB000470259611A601A61704770B582B001AB71
:101DC0006A460C460646FFF7BFFF009905463046B7
:101DD000FEF79EFEB4F90C3070B1164A0099B2625B
:101DE000019A43F08003A3812060C4E904018AB909
:101DF0002B43A38102B070BD9A05FBD4012123F0CF
:101E0000030304F1470243F00203A38161612260EE
:101E10002261EFE73046B4F90E100AF07CFE10B9EB
:101E2000B4F90C30E4E7A38923F0030343F0010382
:101E30001BB2DDE7D1160008830770B4CDB23DD0E8
:101E4000541E0AB30378AB421FD0431C05E014F1C3
:101E5000FF3419D30278AA4217D013F0030F1846A3
:101E600003F10103F3D1032C11D84CB30378AB4237
:101E70000BD00444431C02E00278AA4205D09C42E5
:101E8000184603F10103F7D1002070BC70470246E9
:101E90000E02B6B22E4346EA064613681046734059
:101EA000A3F1013121EA030313F0803F02F10402A0
:101EB000DCD1043C032C1046EFD8D6E71446D2E719
:101EC0002046E2E78842F0B40DD98B1883420AD944
:101ED000841832B1224613F8014D994202F8014D9F
:101EE000F9D1F0BC70470F2A0ED80346541E002AC1
:101EF000F7D001340C44013B11F8012BA14203F847
:101F0000012FF9D1F0BC704740EA01039B073AD199
:101F1000A2F110073F0901F1200606EB071601F1B7
:101F2000100300F1100453F8105C103344F8105CF7
:101F300053F81C5C103444F81C5C53F8185C44F8EB
:101F4000185C53F8145CB34244F8145CEBD17B1C6E
:101F50001B0112F00C0F194402F00F05034415D0B9
:101F60000E46043DAD0803EB850C1C1F56F8047BA0
:101F700044F8047F6445F9D10135AD002B44294470
:101F800002F00302B2E7541E0346B2E72A46ADE769
:101F90000148FFF7CFBE00BF883300200148FFF79C
:101FA000D1BE00BF8833002009B3F8B51446CAB1CA
:101FB00006460D4600F066F8A04202D32F4638468A
:101FC000F8BD21463046FEF7A3FD07460028F6D0AF
:101FD00022462946FEF7C4FA30462946FEF744FD5C
:101FE0003846F8BD2746FEF73FFD3846F8BD114696
:101FF000FEF78EBD10B50C46B1F90E100AF067FD64
:10200000002803DB636D0344636510BDA38923F4DB
:102010008053A38110BD00BF002070472DE9F0411F
:10202000B1F90C409846E3050D461746B1F90E107C
:10203000064609D424F48054AC8143463A463046DF
:10204000BDE8F0410AF04ABD022300220AF044FD37
:10205000B5F90C40B5F90E10ECE700BF10B50C4611
:10206000B1F90E100AF038FDA389421C0EBF23F40B
:10207000805343F480536065A38110BDB1F90E1005
:102080000AF02EBD51F8043C181F002BBCBF0B58A2
:10209000C01870470E4A0023114610B5147C8442C4
:1020A0000FD11C225343CA18906848B1CB58FF285F
:1020B00018BF43434FF0010018BF5B00013353606A
:1020C00010BD0133082B02F11C02E7D10020F7E715
:1020D000D80E0020F0B50A4D00242E462F7C8742F2
:1020E00007D11C2000FB0464012061762276A376D0
:1020F000F0BD0134082C05F11C05EFD10020F7E7F5
:10210000D80E0020094A30B500231446157C8542BC
:1021100005D11C22012002FB0343596030BD01336D
:10212000082B02F11C02F1D10020F7E7D80E0020A5
:1021300070B50B4C00232546267C864209D11C2015
:102140004343E818E95000238260C36043740120D0
:1021500070BD0133082B04F11C04EDD10020F7E71A
:10216000D80E0020F8B500252E46334C6368002BAE
:102170005ED0E06858BB637CB3FA83F35B09637499
:1021800008F046FCD4E900239342E06035D2666053
:102190006674E66063699BB1207C984780B1A36850
:1021A000FF2B0DD1677E217EA37E47EA01021A43F1
:1021B00006D0207CFF2823D11A46384606F0E2F9E3
:1021C0000135082D04F11C04D0D10120F8BD08F020
:1021D00065FC23689842CED26368002BDAD0204693
:1021E00002F0AAF80028EBD0637C207CABB1FF287A
:1021F0000DD1A27E217E607EE0E79B1A6360EBE753
:102200005E28DDD80A46394605F012FBD8E75E287D
:10221000D6D8A37E227E617EF6E7FF2803D11A4638
:1022200019461846CAE75E28CAD81A461946EBE787
:102230006374E360C4E700BFD80E002007B543789D
:102240008DF8003083788DF80130C3788DF8023036
:1022500043798DF80330037968468DF804300BF02C
:102260005DFD03B05DF804FB08B5074B5A78022A00
:1022700007D8586808F012FCC72894BF0020012036
:1022800008BD0020FCE700BF9C0C0020704708B58B
:10229000002240214FF080400AF0E0FDFFF7F6FFFA
:1022A00000BF00BF00BF00BF00BF00BF00BF00BF36
:1022B00000BF00BF00BF00BF00BF00BF00BF00BF26
:1022C00000BF00BF08BD08B501F020F808BD000040
:1022D00008B5064C002120780BF034FD2078FFF77C
:1022E000F2FF052009F05BFCF4E700BF702F00202F
:1022F00010B5084C236803F07142074B1343236069
:1023000008F086FB054B18602068BDE8104003F01C
:1023100077BA00BF702F00200001010E4C11002081
:1023200008B5012280214FF080400AF097FD4FF060
:10233000804380229A61BDE8084001F0B3B80120D3
:1023400070470000144B10B51C78BCB9134B1B78B8
:10235000042B13D103F030F903F044F903F0F8F83B
:1023600003F088F904F054F804F06EF8204608F001
:10237000AFF92046BDE8104008F0C6B90BF094FF55
:1023800048B10BF059FC0028FBD1BDE8104044F6E1
:10239000206009F004BC10BD702F00202033002005
:1023A00038B500230D460B70074C30B108F030FBF8
:1023B000002320602B70002038BD206808F06EFBE1
:1023C0003228F3D8F7E700BF5C110020084B9A7859
:1023D000012A07D0022A09D0064B1868B0FA80F00B
:1023E0004009704758780128F6D170470120FCE772
:1023F0009C0C00204016002008B5054B9B78013B43
:10240000012B02D9FFF7E2FF08BD0120FCE700BF66
:102410009C0C002008B508F0FBFA014B986008BD41
:102420009C0C00202DE9F0410C461546074600287B
:1024300038D0B1FA81F35B09A3B14D4E4FF0804221
:102440003378002C32D08021012B91610AD03046A4
:102450000AF0C4FC30460AF0A6F84648464B8360B2
:1024600008F002F9A74201D0FFF76CFF434E337822
:10247000A34200D11DB10022414B9A611A773470FA
:1024800024B1631E042B747098BFB470306803F0DD
:10249000B7F93378062B64D8DFE803F06119303AD6
:1024A000444E58000B1C18BF0123C5E74FF4000130
:1024B000042B9161D6D0334BDFF8B8801C70324BBF
:1024C0003046C8F8083008F075FE4046C8E73120AD
:1024D00045B10BF0F1FB52200BF0EEFB01200BF0AD
:1024E000F7FB51200BF0E8FBFFF794FF2A4621464B
:1024F000384601F0E7FB0120BDE8F0813220002DD5
:10250000F0D00BF0D9FB52200BF0D6FB0220E6E70F
:102510003320002DE6D00BF0CFFB52200BF0CCFB8C
:102520000320DCE73420002DDCD00BF0C5FB52206B
:102530000BF0C2FB0420D2E73520002DD2D00BF0E7
:10254000BBFB52200BF0B8FB0520C8E73020002D64
:10255000C8D00BF0B1FB52200BF0AEFBC1E711204D
:10256000C0E711200BF0A8FBFFF7C2FEBCE700BFDD
:1025700020330020201100203D220008702F002071
:10258000640C0020B0230020B9B20008002313B56A
:102590000DF107018DF80730FFF702FF044690B1F7
:1025A0009DF80730013B032B0DD8DFE803F002064E
:1025B0000F1200221146094B02E00022074B9978C6
:1025C0001878FFF72FFF204602B010BD0022062129
:1025D000F1E7024B00225978F2E700BF702F00208C
:1025E00013B5124C20460BF0CBFA0123637703F0AE
:1025F00004F90F4C206008B9FFF77AFEE37843F046
:102600000103E37008F004FA0A4BFF22186000236C
:102610004FF49A6100930848084B09F08DFAFFF7D0
:1026200036FE0120FFF7B2FF02B010BD640C00209F
:10263000702F00204C11002060110020D1220008D2
:1026400038B5114C054623782070637008F0E0F926
:10265000032D606016D10120FFF798FF40B90B4AA7
:10266000537812785AB1024619461846FFF7DAFE37
:10267000FFF7D0FEBDE8384053200BF01DBB1146DC
:102680001846F3E738BD00BF9C0C0020702F0020D7
:10269000014B1878704700BF9C0C0020014B9870CC
:1026A000704700BF9C0C0020014BD870704700BFE2
:1026B0009C0C0020014BD878704700BF9C0C002078
:1026C0000122014B1A70704758110020F8B5164BC3
:1026D0009C681CB9FFF79EFE0020F8BD134D144EF8
:1026E0002A7892B100232B704FF080431B69F27857
:1026F0009B0963F30002F27032680E4B1340B3F192
:10270000807FE9D000F028FEE7E7F3780A4AC3F3B8
:10271000420352F82370002FDED0204608F0BEF9A5
:10272000B842DFD2D8E700BF9C0C0020581100202F
:10273000702F0020FF00000154E600080C4B10B57C
:102740005A781946012A03D0022A08D0002005E051
:102750009C78012C03D100F061FE204610BD486832
:1027600008F09CF9C728F1D9FFF730FEF6E700BF63
:102770009C0C002008B5074BDB780BB1022B04D171
:102780000220FFF75DFF002008BD0320FFF758FF80
:102790000120F9E79C0C002038B5094D0024E878A9
:1027A000032807D1FFF74CFF2046AC7000F0E4FD92
:1027B000012038BD0220FFF743FF2046F9E700BFA4
:1027C0009C0C002070B5754C754D2068A0B108F0C8
:1027D00065F9B0F5FA6F0FD30026552026600BF08F
:1027E0006BFA57200BF068FA287832460146B0FAA7
:1027F00080F04009FFF716FE2B781BB1694BDA7F9A
:10280000694B1A702368ABB9684C206808F046F928
:1028100040F6B73398420DD92B785BB10BF00CFA28
:1028200040B9604B5B7F2BB108F0F2F82060532079
:102830000BF042FA4FF080431B69EA789B095C4C2D
:1028400063F300020020EA70FFF7A0FE2378032B59
:102850001ED8DFE803F0021E448AE36833B19847CC
:1028600020B10120FFF7ECFE0023A370236933B1F0
:10287000984720B10120FFF7E3FE0223A3706369AC
:1028800033B1984720B10120FFF7DAFE0123A3708E
:1028900070BDA369002BFBD098470028F8D001F049
:1028A0007FFB444B187006F02DFC0021424A2B7828
:1028B00013703C4A51776BB9404C2378012B09D0F7
:1028C0004FF08043802220469A610AF087FA204622
:1028D00009F069FE0220BDE87040FFF7B1BEE36970
:1028E000002BD5D098470028D2D04FF080434FF42A
:1028F00080229A61A37813B3022B0BD86378022B42
:1029000008D0FFF71FFD11200BF0D6F90BF094F95A
:102910000028FBD100F012FD0023E370264B2A783B
:102920001B789A4202D1A07800F088FAA378012B94
:1029300018D0A3B1022BABD1FFF72EFFA8E7194B9C
:102940005B7E002BE6D111200BF0B6F90BF074F989
:102950000028FBD147F2305009F021F9DAE7FFF700
:1029600009FF95E701F02AFD92E7236A002B8FD03B
:10297000984700288CD001220A4B5A770D4B1B78C0
:102980002BB14FF0804304229A6106F0A1FB00F0C6
:10299000C9FCFFF73FFD00209DE700BF4C11002060
:1029A000702F0020640C0020B02300205411002060
:1029B0009C0C0020481100205011002020330020E2
:1029C0000120704708B5FFF7FBFF08BD37B5044687
:1029D0000D46FFF71FFD29462046FFF7F3FF60B1C4
:1029E000074B1A784AB1074B20461B78D90900914A
:1029F000C3F3001369790BF0ABFC03B030BD00BF2B
:102A0000702F0020782F002008B5074807F01EF926
:102A1000064807F01BF90BF00BF907F017F9BDE8B2
:102A20000840034807F012B974E600088FE6000872
:102A3000B6E600082D4B13B51A7804466AB12C4B44
:102A400001211B78DB09009300230BF081FC0BF0C4
:102A5000F3F80028FBD102B010BD0028FBD0031F03
:102A6000DBB2A02B12D8234B0146186807F086FE74
:102A700020B1204602F064FD02F0FCFD204602F089
:102A800057FD02B0BDE8104002F0F4BD00F1200394
:102A9000DBB2072B07D800F007040120A040C0B22A
:102AA00002F07AFDEDE700F15B03DBB2022B06D802
:102AB000114AD05C02B0BDE8104007F009BE00F139
:102AC0005803DBB21A2B07D80C4A32F8130002B0B5
:102AD000BDE8104007F018BE3334E4B2122CBAD867
:102AE000012102B0BDE8104001F0BFBE702F0020F0
:102AF000782F0020C40F002018E600081CE600080C
:102B0000264B13B51A7804466AB1254B1B78DB09AE
:102B10000093002319460BF01BFC0BF08DF80028E6
:102B2000FBD102B010BD0028FBD0031FDBB2A02BED
:102B300006D802F005FD02B0BDE8104002F09ABDD3
:102B400000F12003DBB2072B07D800F007040120B7
:102B5000A040C0B202F028FDEDE700F15B03DBB25C
:102B6000022B05D8104602B0BDE8104007F0B0BDFA
:102B700000F15803DBB21A2B05D8104602B0BDE8AD
:102B8000104007F0C1BD3334E4B2122CC9D811464D
:102B900002B0BDE8104001F068BE00BF702F0020F9
:102BA000782F00202DE9F3410546E0B1134E32782D
:102BB000E2B10127DFF84880284601F0E3FD98F8EC
:102BC00000300446DB09E030009332780023012115
:102BD00080B20BF0BDFB0BF02FF80028FBD107FAF9
:102BE00004F4A543E8D102B0BDE8F08102F0D4FCC2
:102BF00002B0BDE8F04102F03DBD00BF702F0020E3
:102C0000782F00202DE9F3410546E0B1134E3278CC
:102C1000E2B10127DFF84880284601F0B3FD98F8BB
:102C200000300446DB0900930023E0303278194677
:102C300080B20BF08DFB0AF0FFFF0028FBD107FAF2
:102C400004F4A543E8D102B0BDE8F08102F0ACFC89
:102C500002B0BDE8F04102F00DBD00BF702F0020B2
:102C6000782F00202DE9F3410546E0B1134E32786C
:102C7000E2B10127DFF84880284601F083FD98F88B
:102C800000300446DB09E030009332780023012154
:102C900080B20BF05DFB0AF0CFFF0028FBD107FAF2
:102CA00004F4A543E8D102B0BDE8F08102F08AFC4B
:102CB00002B0BDE8F04102F0DDBC00BF702F002083
:102CC000782F00202DE9F3410546E0B1134E32780C
:102CD000E2B10127DFF84880284601F053FD98F85B
:102CE00000300446DB0900930023E03032781946B7
:102CF00080B20BF02DFB0AF09FFF0028FBD107FAF2
:102D000004F4A543E8D102B0BDE8F08102F062FC12
:102D100002B0BDE8F04102F0ADBC00BF702F002052
:102D2000782F002038B51C4B1B7863B91B4C1C4D09
:102D30002378052B04D14FF080431B695A0603D436
:102D400007F066FE286038BD28680028F8D007F034
:102D5000A5FE41F658339842F5D907F059FE286090
:102D600025462378052B05D002F084FCBDE83840C9
:102D700003F04EBB07F015FEB4F84C309B07F0D5BE
:102D800007F0F6FD0028ECD0284609F09BFC284609
:102D900001F082F8E5E700BF702F0020203300200B
:102DA00030160020704700001A4B70B59C6C0F263F
:102DB00044F4C0649C649B6C012301F003048B40C9
:102DC00021F0030101F1804101F5A0518D68A400BB
:102DD000C0F38320A04006FA04F425EA0405284342
:102DE0008860D8430C4912F0010F8C6814BF1C4353
:102DF00004408C6012F0020FCA6814BF1A430240EC
:102E0000CA60054A536111680B431360536803405D
:102E1000536070BD000C0140001800400120704755
:102E200008B5FFF7FBFF38B1BDE8084001220621D5
:102E30004FF08040FFF7B8BF08BD00002DE9F04714
:102E40003023054683F31188824B00269A6C4FF09D
:102E5000010842F4C0629A649A6CD3F890207E4FC5
:102E600042F4C062C3F89020D3F89020DFF81492A7
:102E700022F4C062C3F89020D3F89030FFF7D0FF5F
:102E800057F8040B95B1012D49D1484547D120F0A1
:102E90000F0A00F00F0008FA00F421460522504600
:102EA000240409F0DBFFCAF8184001E0441CEED10D
:102EB0000136112EE4D107240127684EDFF8C881BE
:102EC00056F8040B002D36D0012D40F0B680404559
:102ED00040F0B38000F00F01202207FA01F120F04A
:102EE0000F0009F0BBFF00BF00BF00BF00BF00BF65
:102EF00000BF00BF00BF00BF00BF00BF00BF00BFDA
:102F000000BF00BF00BF00BF00BF56F8040C032283
:102F100000F00F0120F00F00FFF746FF0DE0411C0D
:102F2000C6D000F00F01202208FA01F120F00F00B6
:102F300009F094FFBCE7421CCCD1013CC0D184F322
:102F4000118872B6464A47491368424823F0010384
:102F500013600323444A93620C23D362434B0B60F8
:102F600001238460C36042480860A1F5A0418C67DA
:102F700040499462D462A2F5684251611946002228
:102F8000A30003F1604303F56143D3F80001D5B218
:102F9000012D94BF002000F0010008B1C3F880119A
:102FA0000132202AF1D10134082CE8D1324C636877
:102FB00043F00073636009F031FF2B4B1A6802F095
:102FC00009021A601A6842F46C3242F004021A6074
:102FD00040F2B3321A62294B43F001039847236948
:102FE00043F00403236130BF254B43F001039847AE
:102FF00023691B4A23F004032361136843F0010390
:10300000136008F09BF9134B9A6C42F4C0629A6407
:103010009A6C9A6C42F480429A649A6C9A6C42F46C
:1030200080529A649B6CFFF7BDFE02F08FFF002375
:1030300083F3118862B6BDE8F087431C3FF47DAF8F
:1030400000F00F01402207FA01F120F00F0009F013
:1030500005FF72E7000C01403CE70008DCE70008D0
:1030600010E000E0005401400000014014000003A3
:1030700010000003FFFF070000ED00E0B4E70008C8
:1030800080E700080E040040030000400120704764
:1030900001207047012303FA01F2024210B50C46E9
:1030A0000DD003290CD006290CD10320FFF7FCFA20
:1030B0002046FFF7EBFF10B12046FFF7E9FF10BDF8
:1030C0000420F3E71846F1E710B5094C6369DB0704
:1030D00007D52368002123F0010323600120FFF7B7
:1030E000D9FF4FF0FF336361BDE8104008F000BE28
:1030F0000018004010B5094C606910F0020006D0BD
:103100002368012123F002032360FFF7C3FF4FF080
:10311000FF336361BDE8104008F0EABD00180040CD
:1031200010B5094C606910F0040006D02368022134
:1031300023F004032360FFF7ADFF4FF0FF3363611B
:10314000BDE8104008F0D4BD0018004010B5094C8F
:10315000606910F0080006D02368032123F00803FB
:103160002360FFF797FF4FF0FF336361BDE8104026
:1031700008F0BEBD0018004010B5094C606910F0A1
:10318000100006D02368042123F010032360FFF70A
:1031900081FF4FF0FF336361BDE8104008F0A8BD28
:1031A0000018004038B5214B5C69A00604F478751E
:1031B00007D51A68052122F020021A602846FFF779
:1031C00069FF610608D5194A06211368284623F0CD
:1031D00040031360FFF75EFF220608D5134A07215C
:1031E0001368284623F080031360FFF753FFE305BD
:1031F00008D50E4A08211368284623F4807313600B
:10320000FFF748FF14F4007F084C07D0236809211A
:1032100023F4007323602846FFF73CFF4FF0FF3391
:103220006361BDE8384008F063BD00BF001800408E
:1032300038B5264B5C69620504F47C4507D51A68ED
:103240000A2122F480621A602846FFF723FF200536
:1032500008D51E4A0B211368284623F40063136027
:10326000FFF718FFE10408D5184A0C211368284617
:1032700023F480531360FFF70DFFA20408D5134A0F
:103280000D211368284623F400531360FFF702FF53
:10329000630408D50D4A0E211368284623F48043A1
:1032A0001360FFF7F7FE14F4004F084C07D02368B3
:1032B0000F2123F4004323602846FFF7EBFE4FF075
:1032C000FF336361BDE8384008F012BD00180040CC
:1032D00010B5074C23784BB900F0A6FE01F06FFA49
:1032E00007F0C8F901F06CFA01232370012010BD2A
:1032F0003516002010B5044C23781BB100F096FE63
:1033000000232370012010BD35160020024B1B78CE
:103310000BB10AF09BBC70473816002001207047A3
:103320000120704708B5044B1B780BB9FFF7D0FF9D
:10333000FFF7F4FF08BD00BF3516002008B5044BA9
:103340001B780BB1FFF7D6FFFFF7EAFF08BD00BF00
:10335000351600200120704708B5FFF7FBFF08BDB8
:10336000014B1878704700BF36160020014B1870CB
:10337000704700BF36160020014B1870704700BF21
:1033800036160020014B1878704700BF3716002012
:10339000084B10B50446187058B9FFF779F90228A0
:1033A00007D80320FFF74CF92046BDE81040FFF78F
:1033B00075B910BD37160020FFF7EABF024B187829
:1033C00080F00100FFF7E4BF37160020084B1A78A1
:1033D000084B1B784BB982F00102A0F5A443203BB7
:1033E0001F2B8CBF1046012070470022F5E700BF5D
:1033F000371600203616002000231946054A93721E
:103400001360054A01330B2B917242F80C1BF9D162
:10341000704700BF54160020C00C002008B502F011
:1034200007FEFFF7E9FF0022014B1A6008BD00BF4D
:103430004016002008B505F0ADFE18282CD8172836
:1034400003D2062801D00DD880B9002328201A46BF
:10345000194604F0EDF900235C201A46194604F0E1
:10346000E7F903E00828F0D00A28EED007F00AF9BF
:10347000820705D5442328201A46194604F0D8F9B6
:1034800007F000F9430705D544235C201A46194686
:1034900004F0CEF9012008BD1C28E7D31E28D4D99A
:1034A0002028E2E708B5FFF713FFFFF799F800F0CF
:1034B00095FD50B1012204214FF0804009F0CEFC6F
:1034C0004FF080434FF480229A6108BD00230E4ADA
:1034D00010B513700D4A4FF0804413700C4A1360FE
:1034E000FEF798FF05F02EFE01280AD005F022FE17
:1034F0004FF48023A36100F07DFDBDE8104002F091
:1035000010BA0423F6E700BF341600203916002055
:103510003C16002008B502F0D5F904F03FF902F09E
:1035200065F9084B188060F07F001870188802F069
:1035300060F900F0D3FD18B1BDE80840FFF7C6BF41
:1035400008BD00BF782F002037B504460D4600F0B7
:10355000D6FD002800F0BD80002D00F0BA8047F6AF
:1035600004639C4200F0858029D847F601639C42A1
:103570005BD00AD847F603439C4200F0A780B4F51D
:10358000FC4F3CD0284603B030BD47F602639C4256
:103590005DD047F603639C42F4D100230DF107018F
:1035A00001208DF80730FEF7FBFE9DF80730042B55
:1035B00002D013F0FD0FE5D10122042130E047F6DF
:1035C00012639C427BD00BD847F605639C4263D0C4
:1035D00047F611639C42D5D10020FFF7D9FED1E711
:1035E00047F613639C426ED047F643639C42C9D1B1
:1035F0000122394B1A700022384B1A60C2E70023AF
:103600000DF1070101208DF80730FEF7C9FE9DF886
:103610000730042B02D013F0FD0FB3D10122114665
:103620002F4B1878FEF7FEFEACE700230DF10701E3
:1036300001208DF80730FEF7B3FE9DF80730042B0C
:1036400002D013F0FD0F9DD101220221E8E70023F3
:103650000DF1070101208DF80730FEF7A1FE9DF85E
:103660000730042B02D013F0FD0F8BD10122032170
:10367000D6E700230DF1070101208DF80730FEF792
:103680008FFE9DF80730042B03D013F0FD0F7FF45D
:1036900079AF01220521C3E700230DF107010120C5
:1036A0008DF80730FEF77CFE9DF80730DA1E012A00
:1036B00002D9002B7FF466AF01220621B0E7012278
:1036C000084B1A705EE7FFF779FE5BE7FFF722FF12
:1036D00058E7054656E700BF391600203C16002083
:1036E000702F00203716002070B5154CFFF76AF8D0
:1036F000206858B1A37A4BB907F0D0F963689842B3
:1037000004D301212089A172FFF71EFF00250126A5
:103710000C4C206858B1A37A4BB907F0BFF9636825
:10372000984204D3A67201212089FFF70DFF0135CD
:103730000B2D04F10C04ECD100F07AFC70BD00BF3D
:1037400054160020C00C002008B5064B1B780BB99E
:10375000FFF7BEFD4FF0804304229A61BDE80840A8
:1037600007F005B93516002008B5074B1B780BB1DB
:10377000FFF7C0FD4FF080434FF480229A61BDE80F
:10378000084007F0F3B800BF351600202DE9F743D5
:103790000D46AD4A49790446136891B1032B00D810
:1037A0000133AA4E1360FEF735FE33899C4204D1E3
:1037B0006F7957B107F02CF93060A54B0027984678
:1037C00029E0002BEDD0013BEBE7B37A0BB9336076
:1037D000F3E739462046FFF7B7FEB7723760002897
:1037E000EBD1002095E07E4308EB0607BB7A13B9C6
:1037F00048F806301DE049462046FFF7A5FE87F849
:103800000A9048F806900028EBD012E001370B2F01
:1038100003F10C030DD01A899442F7D195F8059065
:103820000C26B9F1000FDED007F0F2F87E4348F81D
:10383000060029462046FFF7C9FD0028D1D02946B9
:10384000204600F05FFC0028CBD047F604639C4282
:1038500000F0C1802CD8B4F5FC4F67D009D847F6EA
:1038600020039C4200F0158147F603439C42B8D0E8
:103870002EE047F602639C426B7900F0918074D988
:10388000002BAED0734C2278042AAAD000230DF16D
:10389000070101208DF80730FEF782FD9DF8073003
:1038A000042B02D013F0FD0F9BD10022042158E01D
:1038B00047F640639C421ED015D847F606639C42EB
:1038C00000F0CE80C0F0A38047F607639C422AD068
:1038D0002946204600F064FE002882D02946204672
:1038E000FFF774F815E047F642639C4214D009D301
:1038F00047F64363BAE76B79002B3FF472AFFFF7EB
:1039000083F86EE76879544B10B101221A7068E7AA
:10391000187003B0BDE8F0836B79002B3FF461AF02
:10392000FEF7CEFE5DE76A794C4BEFE76B79002B33
:103930003FF457AF474C2278012A3FF452AF00239F
:103940000DF1070101208DF80730FEF729FD9DF8E4
:103950000730042B03D013F0FD0F7FF442AF002299
:1039600001212078FEF75EFD3BE7002B3FF439AFE5
:10397000384C2278022A3FF434AF00230DF10701BE
:1039800001208DF80730FEF70BFD9DF80730042B62
:1039900003D013F0FD0F7FF424AF00220221E0E7F3
:1039A000002B3FF41EAF2B4C2278032A3FF419AFB3
:1039B00000230DF1070101208DF80730FEF7F0FC20
:1039C0009DF80730042B03D013F0FD0F7FF409AFEF
:1039D00000220321C5E76B79002B3FF402AF1D4C99
:1039E0002278052A3FF4FDAE00230DF107010120E6
:1039F0008DF80730FEF7D4FC9DF80730042B03D078
:103A000013F0FD0F7FF4EDAE00220521A9E76B79DD
:103A1000002B3FF4E6AE0F4C2278062A3FF4E1AECD
:103A200000230DF1070101208DF80730FEF7B8FCE7
:103A30009DF80730DA1E012A02D9002B7FF4D1AE9F
:103A4000002206218DE700BF4016002054160020FA
:103A5000C00C0020702F00203816002034160020E3
:103A60006B79002B3FF4BDAE114C2278002A3FF455
:103A7000B8AE00230DF1070101208DF80730FEF7E5
:103A80008FFC9DF80730012B3FF6ABAE00221146AC
:103A900067E76B79002B7FF41BAF05F053FB4FF00A
:103AA000804318B14FF480229A6111E70422FBE7AA
:103AB000702F0020014B1870704700BF4416002083
:103AC000F8B505460C46584E584F2146284600F09A
:103AD00019FC50B1062C08D8DFE804F004085D9307
:103AE00093A0A0000022504B1A60F8BD32687ABB48
:103AF000A5F14703042B0BD8DFE803F025201B16A4
:103B000003000023FF211A464B20FEF7E3FA0122AF
:103B10004FF4FA712846FEF70BFB2846FEF7BAFA77
:103B200006F076FF3060E0E7FF22002311464A20CE
:103B3000EBE70022FF2311464920E6E70023FF229E
:103B400019464820E1E7442347201A461946DCE796
:103B5000104606F0A3FF4EF65F23984203D90524D2
:103B6000334B1C70B1E7334B1B7883B9472D0ED113
:103B7000314B1B78042B3FD103232D4C2846237057
:103B800044231A461946FEF7A5FA24789DE77A7E63
:103B90008AB30324E4E73068F8B9A5F14803032B9E
:103BA000A3D8DFE803F015100B020023FF211A460B
:103BB0004B20FEF78FFA0122C821ABE7FF2200233A
:103BC00011464A20F5E70022FF2311464920F0E77D
:103BD0000023FF2219464820EBE706F05FFF4EF670
:103BE0005F23984201D90624BAE77B7E0BB10424F7
:103BF000B6E7104B1B786BB12846BDE8F840FEF7DE
:103C000049BAFF224FF4FA612846FEF791FA284696
:103C1000FEF740FA0022064B1A7066E70022044BBA
:103C20001A70FEF74DFDE7E748160020640C0020EF
:103C300044160020702F00202033002008B5034BCD
:103C40001978FFF73DFF012008BD00BF4416002092
:103C50000120704770B506460D464B200021FEF747
:103C600051FA10B90024204670BD00214A20FEF709
:103C700049FA0028F6D000214920FEF743FA00282F
:103C8000F0D000214820FEF73DFA0028EAD00021BC
:103C90004720FEF737FA0028E4D029463046FFF7E0
:103CA000D7FF04460028DDD00022044B29461D70B2
:103CB000034B30461A60FFF703FFD4E74416002099
:103CC0004816002070B50D461446FEF738FB064630
:103CD00080B155B3174B5B7E2BBB013D052D09D839
:103CE000DFE805F0030C120808182CB102214B2064
:103CF000FFF7B0FF304670BD0121F8E714B1022193
:103D00004A20F5E70121FBE714B102214920EFE742
:103D10000121FBE714B102214820E9E70121FBE77B
:103D200002214720E4E71E46E4E7002CF8D10121F8
:103D3000F7E700BF640C0020094B1B787BB9094BE7
:103D40001A7832B1084A527E4AB959781046FEF7BD
:103D500069BB064B1B78042B01D01146F6E7704770
:103D600044160020702F0020640C00202033002017
:103D70002DE9FF473F4D06460F4600F0F5FAFFF7E5
:103D8000DBFF2C78002C31D03B4C236813B906F0B4
:103D90003FFE2060206806F081FE40F6B73398426F
:103DA00005D92B7801332B7006F032FE20602B787A
:103DB000013B032B16D8DFE803F0020B0F130022A0
:103DC0001146442004F0DEFB002004B0BDE8F0877B
:103DD000002244211046F5E7002144220846F1E77D
:103DE0004422EDE700232B702360EDE7234B1B7883
:103DF00083B939463046FFF71DFB0028E4D0394629
:103E00003046FEF7AFF93946304604B0BDE8F0471A
:103E100000F0BCBA22462146204604F0B3FBDFF88E
:103E200060A0DFF860900DF104080A2551462A468B
:103E30004046FCF795FB99F81E30E2B2B3FBF5F56E
:103E4000954214F8080011D9312B03D90023FF2221
:103E5000194605E01D2B4FF00003F8D81A46FF2144
:103E6000013403F0E5FC0A2CDFD1C2E700231A4637
:103E7000EEE700BF391600203C1600203416002063
:103E8000A0E40008640C0020012804BF014B187056
:103E900006F044BD1C110020014807F080BE00BFA1
:103EA000A0860100F8B50023374E5E280446337023
:103EB000364D21D1364A374F1269F97882F4806243
:103EC000C2F3802262F30001CA072B70F97015D586
:103ED000314A927F632A17D9304A19461360442227
:103EE000FEF7F8F8FF22C8215E20FEF721F9012332
:103EF0002B705E20FEF7CEF82878F8BD4FF0804397
:103F00001B6913F040030BD00023244A19461360A9
:103F10005E204422FEF7DEF801224FF49671E3E7BB
:103F20001D4FBA7F0A2A23D81A464421FEF7D2F839
:103F30000122C8212046FEF7FBF801232B703370C5
:103F4000BB7F012BD5D8154C236813B906F060FD53
:103F5000206020680028CCD006F0A0FD42F210734B
:103F60009842C6D9002301202360FFF7FFF9C0E77C
:103F70000A4A194613601A46FEF7ACF8FF22C82118
:103F80002046FEF7D5F8B4E74E1600204D16002067
:103F900000080040702F0020640C00205016002004
:103FA000024B1878C0F34000704700BF742F002008
:103FB000034B1A7860F341021A70186801F027BCAD
:103FC000742F0020044A137823F0030343F0030303
:103FD0001370106801F01BBC742F002008B500227C
:103FE0004FF48061024808F039FF012008BD00BF8E
:103FF0000008004010B501F007FC0A4B186008B932
:10400000FFF7E0FF4FF080444FF48023A36105F0F9
:1040100099F808B10423A3615E20FEF73BF8012064
:1040200010BD00BF742F0020012070470120704791
:10403000F8B5254C254A2378002B41D0106806F0AE
:104040002DFDB0F57A7F34D34FF08045204A2B699F
:104050001178C3F3801399421E4E13D02B69C3F31A
:10406000801313702B695B060CD51B4F3B78042B18
:1040700008D006F0CDFC4FF400033060AB61384649
:1040800007F098F83068A0B106F008FDB0F5FA6FB7
:104090000FD30022104D32602B78042B0BD04FF041
:1040A0008043802228469A6108F098FE284608F04E
:1040B0007AFA0120F8BD11462078FEF7B3F9F8E747
:1040C0001360044A1360F4E7702F00206816002084
:1040D00060160020641600202033002008B5442319
:1040E000FF201A461946FDF7F5FF0322FA21FF20AB
:1040F000FEF71EF8FF20FDF7CDFF012008BD0120CF
:104100007047000045F22123984270B505460C46E1
:1041100000F0CD8017D8B0F5A97F00F0B6800AD89E
:10412000E32800F0A58040F251139D4200F0AD80DD
:104130000124204670BD40F22B43984200F0A78036
:1041400040F62C03F1E747F62303984236D020D8F7
:1041500045F22323984200F0AA8047F620039842B4
:10416000E6D14C79002C39D1614D2878C0F340005C
:1041700080F0010000F00100FFF71AFF2B789B0789
:1041800040F1A38004F0B6FF4FF0804304229A610F
:10419000CFE747F6146398422ED047F6156398424E
:1041A0004DD047F607639842C2D1524B1B7803B1FA
:1041B0004B79514A03F0010313700FE004F0EAFF5A
:1041C0000B28B5D00CD8072806D80528B0D201385E
:1041D000C0B2012802D8ABE70928A9D00024A8E77B
:1041E000282805D82128A3D21C28A1D01F28F4E70D
:1041F0002B38C0B20228EDE7404C207800F0C2FA1C
:104200000228EBD0207800F0BDFA88B9022000F037
:104210001EFA002244231146FF20FDF75BFF012216
:10422000FA21FF20FDF784FFFF20FDF733FFD5E7DC
:10423000207800F0A7FA0228EBD10020E7E72F4C06
:10424000207800F09FFA02280546C7D1207800F0B8
:1042500099FA30B9284600F0FAF9002344221946A9
:10426000DAE7207800F08EFA0228F6D10020F2E793
:10427000224B187800F086FA02287FF459AF2846BE
:1042800064798CB100F058F9A8E76479F9E74C79C2
:104290004CB11B4B1A7822B90122E2201A7000F0AF
:1042A0004BF92B20EEE72B2000F05CF941E7667913
:1042B000002E7FF43DAF124D2C78002C3FF438AF28
:1042C000E22000F04FF92E7033E706F0DBF910F032
:1042D000FF0F83D12C78C4F34004002C7FF47EAF11
:1042E00004F028FF4FF080434FF480224FE700BFD7
:1042F000742F0020702F002034160020721600202A
:104300004C1600200539012910B5044610D80020AC
:10431000FFF7D0FB074B1B7833B1FEF7D1F92046EE
:10432000FDF7B8FE002010BD4FF080431B69F6E793
:104330000120F8E7702F002008B5037C5E2B0DD11B
:10434000074B1B7813B1074B187830B900235E2058
:104350001A46194603F06CFA002008BD0120FCE75C
:10436000702F00204D160020064B1B789B0702D5AE
:10437000054B1B7823B100221146104604F002B908
:10438000704700BF742F00204E16002008B5094B5F
:104390001B78DB060BD5084B187800F0F3F90228E0
:1043A00005D044230B201A46194603F041FA012098
:1043B00008BD00BF782F00207216002008B5FEF758
:1043C00079F904280ED0062801D003280AD1032049
:1043D000FEF736F90020FEF761F90020FEF7ECFF4A
:1043E000012008BD0220FEF72BF90020F9E70000AC
:1043F00010B548B104F0A6FE28B904F07BFE4FF0DA
:10440000804304229A6110BD074B1B789A07FAD4A7
:104410004FF0804423695B07F5D504F08BFE4FF421
:104420008023A361EFE700BF742F002038B5037825
:104430000446072B0D4601D0002038BD4378032BDE
:10444000FAD18378022BF7D10F4BC0781A7858B97C
:1044500060F341021A70186801F0D9F92046294624
:1044600006F040FF0120E8E742F002021A701868E7
:1044700001F0CDF94FF080431869C0F380000028A7
:10448000DAD104229A61D8E7742F002003280DD8CE
:1044900006290BD8102A09D8772301EB011103FB59
:1044A0000010034B104433F8100070470120704790
:1044B00000E80008012070470C22024B02FB00308C
:1044C000704700BFB80F0020A0F58073B3F5F85F08
:1044D00010B526D210F4805F00F4007400F48073ED
:1044E00000F4806100F400620DD0002B0CBF0020AE
:1044F00010200CB140F0200009B140F040000AB19A
:1045000040F0800010BD181C18BF01200CB140F015
:10451000020009B140F00400002AF3D040F0080086
:10452000F0E70020EEE710B50C46FFF7CDFF23467D
:10453000BDE8104018470000A0F1E003072B10B5BC
:10454000044600D940B920460449FFF7ECFFE0B229
:10455000BDE81040FEF76EBA0149F6E7A52B00084A
:10456000652C000810B50446C0B2FEF7C9FAA4F1E4
:10457000E003072B00D92CB903492046BDE81040C1
:10458000FFF7D1BF0149F8E7052C0008C52C00084A
:104590000120704708B5FFF7FBFF08BD01207047F9
:1045A00001207047704708B5FFF7FCFF08BD000009
:1045B00013B502AB03E903000F4B1B78B3B99DF8A9
:1045C0000530009873B16AB100F0BAFC04460146A8
:1045D000009800F083FC2046009902B0BDE810402E
:1045E00001F02CBB00F094FC0446F4E7009800F0C6
:1045F000A7FC0099F1E700BF71160020034600896F
:1046000010B40A4638B95C881888998840EA044092
:1046100010BCFFF7CDBF10BC704738B50121044670
:10462000FFF7ECFF21460546FFF7B4FF18B121461E
:10463000284605F077FC00F0010038BD10B50446AF
:104640000021FFF7DBFF2146FFF7ADFF10BD10B5DE
:1046500001248440E4B2204601F0C4F82046BDE8BD
:10466000104000F09CBB704708B500F03DFBFFF721
:10467000FAFFBDE8084046F2A81007F090BA08B566
:10468000FFF7F2FFBDE8084006F020BA08B5FFF7D3
:10469000EBFFBDE8084006F041BA38B501210546F8
:1046A000FFF7ACFF2946044604F0E5FF08B90020F7
:1046B00038BD29462046FFF769F80028F7D029467B
:1046C000204605F035FF0028F1D02946204605F0A8
:1046D00053F90028EBD02946204605F0A7FE002814
:1046E000E5D02946204604F091FE0028DFD0294677
:1046F000204605F06BFF0028D9D06B795BB147F6F7
:1047000003439C421DD00AD8B4F5F84F16D047F6A3
:1047100001439C4217D02846FFF740FFC8E747F601
:104720005B439C4215D047F65C439C420ED047F653
:104730005A439C42EFD101F031F8ECE7FFF79FFFBD
:10474000B5E701F031F8FFF7A1FFB0E701F01AF883
:10475000E1E701F026F8DEE708B5FFF705F804F019
:10476000AFFB00F035F8BDE80840012004F08CBC38
:1047700008B500F032F8002004F086FCBDE80840DF
:10478000FEF7E2BF03091CBF1846042382081EBFC0
:1047900010460233DBB242081CBF0133DBB21846BD
:1047A000704701207047704738B50546FFF7F9FF9D
:1047B000044610B12846FFF7F6FF204638BD704783
:1047C00010B50446FFF714FE2046FFF7EDFF10BDBD
:1047D00008B50020FFF7F4FF08BD08B505F04AFF53
:1047E000FFF7EEFF08BD000010B505F043FF074BD3
:1047F00004461A78824207D0187006F009F9044B73
:1048000018602046FFF7DCFF10BD00BF70160020C7
:104810006C16002010B586B06C4684E803009DF845
:1048200005300BB100F0DEFE0023ADF81230ADF81C
:10483000143094E8030011F0FF0F0390ADF810104E
:1048400003AC05D194E8070000F00EFE06B010BDE1
:104850002046FFF7E2FE0028F4D1F7E70379012BA9
:1048600002D1008800F08EBB704708B529B101F075
:10487000FBFCBDE8084001F0CBBD01F053FDF8E7BB
:1048800038B505460C46FEF7D5F81CB92846FEF7A4
:1048900037F938BD6420013C07F081F9A4B2F4E790
:1048A00008B539280CBF50210121FFF7E9FF08BDE9
:1048B0002DE9F047867981460C46457900F05CFE8B
:1048C0003609804600B3A846F5B1C4F3072303F0C8
:1048D000F002402A09D004F12002D2B2072A25D9D9
:1048E0001EB903F0E003202B23D0A74B93F80180DF
:1048F00018F0040808D0022000F014FF00F03CFE7D
:1049000080F001005FFA80F8C4F303330B2B3FD82B
:10491000DFE813F01100110060006000BC00D2005D
:104920003E003E00D7003201430143014FF0000832
:10493000EAE7B046E8E7C4F30723C4F3032613F01D
:10494000F00F18BF3601E7B285B156B107F1200369
:10495000DBB2072B304600D92FB900F01DFE00F066
:1049600089FE384658E000F02DFEF8E73846FEF79D
:10497000C7F86EB107F12003DBB2072B304600D930
:1049800017B900F011FE01E000F024FE00F072FE05
:10499000C4F30334083C032C03D805F06BFEFFF787
:1049A0000FFFB8F1000F00F04F8100F0DDFD10F0B7
:1049B000010040F0498189F8050000F0CFFD00F0CA
:1049C00021FA484600F05AF900F0C8FDBDE8F0476A
:1049D00000F024BAC4F3072303F0F003C4F3032761
:1049E000202B5FFA84FA18BF3F01BAF1000F07D0FD
:1049F000BAF1010F32D0002D3AD0CEB150460BE0C3
:104A0000614B5B785A0711D44DB127B1384600F09D
:104A1000C3FD00F02FFE0020FEF70CF8B8E7284693
:104A2000FEF76EF8002FB3D03846AAE755B11EB98D
:104A30003846FEF7B7F8ABE7012EA9D1384600F0AB
:104A4000F1FDA5E7002EA3D13846FEF7DBF8384686
:104A500000F0F6FD384600F0D1FD99E715B1052EBE
:104A600096D8E5E7042E93D83846FEF7CBF88FE7C3
:104A7000002EF9D0BAF1390F0CBF4FF4FA50642070
:104A800007F08DF85046FEF73BF881E7C4F3812329
:104A900043B1012B7FF47CAF65B1C4F3090005F08D
:104AA00033FE75E725B1C4F3090005F011FE6FE789
:104AB0002846FAE72846F2E72946E0B2FFF7D5FE96
:104AC00066E714F4407F27D1002D7FF461AFC4F373
:104AD00042108000C3B204F00F009840C2B214F03C
:104AE00010001EBF0F209840C043C4F3812318BF9D
:104AF000C0B2022B40EA020008D00AD8012B02D033
:104B000000F058F944E700F04DF941E700F05AF998
:104B10003EE700F044F93BE7C4F30122D3B205B30A
:104B200002F00103002B3FF433AFC4F342108000C6
:104B3000C3B204F00F009840C2B214F010001EBFC0
:104B40000F209840C043C4F3812318BFC0B2022B8A
:104B500040EA02000AD00CD8012B04D000F07EF904
:104B600016E75B08DEE700F071F911E700F07EF967
:104B70000EE700F035F90BE7E7B2C4F303262DB1D9
:104B8000304600F03FF953E7782F00203846FEF713
:104B900039F8304600F042F9FAE6E7B2A7F1F0033F
:104BA000042B3DD8DFE803F003220E151E003DB1B3
:104BB000042E3FF6EDAEC4F3042000F03BF9E7E627
:104BC000052EF6E7C4F30420002DE3D100F01AF916
:104BD000DEE625B1C4F3042000F00DF9D8E600F0BC
:104BE00007F9D5E6194B5B785B0704D4C4F30420BE
:104BF000002DCFD0EAE74DB1C4F30425284600F0DC
:104C000001F90321284600F06BFDC1E6012000F008
:104C100089FD012E7FF6BCAE022000F083FDB7E6D1
:104C20002DB1002E7FF49DAEC4F30420CEE746B133
:104C3000392F0CBF4FF4FA50642006F0B0FF38460D
:104C400021E7C4F30420A5E7BDE8F087782F002012
:104C500038B50446008960B100F016FF054600F043
:104C60000DF900F09BF829462046BDE83840FFF7D3
:104C70001FBE2188607900F091F9EFE7037910B544
:104C80000446B3B1FFF709FD68B900F075FC80B1C7
:104C9000637973B1074B5B785B070AD5BDE81040B9
:104CA000022000F03FBD2046FFF7D2FF2046FFF76D
:104CB000C5FC10BD782F002008B5002005F008FDC8
:104CC000002005F021FD00F08DFC00F0D3FC01F088
:104CD000BBFBBDE8084001F09BBB08B500F038FC09
:104CE000BDE80840FFF7E8BF08B500F065FCBDE887
:104CF0000840FFF7F2BFC0F303320E3202F00F029A
:104D0000092A10B5C4B21BD8012101FA02F340F2FE
:104D10000332134203D113F010000DD110BDF02C5B
:104D200010D004D8E72C8CBF00200120F6E7F42C2B
:104D300014BF00200120F1E7E72C03D9F12CF7E79D
:104D40000020EBE70846E9E708B50346007958B1CB
:104D5000188928B100F098FEBDE80840FFF7CBBFE6
:104D6000188800F00FF9F7E708BD82B002AB03E93D
:104D7000030002B0704784B004AB03E9070004B03D
:104D80007047704708B5FFF7FCFF08BD08B5FFF78F
:104D9000F9FF014B187008BD721600207047FFF72D
:104DA000F5BF0000024B1B781843FFF7EFBF00BFB1
:104DB00072160020024B1B781840FFF7E7BF00BFB8
:104DC00072160020024B1B785840FFF7DFBF00BF70
:104DD00072160020704708B5FFF7FCFF08BD000001
:104DE00008B5FFF7F8FF014B187008BD73160020D7
:104DF0000020FFF7F5BF012303FA00F0C0B2FFF770
:104E0000EFBF0000012303FA00F0034B1B781843A7
:104E1000C0B2FFF7E5BF00BF73160020012303FAFD
:104E200000F0034B1B7823EA0000FFF7D9BF00BF57
:104E300073160020012303FA00F0034B1B7858403F
:104E4000C0B2FFF7CDBF00BF73160020024B1B7826
:104E50001843FFF7C5BF00BF73160020024B1B7835
:104E60001840FFF7BDBF00BF73160020024B1B7830
:104E70005840FFF7B5BF00BF73160020704701F020
:104E80000703C90830B501EB4101012401390A4487
:104E900000219C40E4B212F8015F20FA01F343F3D1
:104EA00000036B40234001316B4003291370F2D1A2
:104EB00030BD002210B500F00704C00800EB400030
:104EC000014410468B5CE34003F001039340013240
:104ED0001843032AC0B2F5D110BD000017B40C4628
:104EE000C0F307210629ADF804000CD89DF8043062
:104EF000102B08D8204603EB0113044A194403B0D1
:104F000010BCFFF7BCBF03B010BC70477416002084
:104F100082B0ADF80400C0F3072006280AD89DF837
:104F20000430102B06D800EB00100449184402B0DE
:104F3000FFF7BFBF002002B0704700BF741600200B
:104F400073B503240D4BADF804001E780C4B1B7891
:104F50001E4346FA04F3DB07E5B206D414F1FF342E
:104F6000F7D20025284602B070BD0199284600F00E
:104F700076FE80B20128F1D0F4E700BF731600205E
:104F80007216002007B5ADF804000198FFF7D8FFAE
:104F9000019903B05DF804EB00F061BE13B5104B4E
:104FA000ADF804101B782BB1019802B0BDE8104099
:104FB000FFF7E8BF70B10198FFF7C2FF0446014652
:104FC0000198FFF78BFF2046019902B0BDE8104021
:104FD00000F045BE0198FFF79BFF0446F3E700BFD2
:104FE0007116002010B5012404FA02F204FA01F14E
:104FF0001143C9B231EA000204FA03F306BF1843B1
:10500000C0B2984310BD000008B513460A460146D9
:1050100003480078FFF7E6FFBDE80840FFF7E0BE71
:1050200073160020F8B50A270D4B0E4E1C780E4D56
:105030003378A34200D1F8BD07FB04F2AB18A85A9D
:10504000B3F802C09A88D98840EA0C4042EA01418C
:1050500001341A89FFF78FFE04F00704E8E700BF68
:10506000FD160020FC160020AC160020064B10B4E4
:105070009A885C881888D98840EA044042EA01414D
:1050800010BC1A89FFF777BEA2160020F8B51C4B9A
:105090009A7912F0F00F0CD15A7952B14FF00A0CF4
:1050A000184A194912780D781E885F88174CAA4251
:1050B00000D1F8BD0CFB02F1601890F804E0BEF1DD
:1050C000000F19D0615AB14216D14179A1B9418876
:1050D000C91B89B2C7290FD80122997962F3071138
:1050E0009971837962F3071383710548FFF7C6FD51
:1050F000BDE8F840FFF796BF013202F00702D6E79D
:10510000A2160020FD160020FC160020AC16002080
:10511000F0B50A270D4B0E4A1B7816780D4CB3429A
:1051200002D100221046F0BD07FB03F5621992F888
:1051300001C08C4505D1655D854202D15279002AB6
:10514000F0D1013303F00703E9E700BFFD160020AB
:10515000FC160020AC1600202DE9F04F8BB002ABFE
:105160000446014606221846FBF7FAF9B34D0346FA
:10517000297922796779A846C1B9AAB18FB12046A9
:10518000FFF7E2FD064660B10A2221462846FBF7FA
:10519000E7F92846FFF762FBFFF778FFFFF766FFA6
:1051A00069E02046FFF76AFD012664E0B4F802A03A
:1051B00068886E79AAEB000094F800B094F801902A
:1051C00080B2002E00F0FB80C72800F2A380002AE6
:1051D00051D0AB792A8813F0F00F20885CD190422F
:1051E00012D12989228991420ED1002F4DD101225D
:1051F00062F30713AB71FFF739FF2846FFF73EFD57
:10520000AB79A371002636E0002F3ED149465846BF
:10521000FFF77EFF5846FFF77BFF05460028F1D1D8
:105220008DF808B08DF809900298FFF7ABFEC0F337
:1052300003310B2912D801228A4012F4406FC3B205
:105240001DD112F00C0F0ED1910707D010F4706F22
:1052500000D07BB12033DBB2072B0BD92046FFF700
:105260000DFD354606E010F4706FF3D0A27912F010
:10527000F00FEFD12E4630460BB0BDE8F08FEF2B8C
:10528000F8D90F33DBB2022BE7E798F8063043F08A
:10529000010388F80630B5E790420ED128892289AB
:1052A00090420AD14FB92046A371FFF7E7FC0A22CA
:1052B00021462846FBF754F970E72046FFF744FDE6
:1052C00000283FF46EAF002F3FF46BAF98F8063024
:1052D0001F2B15D9B8F800208DF81630ADF8102026
:1052E00098F80420B8F808308DF814200022ADF8A2
:1052F00012A08DF81520ADF8183004A8FFF7BEFCF9
:105300000A2221464D48FBF72BF9FFF7BFFEFFF7B6
:10531000ADFE49E7A87910F0F001019118D18DF8A0
:105320000C208DF808B08DF80990ADF80AA08DF822
:105330000D7093E80300FFF718FD2846FFF79EFC69
:105340000A2201992846FBF781F9FFF78FFE59E7FA
:10535000002A90D02A8823889A420ED12A8923894C
:105360009A420AD14FB9A0712046FFF787FC0A2262
:1053700039462846FBF76AF97DE72046FFF7E4FC4B
:1053800000283FF40EAF002F3FF40BAF98F8063023
:105390001F2BB5D9B8F800208DF82230ADF81C20AD
:1053A00098F80420B8F808308DF820200022ADF8D5
:1053B0001EA08DF82120ADF8243007A89EE7C7284D
:1053C0003ED8002A3FF4F0AE3E46002F3FF4E9AE4F
:1053D0002A8823889A4220D12A8923899A421CD17B
:1053E000AB79DA0713D413F0F00210D0F02AA371CE
:1053F00006D0DBB2C3F30312013262F30713A371C9
:105400002046FFF73BFC0A2221460C4852E70A22BD
:1054100021460A48FBF7A4F82DE72046FFF794FC45
:1054200000287FF46DAF98F80630204643F0010362
:1054300088F80630FFF722FC1DE700BFA216002007
:105440008DF80C208DF808B08DF80990ADF80AA001
:105450008DF80D7093E80300FFF787FC0A223146B0
:105460002846FBF7F3F899E6F0B589B001AC84E87B
:1054700007002046FFF770FE294E0746294D70B100
:105480009DF808301BB194E80700FFF774FC0A246C
:10549000254F28783378834226D109B0F0BD05AB7B
:1054A00094E8070003C31A809DF80830002BEED063
:1054B00033782A785C1C04F0070494420AD00A224C
:1054C000194805A902FB0300FBF74AF83470FFF7FF
:1054D000A9FDDCE7FFF708FC0A22394613483770BC
:1054E0002F70FBF7B3F8D2E704FB0070FFF734FE30
:1054F0000028D2D02A786243BB18B85AB3F802C049
:105500009A88D98840EA0C4042EA01411A89FFF79B
:1055100032FC2B78013303F007032B70B9E700BF8F
:10552000FC160020FD160020AC160020A21600205C
:10553000024B0146186805F089B900BFC40F00206E
:10554000024B0146186805F099B900BFC40F00204E
:10555000014B186805F0AAB9C40F0020014B187858
:10556000C00870473E170020024B187800F0070073
:10557000704700BF3E170020034B187810F007005B
:1055800018BF0120704700BF3E170020014B18785C
:10559000704700BF41170020024A1378184310706B
:1055A000704700BF41170020024A137823EA000029
:1055B00010707047411700200022014B1A7070478D
:1055C00041170020024A137818431070704700BF3B
:1055D00042170020024A137823EA00001070704737
:1055E000421700200022014B1A707047421700201A
:1055F000704708B5FFF7FCFF08BD000008B5054A75
:105600001378034204D023EA00001070FFF7F1FF83
:1056100008BD00BF3F170020704708B5FFF7FCFF2B
:1056200008BD000008B5054A137830EA030C03D022
:1056300003431370FFF7F1FF08BD00BF40170020C0
:1056400008B5054A1378034204D023EA000010701D
:10565000FFF7E3FF08BD00BF4017002008B5044B6B
:105660001A781AB100201870FFF7D7FF08BD00BFE5
:105670004017002010B5124B12491B780978124CC4
:105680000B43124920680978037031B10B43037052
:1056900005F056F808B1FFF7E1FF246820220C4915
:1056A0002046FAF72DFF48B1214620220848FAF794
:1056B00057FF2046BDE8104004F0E8BF10BD00BF12
:1056C0004117002042170020C40F0020401700207F
:1056D0001E170020704708B5FFF7FCFF08BD00004B
:1056E000094A10B5527852070AD5084C41EAC00160
:1056F0002170FFF787FB2078C008FFF7ECFF10BD93
:10570000BDE81040FFF77EBB782F00203E17002039
:10571000002008B5024B1870FFF7DDFF08BD00BF81
:105720003E17002008B50A4A137823EA00001070DB
:1057300042070CD198420AD0064B5B785B0706D52E
:10574000C008FFF76BFBBDE80840FFF7E1BF08BDED
:105750003E170020782F0020094A08B55378C3F37C
:10576000800181420AD060F382035370108800F0F8
:1057700040F8BDE808400220FFF7D4BF08BD00BFD5
:10578000782F0020044B5878C0F3800080F001008F
:1057900000F00100FFF7E0BF782F00200120FFF7A5
:1057A000DBBF0020FFF7D8BF08B500F0CFFFBDE892
:1057B00008404FF6FF71002000F0AABF08B5002096
:1057C00000F03FFF4FF6E663984203D1BDE8084082
:1057D00003F0F7BE002008BD022000F023BF032025
:1057E00000F020BF0146032000F084BF042000F039
:1057F00028BF0146042000F08BBF0F2000F030BF0F
:1058000001460F2000F092BF132000F029BF01468F
:10581000132000F08BBF0020FFF7F9BF08B5002070
:10582000FFF7EEFFFFF7F7FF08BD000013B50024F8
:1058300000F08CFF4FF6E661002000F069FF0021C8
:10584000022000F057FF0021032000F053FF1C4B03
:105850004FF4A05104201C7000F05AFF214606208E
:1058600000F048FFFF21072000F044FF21460820F8
:1058700000F05CFF2146242000F03CFF2146172069
:1058800000F038FF21460C2000F034FF21460D20A7
:1058900000F030FF002300226846CDE900231821E4
:1058A000082200F00DFF2146202000F03FFF204697
:1058B00003F09BFE03F0BEFEFFF7B0FF02B010BD89
:1058C00072160020FFF7B2BF01460E2000F012BF93
:1058D00073B505F0D7F80B4C0546238883420ED0EC
:1058E0000026ADF8006005F0CDF8ADF80460ADF825
:1058F000020002AB13E90300FEF78CFF258002B023
:1059000070BD00BF4C17002008B505F081F8024BB0
:105910001860024B186008BD44170020481700208B
:10592000704770470120704708B5054800F090FAAD
:1059300000F00AFFFFF7F4FFFCF7F2FC08BD00BF20
:10594000495E00080120704708B5FFF7FBFF08BD5E
:1059500008B5FDF7E7F9FDF7C7FE08BD08B500F08B
:1059600097FAFEF72CFFBDE8084003F035BB0000B6
:1059700008B505F04BF803F06DFE00F059FBFFF79A
:10598000EDFF054B1A7842F080021A701888FFF775
:1059900030FFFDF79BFD08BD782F00202DE9F04F6B
:1059A00085B0FFF7BFFF60B9FFF792FF04F06EFA12
:1059B00003F086FA00F070FD05B0BDE8F04FFEF789
:1059C00013BF2F4E00F04EFB37460024E0B257F8CD
:1059D000045B00F087FA062C4FD0854204F10104E5
:1059E000F4D0284B1B789B0701D500F081FAFFF714
:1059F000ABFF00254FF0010B00905FFA85F84046A1
:105A000000F070FA56F8043B074698422FD0002465
:105A10004FF0010943400193019B13EA090F1ED087
:105A2000009B17EA090F14BF4FF0010A4FF0000A5C
:105A300083B18DF808408DF8098005F023F88DF8C2
:105A40000CB0ADF80A008DF80DA002AB93E803008E
:105A5000FEF7E0FE52462146404602F0EBFE0134DE
:105A6000E4B2112C4FEA4909D6D146F8047C01353D
:105A7000072DC2D1FFF748FF98E78542B1D193E7E0
:105A8000501700206C17002038B500F0F3F8B0F57F
:105A9000A04F044622D2B0F5804F77D2DF2812D82B
:105AA000CD2861D2A7280AD8A5284ED2012804D033
:105AB00003B233B1032898BF0024204638BDC22862
:105AC0004AD90024F9E7B0F5005F80F0A280B0F574
:105AD000807F4DD2E82828BF0024EEE745F25F23FF
:105AE000984216D845F2402398425FD245F21F23D0
:105AF000984254D8B0F5A44F7CD30123C4B2A00877
:105B000004F0030403FA04F444EA401444F40D449A
:105B10002CE045F29F23984207D8B0F5A54F52D309
:105B200000F01F044AF2F4003DE045F2BF23984222
:105B300056D945F2DF239842C3D8040204F4F8543E
:105B400044F4204444F0F004B7E75B34394BE4B24A
:105B50001C5D44F48044B0E75834374BE4B233F86A
:105B6000144044F48844A8E740F4A044A4B2A4E755
:105B7000C0F3072000F006F90546E0B200F07AF81D
:105B80002D0205F4F855284384B296E7C0B200F020
:105B900071F804F47064044344F42044E6E700F030
:105BA0001F044AF2F10040EA042486E70123C4B24C
:105BB000C4F3820004F0030403FA04F444EA40143A
:105BC00044F40C44D2E70123C4B2C4F3820004F0CD
:105BD000030403FA04F444EA401444F40A44C5E715
:105BE00000F01F0000F0CEF8040204F4F85444F46E
:105BF000005462E700F01F0000F0C4F8C306C4F3CD
:105C0000431448BF0001240200B2044344F410448A
:105C1000ACE7C0F3042000F0B5F80546E0B200F0B0
:105C200029F82D0205F4F85545EA000444F400541F
:105C30009CE700BFB8EB0008BCEB000882B0ADF8F1
:105C40000410C1F30721062906D89DF80420102A64
:105C500002D802B004F03EBB002002B0704707B586
:105C6000ADF804100199FFF7E9FF03B05DF804EB0C
:105C7000FFF70ABF822825D00CD8312867D004D876
:105C800029285AD02A2869D07047352850D0392879
:105C900018D07047E32833D004D8E0281CD0E2287D
:105CA00029D07047E62835D0E72838D0E42835D108
:105CB000334B5A78910731D51B7813F0100F08BF7A
:105CC000E72015E02E4B1A78920752D15B7813F03B
:105CD000080F18BF29207047294A1378D90744D4E0
:105CE000527812F0010F19D013F0100F08BFE32003
:105CF00018BF00207047224B1B7813F0040FF2E707
:105D00001F4A1378590732D45278D20731D413F08E
:105D1000100FEDE71A4B1B781A07CED47047184ABC
:105D20001378190727D452789107F0D5E4207047EB
:105D3000134B1B7813F0200FCBE7114B1A78920608
:105D40001BD45B7813F0080F18BF392070470C4B39
:105D50001B7813F0400F18BF2A207047084B1B78A0
:105D600013F0400F18BF3120704739207047E220F0
:105D70007047E0207047E62070473520CEE700BF2F
:105D8000782F002010B52F4C21784B0713D500F049
:105D90001402A2F1040C00F01803DCF1000242EB43
:105DA0000C02A3F1080CDCF1000343EB0C039A4254
:105DB00018BF80F00C000B0713D500F01402A2F1FD
:105DC000140C00F01803DCF1000242EB0C02A3F10A
:105DD000180CDCF1000343EB0C039A4218BF80F06F
:105DE0000C006478E30713D500F0110202F1FF3CC8
:105DF00000F01803DCF1000242EB0C02A3F1080CE6
:105E0000DCF1000343EB0C039A4218BF80F0090059
:105E1000A30711D500F0110200F01803A2F111043C
:105E20006242A3F1180C6241DCF1000343EB0C0366
:105E30009A4218BF80F00900CB0648BF00F0E70087
:105E400010BD00BF782F0020002070470020704751
:105E5000014B1860704700BFC80F0020FFF7A4BCBB
:105E600008B500F0FFF8C82005F099FE00F0FAF838
:105E7000002000F037F8C30705D5FFF7EFFFBDE8B6
:105E8000084004F023BE08BD08B5FFF7E9FF08BDD0
:105E900008B5FFF793FC08B9FFF714FDFFF79CFC6A
:105EA000084B1870FFF7A2FC074B1880FFF7ECFFB8
:105EB000FFF795FCFEF773FF044B1878BDE8084028
:105EC000FEF789BF6C170020782F00207316002082
:105ED000704708B5FFF7FCFF08BD704708B5FFF72E
:105EE000FCFF08BD014B53F820007047982F00209D
:105EF00070474FF4076005F08BBC00BF00BF00BFC8
:105F000000BF00BF00BF00BF00BF00BF00BF00BF99
:105F100000BF00BF00BF00BF00BF00BF00BF704791
:105F200008B5FFF7E6FF08BD08B5302383F31188F5
:105F3000012100F00F039940202220F00F0006F00D
:105F40008DFF002383F3118808BD000038B51124AC
:105F50000B4D55F8040B421C01D0FFF7E5FF013C47
:105F600014F0FF04F5D10724064D55F8040B431C2B
:105F700001D0FFF7D9FF013C14F0FF04F5D138BD83
:105F8000F4EB000838EC00082DE9F843264D0E46E6
:105F900055F8211080464B1C174642D0302383F31E
:105FA0001188012221F00F0901F00F0102FA01F41A
:105FB00021464846240406F051FFC9F81840002441
:105FC00084F31188FFF799FF6FEA070C1748A8F1CF
:105FD000040208F1180850F8041B52F8043FB1F10C
:105FE000FF3F1AD021F00F0EDEF810E001F00F0194
:105FF0002EFA01F1C90710D401243B4313609045E8
:10600000E9D155F82600431C01D0FFF78DFF21464A
:106010003046BDE8F843FFF783BF0CEA0303136083
:10602000EDE7BDE8F88300BFF4EB000838EC0008AA
:1060300010B51C24FFF78AFF224600210748FAF713
:1060400005FB224600210648FAF700FB072000F076
:106050003FF8BDE81040FFF73CBF00BF982F00207D
:106060007C2F002070B588B01C22002101A8FAF70F
:10607000EDFA002401252A46E1B201A80134FFF718
:1060800083FF112C4FEA4505F5D11C2201A90E48CA
:10609000FAF736FA002814BF0126002607D00A4D69
:1060A00001AC0FCC0FC594E8070085E80700334624
:1060B00007220649044800F00DF80446FFF70EFFDA
:1060C000204608B070BD00BF7C2F0020982F002014
:1060D000704700002DE9F04180460F461546124EEC
:1060E0002BB10123337004F093FC104B186034780B
:1060F0001CB900242046BDE8F0810C4B186804F060
:10610000CDFC0028F5D0AD002A4641463846FAF7C6
:10611000F7F938B12A4641463846FAF721FA002302
:106120003370E7E70446FAE76D1700207017002088
:1061300008B505F013F9FFF71BFCBDE8084005F0B2
:1061400023B908B505F026F9FFF728FCBDE808409B
:1061500005F022B908B504F01DFC05F0FDF8FFF7C5
:10616000E3FBFFF7E5FFFFF7ECFFFFF7F1FBFAE7D3
:1061700000EB4003C3EB031300EB830003B2002BDF
:1061800007DAB3F1800001D503F17F0040F3072067
:10619000704703F18000F9E7164B1B78D90707D544
:1061A000154B187840007F281FD800B3C0B2704745
:1061B0009A0703D5104B18788000F4E75B0703D5E6
:1061C0000D4B1878C000EEE70C4B1B785BB10C4A06
:1061D0000949127808789342F4D25843C000B0FBC2
:1061E000F2F080B2DFE70820E0E77F20704701206F
:1061F000704700BF7E170020CE0F00207F170020C1
:10620000CF0F0020144B1B78D90705D5134B1878F6
:106210008008F8B1C0B270479A0703D50F4B1878C1
:106220004008F6E75B0705D50C4B18787F28F0D9B6
:106230007F2070470A4B1B7853B10A4A07491278EE
:106240000878934236BF584380B2B0FBF2F0EDE7D6
:106250000120DFE7012070477E170020D20F0020C9
:1062600080170020D30F0020CD2808B505D1FFF7F7
:1062700093FF4042294BD87008BDCE2802D1FFF7CA
:106280008BFFF7E7CF2805D1FFF786FF4042234B6E
:106290009870F1E7D02802D1FFF77EFFF7E7D92801
:1062A00004D1FFF7AFFF1D4B1871E5E7DA2803D1E2
:1062B000FFF7A8FF4042F6E7DB2805D1FFF7A2FF72
:1062C0004042164B5871D7E7DC2802D1FFF79AFFFE
:1062D000F7E700F12F03DBB2072B08D801230F4AA1
:1062E000D13803FA00F0537818435070C4E7DD2822
:1062F00005D10B4A137843F001031370BCE7DE2885
:1063000004D1074A137843F00203F6E7DF28B3D13C
:10631000034A137843F00403EFE700BF7817002027
:106320007E170020364BCD2893F902200AD193F92D
:10633000031000290CDA0021D97052B90021314A2A
:10634000117006E0CE280DD193F903100029F2DC7C
:1063500072B11A795B7913435BB2002B4FD12A4A91
:1063600013707047CF2806D1002AF1DA00229A7004
:1063700093F90320E1E7D02802D1002AF6DCE7E711
:10638000D92893F9041004D10029E1DD0021197105
:10639000DEE7DA2802D10029DADAF7E7DB2893F919
:1063A000051004D10029D3DA00215971D0E7DC2887
:1063B00002D10029F8DCCBE700F12F01C9B207298F
:1063C00007D80121D1388140587820EA010058705F
:1063D000BEE7DD2805D10D48017821F001010170EB
:1063E000B6E7DE2804D10948017821F00201F6E77A
:1063F000DF28ADD10548017821F00401EFE77047AF
:10640000781700207F170020801700207E170020BB
:1064100008B504F037FB094BDA7899780A431CBFBA
:10642000074A10801A795B7913431CBF054B18800B
:106430000248BDE8084004F041B900BF78170020C9
:10644000741700207617002008B5062200210548A1
:10645000FAF7FCF80023044A1370044A1370044A44
:10646000137008BD781700207F17002080170020C8
:106470007E17002090F902305BB990F9033043B9E0
:1064800090F904302BB990F90500003018BF0120B5
:10649000704701207047000037B5594C062221464D
:1064A0006846FAF75DF800239DF80220A370E370B8
:1064B000237163719DF8033013430AD0514B188840
:1064C00004F0E5FA504A13783BB350490978884202
:1064D0002CDC9DF804209DF8053013430BD04C4B69
:1064E000188804F0D4FA4B4A1378002B4ED04A494E
:1064F0000978884253DC6946414804F0EBF918B941
:106500003F48FFF7B7FF08B1FFF782FF0622694651
:106510003B48FAF725F803B030BD40490D780A2111
:1065200069438842D5DD0133137001E0FF2BFAD1B6
:106530009DF902503DB1FFF72FFE002DCCBF012386
:10654000FF235843A0709DF903503DB1FFF724FE8F
:10655000002DCCBF0123FF235843E07094F90200C3
:106560000028B6D094F90320002AB2D0FFF700FE2D
:1065700030B1A0701046FFF7FBFD20B1E070A8E736
:106580000123A370F6E70123E370A2E724490D7805
:106590000A2169438842AEDD0133137001E0FF2B0D
:1065A000FAD19DF904503DB1FFF72CFE002DCCBF70
:1065B0000123FF23584320719DF905503DB1FFF79A
:1065C00021FE002DCCBF0123FF235843607194F9B5
:1065D000040000288FD094F90520002A8BD0FFF703
:1065E000C7FD30B120711046FFF7C2FD20B16071C8
:1065F00081E701232371F6E7012363717BE700BF85
:1066000078170020741700207F170020CD0F00207E
:106610007617002080170020D10F0020CC0F00201B
:10662000D00F0020002307B5014601220DF107001D
:106630008DF8073000F08CF89DF8070003B05DF886
:1066400004FB002307B5014602220DF10600ADF858
:10665000063000F07DF8BDF8060003B05DF804FBDD
:1066600007B50422002301460DEB0200019300F060
:106670006FF8019803B05DF804FB07B501228DF8AF
:10668000071001460DF1070000F067F803B05DF850
:1066900004FB07B50222ADF8061001460DF1060015
:1066A00000F05BF803B05DF804FB07B5042201912C
:1066B00001460DEB020000F050F803B05DF804FB5A
:1066C000F8B505461446D31D23F0070300AFADEB24
:1066D000030D68460E4600F03BF822466946284600
:1066E000F9F70EFF20B122463146284600F035F872
:1066F000BD46F8BD38B50C460546FFF793FFA042EE
:1067000005D021462846BDE83840FFF7B6BF38BD62
:1067100038B50C460546FFF794FFA04205D0214648
:106720002846BDE83840FFF7B4BF38BD38B50C4641
:106730000546FFF795FFA04205D021462846BDE853
:106740003840FFF7B2BF38BD00F01EB900F03CB8CA
:106750000B460146184600F051B80B460146184654
:1067600000F09EB808B5064B4FF4006200211846B1
:10677000F9F76CFF40F60802C0F8002808BD00BF1A
:106780008817002010B5064C94F8043833B900F08F
:1067900076F910B1012084F8040810BD0220FCE74E
:1067A0008817002010B5074C94F804383BB100F06E
:1067B00070F918B10023012084F8043810BD0220BC
:1067C000FCE700BF8817002038B5FFF7DBFF044661
:1067D00018B9FFF7E7FF204638BD00F052F905462B
:1067E000FFF7C0FF012C06D1FFF7DCFF00280CBF2C
:1067F000002505F001052C46EDE7000008B503462D
:1068000008469918B1F5006F05D804491944F9F7FD
:10681000A7FE012008BD0020FCE700BF881700206C
:1068200038B5FFF7AFFF4FF48072054610490020DE
:1068300000F04CF970B10CA3D3E900234FF40061D0
:106840000B4803F05BF802460B464FF4006000F083
:1068500076F930B90024012D01D1FFF7A3FF2046BE
:1068600038BD0224F7E700BF25232284E49CF2CB45
:106870008817002010B5094CD4F80038B3F5805FB4
:1068800009D300F0FEF828B1FFF7CAFF40F608036D
:10689000C4F8003810BD0120FCE700BF88170020B5
:1068A0008318B3F5006F2DE9F74F06460D461746DE
:1068B00004D90024204603B0BDE8F08FDFF8C08083
:1068C00008EB000421462846F9F71AFE002854D0A8
:1068D0003A4629462046F9F743FEFFF753FF824622
:1068E00028B14FF0000B2FB9FFF7C4FF29E0FFF7E5
:1068F00059FFDEE7052FB94628BF4FF00509C6F35B
:10690000024343EAC9038DF80030330AADF802B000
:106910008DF80130ADF804B0ADF806B08DF8026026
:106920000DF1030305EB090215F8011B954203F86D
:10693000011BF9D1DDE90023D8F8000800F0FFF8C9
:1069400008B9044611E0D8F800380833C8F8003810
:10695000FFF790FF0128044603D1A7EB09074E4437
:10696000C1E710B1022818BF0024BAF1010FA1D16C
:10697000FFF718FF00289CD09CE701249AE700BF8E
:106980008817002000000000F0B585B0FFF7EAFE90
:1069900000F070F820B9FFF7E5FE002005B0F0BD6B
:1069A0004FF480723249002000F075F8304E10B973
:1069B000FFF7D8FEEFE72CA3D3E900234FF40061E3
:1069C000304602F09BFF0D46044602A94FF40060DA
:1069D00000F079F8DDE902239D4208BF944201D01E
:1069E000FFF7C0FE40F608076946384600F06BF82E
:1069F00010B3DDE9004554EA05031CD0E2B2930967
:106A000007F10807CDE9024526D104F47F431004BD
:106A1000C4F307441C4300F4E0202043D208831849
:106A2000B3F5006F18D80DF10B013044F9F798FD5C
:106A3000B7F5805FD8D10120C6F8007870B900F0B2
:106A400020F80028A7D0FFF7EBFE40F60803C6F8B1
:106A500000380028A2D19EE70020EDE7FFF70AFFEB
:106A6000F7E700BFAFF3008025232284E49CF2CB3C
:106A70008817002008B500F0D1F8012008BD0120DA
:106A8000704708B5002000F0CBF8B0FA80F040095C
:106A900008BD0120704738B5D5002A460C4600F0E5
:106AA000DCF818B921462544A94203D1B0FA80F098
:106AB000400938BDD1E90023D243DB4341F8082B1C
:106AC00041F8043CF0E70122FFF7E5BF2DE9F04370
:106AD0000746884615460026C1B06B46202DAE46B7
:106AE00028BF4FF0200E1C469C4608EBC602764499
:106AF00008EBC6094A4511D10024744513D14FEA69
:106B0000C4094A466146384600F0C5F8A8B92D1BAD
:106B10004F44E2D1012041B0BDE8F083F2E8020128
:106B2000E4E80201E6E7D3E90002C043D24343F8B8
:106B3000080B43F8042C0134DFE70020EBE707B52E
:106B4000CDE9002369460122FFF7C0FF03B05DF8DD
:106B500004FB0000002208231146014804F06CB831
:106B60000C08004008B5FFF7F5FF30B1062004F02F
:106B7000A1F804F0D7F8002008BD4FF0FF30FBE784
:106B800038B503F045FF00F57A75FFF7E3FF78B1FC
:106B9000052004F08FF804F09FF8C4B204F0C2F8A6
:106BA00003F036FFA84206D214F00100EDD138BD43
:106BB0004FF0FF30FBE76FF00100F8E7F7B51F4635
:106BC0004BBA090C064615468DF80400ADF80630A0
:106BD0008DF80510FFF7BEFFE8B104210DEB0100B1
:106BE00004F08CF8044648B945B1022E0BD0032EB0
:106BF0000ED1B9B2284604F08BF8044604F092F89E
:106C0000204603B0F0BDB9B2284604F077F8F4E7A7
:106C10004FF0FF34F2E74FF0FF34F1E703F0D0BF5D
:106C200000F58033B3F5002F10B5044612D283B2BD
:106C300083B9FFF7A5FF78B9FFF794FF60B9034662
:106C400002462146D820FFF7B9FF28B9BDE8104019
:106C5000FFF796BF4FF0FF3010BD2DE9F0418046A1
:106C60000D461646FFF78CFF0446074638B13246FC
:106C700000212846F9F7EAFC2046BDE8F0813346BA
:106C80002A4641460320FFF799FF04460028F3D027
:106C900032463946EDE72DE9F0410746884616466B
:106CA00076B9FFF76DFF044638B9FFF753FF20B3FD
:106CB000042003F0FFFF04F035F82046BDE8F08122
:106CC000FDB2C5F58075B54228BF3546FFF758FFC0
:106CD00004460028F1D1FFF745FF04460028ECD117
:106CE0002B46424639460220FFF768FF044600283B
:106CF000E3D1A8442F44761BD2E74FF0FF34DCE702
:106D000030B5C0F3072285B00190C0F30740BAB98F
:106D100009B1304B185C8DF80C008DF80D008DF822
:106D20000E0000209DF80C3063F307009DF80D3035
:106D300063F30F209DF80E3063F3174005B030BDAC
:106D40009DF8043061B32349085C0625FF215D43AB
:106D50006FF05404B5FBF1F56C4304EB430404EB12
:106D60004404E4B204FB02F3C4F1FF04891A624351
:106D70001B121212C3F1FF03C2F1FF02414343434E
:106D80004243C1F30721C3F30723C2F30722C0B272
:106D9000062D19D8DFE805F00608110F14180600B3
:106DA00080B2D2E7034610468DF80C008DF80D3006
:106DB0008DF80E10B5E7024618460B461146F3E76C
:106DC000134602460846F9E70246084619461346A6
:106DD000EAE700BF6CEC0008012184B004B0FFF7C3
:106DE0008FBF012830B501D8C0B230BDB0F5F75F14
:106DF00088BFFF224FF001019EBF42090832D2B284
:106E00008B185B1003FB03F5ADB28542DCB205D9EC
:106E1000621ED2B29142F3D9481EE5E7FF2B02D0A1
:106E2000611CC9B2F6E71846DFE70000074B188877
:106E300000EB402200EB820000F55850193080B280
:106E4000188000EB1020C0B2704700BFDA0F00209E
:106E500010F0400116BFC3430346DBB210B503F088
:106E60000F0201B101320949C3F301135B00CC18D1
:106E70006478CB5C624303EB2213DBB2020644BFAF
:106E80005B42DBB283F0800010BD00BF54EC000811
:106E9000144B84B003EB4101E423019091F8771087
:106EA000C0F307204B43C2EB13231C33002BB8BFA6
:106EB0005B42A0EBC3031BB223EAE3735843001207
:106EC0008DF805000020019BDAB262F30700C3F3DE
:106ED000072262F30F20C3F3074363F3174004B0A4
:106EE000704700BF440D0020144B84B003EB4101F8
:106EF000E423019091F87710C0F307404B43C2EBB5
:106F000013231C33002BB8BF5B42A0EBC3031BB29F
:106F100023EAE373584300128DF806000020019B1A
:106F2000DAB262F30700C3F3072262F30F20C3F360
:106F3000074363F3174004B0704700BF440D0020BF
:106F400084B0019000208DF80420019BDAB262F336
:106F50000700C3F3072262F30F20C3F3074363F371
:106F6000174004B07047000084B0019000200B4B24
:106F700003EB410191F877309A1A8DF80420019BB8
:106F8000DAB262F30700C3F3072262F30F20C3F300
:106F9000074363F3174004B0704700BF440D00205F
:106FA00084B0019000200B4B03EB410191F8783045
:106FB0009A1A8DF80420019BDAB262F30700C3F33A
:106FC000072262F30F20C3F3074363F3174004B0B3
:106FD000704700BF440D002030B5134B85B03831E9
:106FE000019003EB4104257A03EB4103A5F1200452
:106FF00064B2002CDB79BCBFC5F1200464B29B1ADB
:10700000C0B22344034400208DF80430019BDAB25F
:1070100062F30700C3F3072262F30F20C3F30743B1
:1070200063F3174005B030BD440D002084B00190DB
:1070300000209DF8102003EB430302EB53028DF870
:107040000420019BDAB262F30700C3F3072262F364
:107050000F20C3F3074363F3174004B070471FB515
:1070600092B2019048B2002802FB02F2BCBF484233
:1070700040B2C0F1380000FB002080B21C46FFF790
:10708000B0FE00EB4000044400208DF80440019B5A
:10709000DAB262F30700C3F3072262F30F20C3F3EF
:1070A000074363F3174004B010BD000084B00190A3
:1070B00003F13800104B03EB4003187ADB792038DA
:1070C000703B594302FB00120020002A9DF8041077
:1070D000B8BF7F3201EBE2128DF80420019BDAB2D7
:1070E00062F30700C3F3072262F30F20C3F30743E1
:1070F00063F3174004B07047440D002084B0019042
:1071000003F13800104B03EB4003187ADB79203889
:10711000703B594302FB00120020002A9DF8041026
:10712000B8BF3F3201EBA2128DF80420019BDAB206
:1071300062F30700C3F3072262F30F20C3F3074390
:1071400063F3174004B07047440D00201FB503F1EE
:107150003804164B019003EB44031C7AC0B2203C68
:107160006243DC79A4F170035BB2002BBCBFC4F1B5
:1071700070035BB2C3F1380301FB032111EB410142
:1071800048BF7F3100EBE11100208DF80410019B16
:10719000DAB262F30700C3F3072262F30F20C3F3EE
:1071A000074363F3174004B010BD00BF440D002037
:1071B00030B50D4685B00190C4B21046FFF748FEC9
:1071C000124B0C2203EB450393F877301844C0B2FE
:1071D000A0F180035BB2002BBCBFC0F1800043B2C2
:1071E00000205B00DBB2534304EB13248DF8044012
:1071F000019BDAB262F30700C3F3072262F30F20A8
:10720000C3F3074363F3174005B030BD440D0020BE
:10721000114B84B0019003EB410191F87710C0B29B
:107220008B1A5BB2002BBCBF521A53B21822DBB2CE
:10723000534300EB13208DF804000020019BDAB2C9
:1072400062F30700C3F3072262F30F20C3F307437F
:1072500063F3174004B07047440D0020054B40F61F
:10726000B8301B791033FF2B28BFFF231B09B0FB5D
:10727000F3F07047B82F0020C94384B00190C9B221
:10728000C0F30740484300128DF806000020019B20
:10729000DAB262F30700C3F3072262F30F20C3F3ED
:1072A000074363F3174004B0704784B0C9B201903C
:1072B000C1F18201C0B20029A8BF40188DF80400B6
:1072C0000020019BDAB262F30700C3F3072262F3E6
:1072D0000F20C3F3074363F3174004B0704784B033
:1072E000BDF8102003EB830313449BB2FF2B28BF90
:1072F000FF23DB430190DBB2C0F307400344FF2BC5
:1073000028BFFF2300208DF80630019BDAB262F31C
:107310000700C3F3072262F30F20C3F3074363F3AD
:10732000174004B0704700291FB5B8BF4942002A72
:10733000B8BF524209B2090112B2FF294FEA021244
:10734000A8BFFF21FF2AA8BFFF22BDF8184009B23D
:10735000234412B29BB29142D4BF5B189B189BB2DC
:10736000FF2B28BFFF23DB430190DBB2C0F30740B4
:107370000344FF2B28BFFF2300208DF80630019B1C
:10738000DAB262F30700C3F3072262F30F20C3F3FC
:10739000074363F3174004B010BD00001FB5482B2E
:1073A0000190C0F3074030D8BDF81840E31A9BB2F3
:1073B000FF2B28BFFF23083189B2102905D902F11C
:1073C000080189B2112928BFFF23DB43DBB2034444
:1073D000002AB8BF0332FF2B28BFFF2300200C492F
:1073E0008DF80630497801EBA2028DF80420019B4C
:1073F000DAB262F30700C3F3072262F30F20C3F38C
:10740000074363F3174004B010BDFF23D3E700BF69
:10741000B82F002084B0BDF810200190D31A9BB281
:10742000FF2B28BFFF23DBB2D943C0F30742C9B209
:107430000A44FF2A28BFFF2218448DF804000020C8
:107440008DF80620019BDAB262F30700C3F307222E
:1074500062F30F20C3F3074363F3174004B0704790
:1074600084B0BDF810200190D31A9BB2FF2B28BF27
:10747000FF23DB43C0F30740DBB20344FF2B28BFED
:10748000FF2300208DF80630019BDAB262F307007B
:10749000C3F3072262F30F20C3F3074363F31740DC
:1074A00004B07047024A137818431070704700BF49
:1074B000921F0020012310B5044C08221821044813
:1074C0002370FFF745F90023237010BD921F0020A1
:1074D000B82F002028B90029ACBF0023802318460C
:1074E000704780EAE072A2EBE072002912B201EB71
:1074F0000203ABBF891A5B014901511AABBF91FB73
:10750000F3F393FBF1F3C3F12003C3F160035BB228
:10751000DBB20028BCBF5B42DBB2E0E730B5C0F3B2
:10752000072585B0EB1A01901046DCB2FFF7D2FFB9
:10753000C0EB801300EB830004440020E4B26C43F2
:1075400024128DF80540019BDAB262F30700C3F301
:10755000072262F30F20C3F3074363F3174005B01C
:1075600030BD30B5C0F3074585B0EB1A0190104629
:10757000DCB2FFF7AFFFC0EB801300EB83000444E5
:107580000020E4B26C4324128DF80640019BDAB26D
:1075900062F30700C3F3072262F30F20C3F307432C
:1075A00063F3174005B030BD30B585B09DF820407D
:1075B000C0F30725019010461C1BFFF78BFF2C44DE
:1075C000E4B2201AC0B2684300128DF80500002012
:1075D000019BDAB262F30700C3F3072262F30F20C4
:1075E000C3F3074363F3174005B030BD30B585B032
:1075F0009DF82040C0F30745019010461C1BFFF783
:1076000069FF2C44E4B2201AC0B2684300128DF81E
:1076100006000020019BDAB262F30700C3F30722E1
:1076200062F30F20C3F3074363F3174005B030BD87
:107630001FB5019010461C46FFF74CFF20448DF803
:1076400004000020019BDAB262F30700C3F30722B3
:1076500062F30F20C3F3074363F3174004B010BD78
:107660001FB59DF81840019010461C1BFFF732FF14
:10767000E4B2201A8DF804000020019BDAB262F314
:107680000700C3F3072262F30F20C3F3074363F33A
:10769000174004B010BD000008B5082218210348A7
:1076A000FFF70EF80022024B1A7008BDB82F002019
:1076B000921F002084B004B0FFF78EBB2DE9F74F76
:1076C000334D00EB0017EB195B5C8346FF2B8A46BA
:1076D0002AD000262F4A17444FF0000906EB061463
:1076E00003F13808291905EB4808144411F801EB97
:1076F000BEF1FF0F0ED0F0B2834518D15FFA89F0CA
:10770000824514D117F80A002030FF2828BFFF2037
:1077100007F80A0009F10109B9F1110F04F1010498
:10772000E4D10136072ED7D103B0BDE8F08F0EF1BA
:10773000380E05EB4E0E9EF807C098F807009EF82D
:1077400008E0A0EB0C0098F808C00191ACEB0E0C1F
:107750001FFA8CFC0CFB0CFC00FB00C080B20093F9
:10776000FFF73FFB2828009B01990A4AD2D8C0F1B5
:1077700028001FFA80FC2078BCF1100F94BF6044F1
:10778000103080B2FF2828BFFF202070C2E700BF62
:10779000440D0020941F0020FFF77EBF10B5084C59
:1077A00035232046032200F8013B0649F8F7D8FEAE
:1077B0004FF68073A380BDE81040FFF76DBF00BF98
:1077C000B82F0020AAE400080020704770B50446D6
:1077D0000E461546FFF7F8FF054B04EB04141C4456
:1077E000A35DFF2B1EBF2B540130C0B270BD00BF84
:1077F000440D0020014BDB68184700BF5CEC00081B
:1078000008B5074B074A1870074B1B78C3F30103F1
:107810001370FFF7EFFF0322044B1A7008BD00BF7F
:10782000D70F0020D80F0020B82F0020D90F00203C
:107830005E2817B406DC054C6468A446019403B0C6
:1078400010BC604703B010BC704700BF5CEC000880
:107850002DE9F04F0478824604EBC40304EB4304A3
:10786000E4B204F11307FFB25F2FBB4628BF4FF00D
:107870005F0B2E4D2E4A2E7989B07308168803911E
:107880005E43C6F3072302932A4B03EB440803F23B
:107890003519E3B29B4506D85E2F8CBF002001202E
:1078A00009B0BDE8F08F14F809209AF801301A42A7
:1078B00037D098F8782098F87710203A92B202FBE7
:1078C00002F0703989B201FB010080B20592049187
:1078D000FFF787FA029B95F801C00093AB7895F803
:1078E00003E0059A04994CEA032C12B2034609B24C
:1078F0004CEA0E40039EB047C0F307238DF81C00EE
:10790000C0F307408DF81D308DF81E000798FFF773
:10791000D1FEC0F30743C2B2C0F307212046FFF7F0
:1079200087FF08F102080134B3E700BFB82F002039
:10793000C02F0020440D00200149FFF789BF00BF80
:10794000A97500080149FFF783BF00BFED75000866
:107950000149FFF77DBF00BF2D7000080149FFF707
:1079600077BF00BF617600082DE9F04F04788246AA
:1079700004EBC40304EB4304E4B204F11307FFB2C5
:107980005F2FBB4628BF4FF05F0B254D254A2E7950
:1079900085B07308168801915E43C6F307230093F0
:1079A000214B03EB440803F23519E3B29B4506D89B
:1079B0005E2F8CBF0020012005B0BDE8F08F14F8C9
:1079C00009209AF801301A4225D0AB78687895F8EA
:1079D00003C098F8782098F8771040EA0320203AFE
:1079E0007039009B40EA0C40019EB047C0F307236A
:1079F0008DF80C00C0F307408DF80D308DF80E00A7
:107A00000398FFF757FEC0F30743C2B2C0F3072144
:107A10002046FFF70DFF08F102080134C5E700BF5B
:107A2000B82F0020C02F0020440D00200149FFF78F
:107A30009BBF00BF1D7500080149FFF795BF00BF40
:107A4000637500080149FFF78FBF00BF5F70000832
:107A50000149FFF789BF00BF317600082DE9F74FD4
:107A60000478074604EBC40304EB4304E4B204F1D6
:107A700013095FFA89F9B9F15F0FCA46884628BF32
:107A80004FF05F0A1D4E1E4A3579DFF878B0AB081B
:107A9000158803FB0555C5F30725E1B28A4507D8CC
:107AA000B9F15E0F8CBF0020012003B0BDE8F08F5C
:107AB00014F80B207B781A421DD0B07873782A46D0
:107AC00043EA0023F07843EA0040C047C0F30723AD
:107AD0008DF80400C0F307408DF805308DF80600DE
:107AE0000198FFF7E7FDC0F30743C2B2C0F30721D7
:107AF0002046FFF79DFE0134CFE700BFB82F0020DE
:107B0000C02F0020790E00200149FFF7A7BF00BF5A
:107B1000916E00080149FFF7A1BF00BFE96E0008A0
:107B20000149FFF79BBF00BF416F00080149FFF704
:107B300095BF00BF696F00080149FFF78FBF00BF05
:107B4000A16F00080149FFF789BF00BFD96F000886
:107B50000149FFF783BF00BFB17100080149FFF77A
:107B60007DBF00BF117200082DE9F04F2E4E047842
:107B70002E4A357904EBC40304EB4304AB081588A3
:107B8000E4B25D4304F11307C5F30725FFB2814654
:107B900005F1400087B05F2FC0B20391BA4628BFFD
:107BA0004FF05F0AFFF754F980384FFA80FB284600
:107BB000FFF74EF980384FFA80F80296E3B29A4503
:107BC00006D85E2F8CBF0020012007B0BDE8F08FE3
:107BD000174AA15C99F80120114223D0029A00951E
:107BE00050789278594640EA0220029A039E92F811
:107BF00003C0424640EA0C40B047C0F307238DF86B
:107C00001400C0F307408DF815308DF81600059864
:107C1000FFF750FDC0F30743C2B2C0F3072120466F
:107C2000FFF706FE0134C9E7B82F0020C02F00205F
:107C3000790E00200149FFF797BF00BFAD70000823
:107C40000149FFF791BF00BFFD7000080149FFF730
:107C50008BBF00BF4D7100082DE9F04F0478384DFF
:107C600004EBC40304EB4304E4B22F7904F11306DC
:107C7000F6B27B1C5F2EB24628BF4FF05F0AB3F509
:107C8000807F08BFFF234FF6FF778046B7FBF3F7EF
:107C900085B0DFF8B0B0DFF8B0900191E0B2824576
:107CA00006D85E2E8CBF0020012005B0BDE8F08F05
:107CB00014F80B2098F801301A422FD099F80030B0
:107CC000DFF888C0013B5BB21A0629D53A4629790C
:107CD000A8780131B1F5807F08BFFF216B7851434F
:107CE00043EA0023E878C1F30F2143EA0040019BF7
:107CF0009847C0F307238DF80C00C0F307408DF8B8
:107D00000D308DF80E000398FFF7D4FCC0F3074345
:107D1000C2B2C0F307212046FFF78AFD0134BDE758
:107D200013F80C20824209D103F10C0209EB420244
:107D30005178927841EA0222BA42C8D3013BC3E7A4
:107D4000B82F0020790E0020C42F0020D52F00204E
:107D50000149FFF781BF00BF797200080149FFF7B1
:107D60007BBF00BFAB7200082DE9F04F0C78824654
:107D700004EBC40304EB4304E4B204F11307FFB2C1
:107D80005F2F3B4628BF5F238B46454D8DB0049344
:107D90002B7805920393434B029503EB440803F2BF
:107DA00035130693049AE3B29A4206D85E2F8CBF2D
:107DB000002001200DB0BDE8F08F069BE25C9BF82F
:107DC00001301A4220D0032237490AA8F8F7C8FB2D
:107DD000029B0AF101061E44D146002303995FFA73
:107DE00089F2914214D8314AD07843431B128DF85E
:107DF0002A300A98FFF75EFCC0F30743C2B2C0F313
:107E000007212046FFF714FD013408F10208C9E7F5
:107E100016F8012B98F8770098F878C0801AF27954
:107E200080B2ACEB020C1FFA8CFC0FFA8CF20CFB4C
:107E30000CFC01B200FB00C080B2099308910792CC
:107E4000FEF7CFFF029B09F10C0E03EB4E0E9EF8DE
:107E500001C0164B9EF802E0079A4CEA0E2C93F8EC
:107E600004E0099B0EF1010EBEF5807F08BF4FF0C4
:107E7000FF0E0CFB0EFC8DF82A30CCF30F23009381
:107E800008990346059D0A98A847C0F307238DF873
:107E900029308DF8280009F10109C0F307439DE757
:107EA000C42F0020440D0020B92F0020B82F00203F
:107EB000054B01461B78054A013BB3F1FF3F08BF64
:107EC0000023D8B2FFF750BFC42F0020DF72000894
:107ED0000146024A0020FFF747BF00BFDF720008DB
:107EE000054B01461B78054A013BB3F1FF3F08BF34
:107EF0000023D8B2FFF738BFC42F00202773000833
:107F00000146024A0020FFF72FBF00BF2773000879
:107F1000054B01461B78054A013BB3F1FF3F08BF03
:107F20000023D8B2FFF720BFC42F00209D730008A4
:107F30000146024A0020FFF717BF00BF9D730008EB
:107F4000054B01461B78054A013BB3F1FF3F08BFD3
:107F50000023D8B2FFF708BFC42F00201574000813
:107F60000146024A0020FFF7FFBE00BF157400085B
:107F7000054B01461B78054A013BB3F1FF3F08BFA3
:107F80000023D8B2FFF7F0BEC42F002061740008B0
:107F90000146024A0020FFF7E7BE00BF61740008F7
:107FA0002DE9F34104781E4A04EBC40304EB4304B7
:107FB000064653789078E4B243EA002304F11305AF
:107FC000D078EDB25F2D43EA00402F4628BF5F27EF
:107FD000FFF770FBDFF84C80C0F307238DF8040037
:107FE000C0F307408DF805308DF80600E3B29F42DC
:107FF00006D85E2D8CBF0020012002B0BDE8F081C4
:1080000014F8082073781A4208D09DF806309DF8BD
:1080100004209DF805102046FFF70AFC0134E5E72F
:10802000B82F0020790E00202DE9F0430478DFF806
:10803000BC9004EBC40304EB4304E4B204F1130565
:1080400085B0EDB25F2D4FF0030209F10101064644
:1080500001A82F4628BF5F27F8F782FA99F8018018
:108060008DF804800198FFF725FBC0F307238DF8F6
:10807000093099F804308DF8080098448DF8048090
:10808000C0F307408DF80A000198FFF713FBDFF8F3
:108090006080C0F307238DF80C00C0F307408DF813
:1080A0000D308DF80E00E3B29F4206D85E2D8CBFD6
:1080B0000020012005B0BDE8F08314F80830727884
:1080C000134211D0DB0743BF9DF80E309DF80C2002
:1080D0009DF80D109DF80A305CBF9DF808209DF8B2
:1080E00009102046FFF7A4FB0134DCE7B82F00207D
:1080F000790E00202DE9F74F0478204D04EBC403DE
:1081000004EB4304E4B204F11306F6B25F2E80469A
:108110004FF0030205F101016846B246DFF86090B6
:1081200028BF4FF05F0AF8F71BFA2F79A9F1BD0BB2
:10813000BF08E3B29A4506D85E2E8CBF002001200E
:1081400003B0BDE8F08F14F8092098F801301A4206
:1081500012D01BF814306A781B0903FB07238DF833
:1081600000300098FFF7A6FAC0F30743C2B2C0F38D
:1081700007212046FFF75CFB0134DAE7B82F002027
:10818000790E00202DE9F74F0478214D04EBC4034C
:1081900004EB4304E4B204F11306F6B25F2E80460A
:1081A0004FF0030205F101016846B246DFF8649022
:1081B00028BF4FF05F0AF8F7D3F92F79A9F1BE0B6A
:1081C000BF08E3B29A4506D85E2E8CBF002001207E
:1081D00003B0BDE8F08F14F8092098F801301A4276
:1081E00013D01BF8143007FB03F26B7803EB521328
:1081F0008DF800300098FFF75DFAC0F30743C2B274
:10820000C0F307212046FFF713FB0134D9E700BF75
:10821000B82F0020790E00202DE9F7430478DFF80D
:10822000B89004EBC40304EB4304E4B204F1130577
:10823000EDB25F2D4FF0030209F1010106466846D9
:108240002F4628BF5F27F8F78BF9224B99F80400D7
:108250001B88C0085843C0F30720FEF7F9FDA0F1C2
:1082600080035BB2002BBCBFC0F1800043B299F821
:1082700003805B00DBB208FB03F31B128DF80230B6
:108280000098FFF717FADFF85480C0F307238DF842
:108290000400C0F307408DF805308DF80600E3B206
:1082A0009F4206D85E2D8CBF0020012003B0BDE8A0
:1082B000F08314F8082073781A4208D09DF806302D
:1082C0009DF804209DF805102046FFF7B1FA01340F
:1082D000E5E700BFC02F0020B82F0020790E002056
:1082E00037B5154B04469A7859788DF80120DA781D
:1082F0008DF80220FEF79AFD4FF4B47201F1B40537
:10830000B5FBF2F302FB13535B1A48BF033300F0D3
:1083100003009B1003FB00138DF800300098FFF75B
:10832000C9F9C0F30743C2B2C0F30721204603B026
:10833000BDE83040FFF77CBAB82F00202DE9F041AE
:108340000478064604EBC40304EB4304E4B28378E8
:1083500004F11305EDB22BBB1B4B0A211B791B4A01
:108360001033FF2B28BFFF2312885343C3F30F237F
:10837000B3FBF1F201FB12339BB26BB9FEF756FD72
:108380005F235843124B00120344727893F835313F
:108390001A4201D0FFF7A4FF5E2D8CBF0020012000
:1083A000BDE8F0815F2D2F4628BF5F27DFF82480CE
:1083B000A742F1DD727814F808301A4202D0204644
:1083C000FFF78EFF0134F3E7B82F0020C02F002005
:1083D000440D0020790E002013B50446FEF726FD5B
:1083E0008DF80000FEF722FD0B4B40F35700DB78C1
:1083F0007F308DF802308DF801000098FFF75AF9B0
:10840000C0F30743C2B2C0F30721204602B0BDE863
:108410001040FFF70DBA00BFB82F00202DE9F04142
:108420000478064604EBC40304EB4304E4B2837807
:1084300004F11305EDB233BB1C4B1D4A1B791288A6
:108440001033FF2B28BFFF2353430522C3F30F2311
:10845000B3FBF2F202EB82029B1A9BB26BB9FEF7FE
:10846000E5FC5F235843134B00120344727893F8E2
:1084700035311A4201D0FFF7AFFF5E2D8CBF0020CF
:108480000120BDE8F0815F2D2F4628BF5F27DFF870
:108490002880A742F1DD727814F808301A4202D021
:1084A0002046FFF799FF0134F3E700BFB82F002003
:1084B000C02F0020440D0020790E00202DE9F74345
:1084C0000478DFF8B89004EBC40304EB4304E4B28F
:1084D00004F11305EDB25F2D4FF0030209F1010124
:1084E000064668462F4628BF5F27F8F739F8224B23
:1084F00099F804001B88C0085843C0F30720FEF712
:10850000A7FC0C22A0F180035BB2002BBCBFC0F122
:10851000800043B25B00DBB2534399F8018008EB63
:1085200013288DF800800098FEF756FCDFF8508085
:10853000C0F307238DF80400C0F307408DF8053021
:108540008DF80600E3B29F4206D85E2D8CBF002056
:10855000012003B0BDE8F08314F8082073781A42B4
:1085600008D09DF806309DF804209DF8051020469F
:10857000FFF75EF90134E5E7C02F0020B82F002097
:10858000790E0020014B9B68184700BF5CEC000887
:108590002DE9F04F037885B003EBC30203EB4203F0
:1085A0005FFA83FB0BF113095FFA89F94B465F2BE6
:1085B00028BF5F230093837882464BB10022114687
:1085C0001046FFF7DFFF772200213A48F8F73EF820
:1085D0009AF800306BB9384C208802F058FA182805
:1085E0008CBF01220022354B1A7002D902F04AFAE0
:1085F000208000252C462F4602E0122F52D800245E
:108600002F4A05EB051802EB080319191B5D0191B0
:108610005B453FD300998B423CD2134493F83521FC
:108620009AF8013001371A42FFB233D0214B254A64
:10863000984418F80460A6F1550323EAE373C3F1E4
:10864000AA038DF808309378D2788DF8093006F1B6
:10865000AA03FF2B28BFFF2303EB43030233DBB244
:1086600053431B128DF80A300298FFF723F8C0F32A
:108670000743C2B2C0F3072101980078FFF7D8F88A
:108680000E4B1B7833B1013EB6F1FF3F08BF002609
:1086900008F804600134E4B2112CB1D10135EDB217
:1086A000072DAAD1B9F15E0F8CBF0020012005B0C3
:1086B000BDE8F08F941F00200C200020911F0020A7
:1086C000440D0020B82F0020544B2DE9F04FDC78EA
:1086D00087B004EB4406B610F3B20293FF23B3FB5A
:1086E000F4F301938378DFF8488163B100221146E7
:1086F0001046FFF747FF772200214948F7F7A6FF0A
:10870000002388F800300027464DDFF814B12B789D
:1087100001332B70D9464FF0000A98F800205FFA19
:108720008AF31A4362D10393F8F712F83E4B98424A
:10873000039B5BDC8BF8004004AA39461846FFF720
:1087400045F880B199F80020029B9DF810009A42EC
:108750005BD9931B7343A21B93FBF2F32246DBB25C
:108760001946FFF765F80AF1010ABAF1070F09F196
:108770001109D2D10137FFB2112F0BF1010BC9D171
:108780002B78019A934204BF00232B7098F8003095
:108790000133DBB21C2B3ED9002388F800300623BE
:1087A000224D661E294611221D48062B05D190F840
:1087B0006670BC4208BF80F8666011F8117C013A0F
:1087C000A74224BF01F8116C0C7012F0FF0201F1F6
:1087D000010100F10100E8D1013B13F0FF03A5F115
:1087E0001105DFD1002007B0BDE8F08F99F8002017
:1087F000002AA1D094429FD929780198814204BFD0
:1088000002F1FF3289F8002096E76243B2FBF6F2EC
:108810000023D2B2A4E788F80030E3E7B82F0020A5
:10882000941F0020901F002054555505FA1F00206A
:10883000931F00202DE9F04F85B007468846164665
:10884000FDF780F8814600284AD0002E4BD002AABE
:1088500041463846FEF7BAFF0546324C23782B4492
:10886000082B22DDC5F1080A691C52462144601C10
:10887000F7F776FE05F109015246214404F109009B
:10888000F7F76EFE04EB45014FEA4A02193104F195
:108890001900F7F765FE05F111015246214404F174
:1088A0001100F7F75DFE84F800A0002211469646FD
:1088B00094F800C0D0B200EB0C03DBB28542019308
:1088C00013D86544EDB201B125704EB1164B1B783B
:1088D00003F0FC037C2B03D141463846FEF7EEFE45
:1088E00005B0BDE8F08F3546B7E702AB13F802A03C
:1088F000019B0AF13801E0180C4B80F811A003EB42
:108900004101019B91F807B00C33097A04EB430352
:10891000417280F801B0013283F801E083F802E08F
:108920004946C7E70E200020B82F0020440D002044
:108930002DE9F04F924B89B01B7801908342914F03
:1089400045D1914A3B78127803F003039B1A18BF74
:1089500001238E4DAB706A787B799A4205D0002254
:10896000114610466B70FFF70DFE019B2C2B37D87C
:10897000DFE813F02F0038004C005000540058007E
:108980005C006000640068006C0070007400780097
:108990007C008000840088008C0090009400980087
:1089A0009C00A000A400A800AC00B000B400160118
:1089B000C201430247024B024F02530257025B02BD
:1089C0005F02630267026B026F0273027702012388
:1089D000BFE7A87848B1002211461046FFF7D2FD44
:1089E000002002E06948FFF7DBFA684B1A78013291
:1089F0001A7040B90221664A9B7811701BB9019B1D
:108A00000BB90323137009B0BDE8F08F5F48FFF77F
:108A10000BFBEAE75D48FFF76DFBE6E75B48FFF716
:108A2000B1FBE2E75948FFF7F7FBDEE75748FFF7EE
:108A30006BF8DAE75548FFF76DF8D6E75348FEF7CD
:108A4000F5FFD2E75148FEF7F7FFCEE74F48FEF7B4
:108A500073FFCAE74D48FEF775FFC6E74B48FFF7BF
:108A60005FF8C2E74948FFF761F8BEE74748FFF7FC
:108A700063F8BAE74548FFF765F8B6E74348FEF7FD
:108A800067FFB2E74148FEF7DDFFAEE73F48FEF77C
:108A9000DFFFAAE73D48FEF761FFA6E73B48FFF787
:108AA000C9F8A2E73948FFF7CBF89EE73748FFF748
:108AB000CDF89AE73548FFF741FC96E73348FFF7D2
:108AC000ADFC92E73148FFF7F9FC8EE72F48FFF73E
:108AD0003FF88AE72D48FFF741F886E72D4B2878C5
:108AE0002D4E01301968326800EBC00400EB4400E1
:108AF0009142C4B2984630D9FEF798F94FF05F0919
:108B000009FB00F9254B4FEA29294B4493F83521FD
:108B10006B781A4221D0FEF789F9810722D500230C
:108B2000ADF818308DF81A300698FEF7C3FDC0F383
:108B30000743C2B2C0F307214846FEF779FE3B79EE
:108B40004FF4FA721033FF2B28BFFF231B09B2FB2F
:108B5000F3F3D8F80020134433605E2C8CBF002060
:108B6000012042E7FEF762F98DF81800FEF75EF982
:108B700040F357007F308DF81900FB78D2E700BF33
:108B8000D70F0020B82F0020D80F0020D40F0020CE
:108B9000D90F0020C02F002094210020440D002078
:108BA000B34BB44A186811680092884202933FF6AA
:108BB00017AFAB78B04E9BBB2C78DFF8D4B204EB88
:108BC000C40304EB4304E4B204F113095FFA89F926
:108BD000B9F15F0FCA4628BF4FF05F0A04EB4408A3
:108BE000B044E3B29A4553D8B9F15E0F40F23D81EB
:108BF0005F24A14D013C05F103055BD1FEF716F999
:108C000083075DD586F81A4186F81B4186F81C411A
:108C1000FEF724FB009B1B681844029B1860DFE6EC
:108C20000022002411461046FFF7ACFCB046A146D6
:108C3000FEF7FCF882070BD588F8009088F80190C1
:108C400088F8029001345F2C08F10308F0D1B3E7F3
:108C5000FEF7ECF88DF81400FEF7E8F8FB7840F327
:108C600057007F308DF816308DF815000598FEF707
:108C7000B3F804EB440B06F80B0006EB0B0AC0F349
:108C80000723C0F307408AF801308AF80200D9E7C9
:108C900014F80B206B781A4208D098F8023098F834
:108CA000002098F801102046FEF7C2FD08F10308E5
:108CB000013496E703222946E81EF7F751FC99E7AD
:108CC000FEF7B4F88DF81800FEF7B0F8FB7840F323
:108CD00057007F308DF81A308DF819000698FEF78E
:108CE0007BF8C0F3072386F81A01C0F3074086F823
:108CF0001B3186F81C018BE7AB7823B100221146AB
:108D00001046FFF73FFC2878013000EBC00300EB72
:108D10004300C3B20393574B1A68584B1B689A42DF
:108D200056D9B8787B78564D43EA0023F878554FEA
:108D300043EA0040FEF7BEFCC3B20093C0F3072B2A
:108D4000C0F30746AA46B94607240295029B19F8C4
:108D5000018B13F8010B0293B8F1000F3BD033469F
:108D6000009A5946FEF764FD33465946009A9AF830
:108D70001000FEF75DFD013C99F8003014F0FF048F
:108D800009F8013C0AF1FF3AE0D1FB79E8795BB3DD
:108D90003346009A5946FEF74BFD33465946009A32
:108DA000687AFEF745FDFEF741F810F0030F0CBF9F
:108DB00001230023FB71344B1135AB4207F1080747
:108DC000C0D1FEF74BFA2B4B1B6818442B4B186095
:108DD000039B5E2BC2E6434642464146FEF728FD12
:108DE000434642464146C2E7234622462146FEF715
:108DF0001FFD234622462146D2E72448FFF7C8FB41
:108E0000F3E52248FFF760FCEFE52048FEF7A0FFFE
:108E1000EBE51E48FEF7A2FFE7E51C48FFF748F820
:108E2000E3E51A48FFF754F8DFE51848FFF758F86C
:108E3000DBE51648FFF764F8D7E51448FFF768F854
:108E4000D3E51248FFF774F8CFE51048FFF778F83C
:108E5000CBE50E48FFF784F8C7E50C48FFF788F824
:108E6000C3E50A48FFF794F8BFE50120BDE500BF60
:108E700098210020C02F0020372000209C210020B6
:108E8000440D002054210020BB0D0020D40F0020F1
:108E9000790E00200120704708B5FFF7FBFF08BDE1
:108EA00008B5017801EBC10301EB4301C9B2A1F19F
:108EB00013005F2928BF5F21C0B2FAF759FF08BD30
:108EC0002DE9F8433B4E337803F00303012B4DD1DA
:108ED000394C0025206801F0E1FD804601F098FD45
:108EE0003649206091F800E0AC467446C8F57F47EB
:108EF000FF37EBB29E4513D8BCF1000F00D00C70C9
:108F00002F4B1B7823BB337813F0030500D09D084B
:108F10002C4C2378032B29D8DFE803F01C2A3A3F96
:108F200005F10C0201EB4202537892F802900135F0
:108F300043EA09239F4225BF43449BB204F1FF3417
:108F400053702DBF1B0AE4B24FF0010C9370D0E7B1
:108F50000025DDE700221C4B18491A701B4B292203
:108F600018601B48F7F7FCFA01232370BDE8F8836B
:108F70002846FFF7DDFC002DF8D0134B1B78052B9E
:108F800001D1FFF789FFBDE8F8430F48FFF788BF1D
:108F90002846BDE8F843FEF733BC0E4B1B780BB1F7
:108FA000FEF77AFB094B186801F078FD0F28DDD930
:108FB0000023DAE7B82F00208C2100200E200020AB
:108FC00090210020D90F0020D40F0020C02F0020B6
:108FD000C42F0020921F002008B5274B1B6898471C
:108FE0004FF0FF330021254A117053769376D376E4
:108FF000137753779377D37782F8203082F8213034
:1090000082F8223082F8233082F8243082F825302A
:1090100082F8263082F8273082F82830184A1170FA
:1090200053769376D376137753779377D37782F803
:10903000203082F8213082F8223082F8233082F802
:10904000243082F8253082F8263082F8273082F8E2
:109050002830FCF7B3FB18B9FCF734FCFEF79EFB95
:10906000FEF728FA074B1B7813F0FC0F03D1BDE87D
:109070000840FEF793BB08BD5CEC0008C42F00203D
:109080000E200020B82F002070B50646054D38B1DF
:109090002C782CB92046FFF74BFC2046FEF7B0FB9E
:1090A0002E7070BD90210020044A137883F00103D4
:1090B00013700022024B1A70FEF7F4B9B82F00208B
:1090C000D90F00200020FFF7EFBF0120FFF7ECBF12
:1090D000064B1A7812F0030204BF05490A700121F9
:1090E0001A7861F301021A70704700BFB82F002090
:1090F000D90F002008B5FFF7EBFFBDE808400120BD
:10910000FEF7D0B908B5094B00201A7892071EBFA8
:109110000021074A11701A786FF301021A70FFF7E5
:1091200007FCBDE808400020FEF76ABBB82F00200E
:10913000D90F002008B5FFF7E5FFBDE80840012082
:10914000FEF7B0B9024B187800F00300704700BF7B
:10915000B82F00200A4A137813F0030F0ED048B935
:10916000012060F3870313700022064B08461A7033
:10917000FEF798B92C2888BF2C20F2E7704700BF73
:10918000B82F0020D90F00200021FFF7E3BF0121F5
:10919000FFF7E0BF014B187880087047B82F002018
:1091A000054B01461B789B0801332D2B34BF184615
:1091B0000120FFF7CFBF00BFB82F00200120FFF72D
:1091C000EFBF0000064B01461B78C3F38503013B4C
:1091D00013F0FF0314BF18462C20FFF7BBBF00BFDE
:1091E000B82F00200120FFF7EDBF000030B4084C7D
:1091F0002578AD0709D0442A28BF44226070A170A9
:10920000E270184630BCFEF74DB930BC704700BF65
:10921000B82F00200023FFF7E9BF0000014B58786A
:10922000704700BFB82F0020014B9878704700BFEF
:10923000B82F0020014BD878704700BFB82F00200E
:10924000054910B44C780346CA7804F108008978BF
:1092500010BCFFF7CBBF00BFB82F00200120FFF7E5
:10926000EFBF0000054910B44C780346083CCA78AB
:10927000A0B2897810BCFFF7B9BF00BFB82F00209B
:109280000120FFF7EFBF000010B4064C0346A178A1
:10929000E2781031FF2928BFFF216078C9B210BCE5
:1092A000FFF7A4BFB82F00200120FFF7EDBF00009B
:1092B00010B4064C0346A178E278103921EAE17136
:1092C0006078C9B210BCFFF791BF00BFB82F002073
:1092D0000120FFF7EDBF000010B4064C0346E27812
:1092E000A1781132FF2A28BFFF226078D2B210BCC9
:1092F000FFF77CBFB82F00200120FFF7EDBF000073
:1093000010B4064C0346E278A178113A22EAE272E0
:109310006078D2B210BCFFF769BF00BFB82F002041
:109320000120FFF7EDBF0000024B18710020FEF78F
:10933000B9B800BFB82F0020014B1879704700BFA3
:10934000B82F0020044A13794033FF2B28BFFF2396
:109350001371FEF7A7B800BFB82F00200120FFF758
:10936000F1BF0000034A1379403B23EAE373137112
:10937000FEF798B8B82F00200120FFF7F3BF0000D8
:109380000022014B1A707047A0210020F0B50B4C51
:1093900045002F18E61996F801C08C4505D1E75D08
:1093A000974202D1B6789E4207D001270544044E69
:1093B00060193770417062558370F0BDED2F002049
:1093C000A0210020F8B505460E4617460024204689
:1093D0003B46324629460134FFF7D8FF5F2CF6D1D1
:1093E000F8BD000010B5054C23782BB15F2104486F
:1093F00000F0B2F80023237010BD00BFA0210020B0
:10940000ED2F002000B110470847000038B54D7916
:109410000446BDB9FCF7BAF8A4F5F043203B00F0D0
:109420002200142B3AD8DFE803F00B0F14171A1D93
:10943000202326292C2F3335370D0D0D0D0D0D0052
:10944000FFF743FE284638BD154A1649FFF7DAFFF5
:10945000F8E7144A1249F9E7134A1449F6E7134AA0
:109460001149F3E7124A1349F0E7124A1049EDE7B0
:10947000114A1249EAE7114A0F49E7E7104A114930
:10948000E4E7104A0E49E1E70120FFF780FED9E743
:109490000520FAE70D20F8E71220F6E70125D1E7CD
:1094A000E5910008BD910008819200085D920008D6
:1094B000D1920008A992000821930008F9920008AF
:1094C000799300085D93000870B5072301264FF4D7
:1094D00000444FF000451B4A06FA03F10142946133
:1094E00019D0052100BF00BF00BF00BF00BF00BFF3
:1094F0000139F7D1956100BF00BF00BF00BF00BFB9
:1095000000BF00BF00BF00BF00BF00BF00BF13F11E
:10951000FF33E1D270BD00BF00BF00BF00BF00BF7E
:1095200000BF00BF00BF00BF00BF00BF00BF0521DC
:10953000956100BF00BF00BF00BF00BF00BF013981
:10954000F7D1E4E70004004001224FF40041014854
:1095500003F084BC00040040F8B5164D04462B7897
:109560000E461BB9FFF7F0FF01232B70302383F366
:10957000118800235F1CDBB2B3420CD34FF4A86305
:1095800000BF00BF00BF00BF00BF00BF013BF7D15D
:1095900083F31188F8BD03EB4303E518E05CFFF7A4
:1095A00093FF6878FFF790FFA878FFF78DFF3B46A1
:1095B000E0E700BFA121002008B52820FDF732F820
:1095C00008BD08B52520FDF72DF8262801D000207C
:1095D00008BDFDF727F80128F9D12720FDF722F86B
:1095E000A0F1120358425841F2E710B5041E14BF0F
:1095F0002621FF212520FDF77DF8002C14BF012135
:10960000FF212620FDF776F8002C18BF1221BDE8B7
:10961000104008BFFF212720FDF76CB87047704746
:1096200010B50446FFF7FBFFE1B22820BDE810406B
:10963000FDF760B808B50020FFF7D7FF0020FFF75F
:10964000EFFF00F0F9FD00F08DFEBDE808400120BD
:10965000FFF7CBBF08B5FFF7E1FFFFF7ADFFFFF75F
:10966000DEFFFFF7AEFF18B9BDE80840FFF7E2BF25
:1096700008BDFFF727BD08B54B794BB1A0F5EE4209
:109680007F2A03D8C0B200F079FE0023184608BD37
:109690000123FBE7FF230370704710B503780446EE
:1096A000013B032B0BD8DFE803F0020B1215FFF789
:1096B000C1FD4423C0EB0020B0FBF3F0607010BD8F
:1096C000FFF740FD0028F9D0FFF764FDF6E7FFF74C
:1096D00033FEF3E7FFF7A2FD6070FFF7A5FDA07072
:1096E000EDE738B503780446013B032B2CD8DFE8BF
:1096F00003F002111E23FFF791FD0546FFF794FDCD
:109700004422637801465A43A8B2120ABDE83840A1
:10971000FFF780BD43781BB9BDE83840FFF7F2BCC6
:10972000FFF7D6FC6078BDE83840FFF72DBD4078E4
:10973000BDE83840FFF7F8BD45788478FFF77AFD3B
:10974000214602462846E1E738BD024610F8023BB2
:10975000082B05D0092B05D0072B05D1FFF7C1BF7A
:10976000FFF79BBFFEF718B8FF231370704708B5CB
:109770004378032B03D1BDE80840FFF7E6BFFFF7AE
:1097800089FF08BD2DE9F04104460F46FAF74EFE69
:10979000002840F0B1802378013B122B4BD8DFE842
:1097A00003F00A14455F656F7272724A4A777B81D3
:1097B0008A939699A200002363700C23A370394604
:1097C0002046BDE8F04101F08DBD6378013B032BDD
:1097D00031D8DFE803F0020C0F2301F019F9030E72
:1097E000A370030CE370030A23716071E7E7FFF7CE
:1097F000E3FEF4E72546A67804F11B08062EDED822
:10980000F0B2FCF76FFB030CEB70030A2B7168716D
:109810000335454506F10106F0D1D0E70023A370DA
:10982000E3700423237109236371C8E76378022B73
:1098300004D0052B10D0FF232370C0E7E378A07875
:1098400040EA0320237940EA0340637940EA036059
:1098500000BAFFF7E5FEB2E7A078FFF70AFFAEE730
:10986000E278A178607800F0BCFCBCE722796379EB
:10987000A17843EA02236078E27800F0C8FC9EE712
:1098800000F0DAFC9BE739462046FFF770FF96E7C9
:1098900000F02DFD607092E700F02BFD030A63706D
:1098A000A0708CE76078A378221DE17843EA00205D
:1098B00000F022FD83E76078A378221DE17843EA77
:1098C000002000F036FD7AE700F04CFD77E700F06D
:1098D0007DFCDFE76078A378221DE17843EA002071
:1098E00000F0CCFC6BE76078A378221DE17843EAB6
:1098F000002000F0DAFC62E7BDE8F081F0B5014439
:10990000884202D310461946F0BD002710F8014BDB
:109910004FEA031C624094184FEA021E43EB030512
:109920004CEA127C14EB0E0445EB0C054FEA421E88
:10993000A4184FEA431C43EB05054CEAD26C14EB28
:109940000E0445EB0C054FEAC21E4FEAC31C4CEA5D
:10995000526C14EB0E044FEA022645EB0C054FEA5D
:10996000032C4CEA126CA41945EB0C033A19B646C9
:1099700046EB0303C4E7000038B5054648790028E4
:1099800000F0DC80A5F5E045ABB2222B00F2BB80F5
:10999000FBF72CFF6A4C013D2080212D12D8DFE817
:1099A00005F04DBD551B1F59235D692FB5336D372C
:1099B00071973B759F417B8327612B65477F8EA9FC
:1099C000B31651C5237843F00103237095E0637803
:1099D00043F00803637090E0237843F00203F4E758
:1099E000237843F00403F0E7237843F00803ECE71F
:1099F000637843F00103EDE7637843F00203E9E79E
:109A0000237843F01003E0E7237843F02003DCE7FA
:109A1000237843F04003D8E7FBF766F9237843F057
:109A20008003D2E7237823F00C0343F00C03CCE748
:109A3000637823F0030343F00303CBE723786FF34A
:109A40000003C2E763786FF3C303C3E723786FF3C0
:109A50004103BAE723786FF38203B6E723786FF305
:109A6000C303B2E763786FF30003B3E763786FF380
:109A70004103AFE723786FF30413A6E723786FF36E
:109A80004513A2E723786FF386139EE7FBF72CF9C3
:109A900023786FF3C71398E7237823F00C0394E738
:109AA000637823F0030395E72378C3F3800282F001
:109AB0000102D2B262F3820362F3C30385E76378E3
:109AC000DA4302F0010262F3000362F3410381E72B
:109AD0002378C3F3801282F0010262F3861374E7E5
:109AE000FBF702F92378C3F3C01282F0010262F39C
:109AF000C7136AE70120FBF7E7FE2088FBF779FE32
:109B0000FBF7F2F8002038BD0020F4E72378C3F318
:109B1000001282F0010262F3041356E72378C3F3C4
:109B2000000282F0010262F300034EE76378C3F3A0
:109B3000C00282F0010262F3C3034BE70120E2E7B7
:109B4000782F0020F8B5174B1749C2081F5C174B38
:109B50008D5C17499B5C00F007008E5C034105415A
:109B600013F0010446FA00F005F0010500F00106CB
:109B700002D0E120F8F75EFF15B1E620F8F75AFFB2
:109B80003846FAF78DFE15B1E620F8F7B9FF14B1A3
:109B9000E120F8F7B5FF26B1BDE8F8402C20FAF730
:109BA0007FBEF8BD8CED00086CED00080CEE0008DF
:109BB0007CED00082DE9F04104460E464FF00A08FE
:109BC000214F207800283DD0012838D16378012B1F
:109BD0000ED1A078A51CFAF763FE2C463546013459
:109BE000013DEDB2FF2DECD0642001F0D8FFF7E786
:109BF000022B04D1A078A51CF8F71CFFEDE7032B7E
:109C000004D1A078A51CF8F77BFFE6E7042B01D070
:109C10000134E3E72246002512F8023FD95D1446DD
:109C2000490706D415F1FF35D8D3642001F0B7FFFA
:109C3000F8E7303B08FB053512F8013FEEE7FFF788
:109C400081FFCBE7BDE8F081B1E400080021FFF718
:109C5000B1BF70472DE9F84F244F3B786BB14FF0FF
:109C6000000A4FF00E0B224EDFF8889035783B78D3
:109C7000AB4204D800233B703370BDE8F88F0BFB78
:109C800005F309EB030405F1010822795FFA88F86E
:109C900086F80080DAB12289DAB94FF6FF7260895E
:109CA000904216D00121FFF7D4FF00230BFB05954E
:109CB0002B71FBF797FCBAF1000F08D12046FBF798
:109CC00043F820B9642001F06AFF4FF0010A4546CD
:109CD000CDE739F803206088A388E18842EA004094
:109CE00043EA01412289FBF7BFFBDEE71D2200208A
:109CF0001C220020AC2100207047000038B5002451
:109D0000084B1C80FAF7D6FBA5B2A84200D838BD94
:109D10002846FAF7D1FBC3790BB98371037201347A
:109D2000F0E700BF1E22002038B50D4D0D4B2C78FA
:109D30001B780D4AA3420ED032F8141081420BD189
:109D4000FAF7BAFB012383712B78A34203D10134C4
:109D500004F003042C7038BD013404F00304E9E777
:109D6000AA210020AB210020A22100208B792DE91F
:109D7000F74F002B40D1224D9C46A8464FF6FF7965
:109D80004FF0010E1F4A92F800B0DAB293452AD97B
:109D900000264FF6FF740A68B5F80CA00192019FE7
:109DA000F2B237F812700136BA4508BF94B2002FEC
:109DB000F5D14C451DD00EFA04F444EA0C0C0EFA11
:109DC00002F25FFA8CFC013A624511D10E22534334
:109DD0008C8808EB030214810424147128F80370A2
:109DE000508181F807E003B0BDE8F04FFFF79CBF5A
:109DF0002F7101330E35C8E703B0BDE8F08F00BF07
:109E0000AC2100201D22002070B50D4B0D4E1C789A
:109E10000D4D3378A34205D1FFF71CFFBDE870401C
:109E2000FFF76CBF35F81400FAF746FB014635F82A
:109E300014000134FFF79AFF04F00304E9E700BFC0
:109E4000AA210020AB210020A22100200023F0B590
:109E50001A461C46D0F800E0DDB23EF8156076B137
:109E6000D1F800C0002503E0BE4208BF0122013541
:109E7000ECB23CF81470002FF6D10133ECE71AB1C4
:109E8000AC4238BF0846F0BD1046FCE70F4B70B53A
:109E90001B789BB10E4C208880B100F0F8FD0D4E70
:109EA000338883420AD20C4B00251A780B4B1B785F
:109EB0009A4204D0FFF7A8FF3580258070BDFFF7D8
:109EC000C9FE2580BDE87040FFF718BFDC0F0020F9
:109ED000202200201E220020AA210020AB210020E9
:109EE00008B50023064A1380064A1370064B1A78F9
:109EF000064B1A70FFF702FFBDE80840FFF7AABE45
:109F000020220020DC0F0020AB210020AA2100200D
:109F1000034B1A780AB1FFF7E3BF01221A707047AA
:109F2000DC0F002047F650432DE9F04F984287B0F0
:109F300007460E4608D14D79C5B10122994B1A70DA
:109F4000284607B0BDE8F08F47F65143984204D148
:109F50004D795DB1FFF7C4FFF2E747F652439842EF
:109F600004D14D7915B1FFF7D3FFE9E78E4B18788F
:109F70008E4B1B781843FAF705FC0446FFF7BCFE2E
:109F8000844203D03188FBF759FE07464FF0000AA0
:109F90005546FAF78FFA1FFA8AF8404525D87379A3
:109FA000002B00F0ED80002D00F0EA8000F06AFD4B
:109FB0007F4B18807F4B1C78072C13D8621C1A70BB
:109FC00031460A2203A8F6F7CBFA0E227A4B03A9F0
:109FD00002FB04330A221846F6F7C2FA4FF6FF7264
:109FE0008781428185F00105AAE74046FAF764FAC5
:109FF0004FF6FF7B4FF0000C044600685FFA8CF1CF
:10A0000030F811200CF1010C974208BF1FFA81FBB8
:10A01000002AF3D14FF6FF70834530D0A379002B8F
:10A0200032D1604A1078727994F8079094F808C099
:10A03000002A64D0002862D0B9F1000F0CD10120B1
:10A0400000FA0BF343EA0C0C5C4B84F808C0188848
:10A0500031289CBF322018804FF00109237A09FA79
:10A0600001F1013999420AD1514B188870B100921F
:10A0700000F00DFD3228009A08D984F806901543A7
:10A08000EDB20AF1010A84E71046CCE700204C4B00
:10A09000DFF834B193F800909BF8001089450BD19C
:10A0A0008442ECD0474921F8198009F1010909F0EF
:10A0B00003098BF80090E2E7424B019233F8190054
:10A0C000FAF7FAF921460090FFF7C0FE019A88B12D
:10A0D0004FF0010384428371D1D0394B19788945FF
:10A0E00008D1009B834201BF09F10101344B01F00B
:10A0F0000301197009F1010909F00309CCE7B9F16D
:10A10000000F15D1012202FA01F10139614502D196
:10A1100053B900EA02090122237A02FA0BF223EA78
:10A12000020323724A46AAE74046FFF7FDFDF2E725
:10A130000CF1FF324CFA0BF112EA0C0201F00101B2
:10A140001BD1D1B1A188A1B10392049200F09AFC75
:10A1500004228DF81020A2880DF10C08ADF80E0035
:10A16000ADF8142098E80700FBF77EF90022E271B1
:10A17000D1E74046FFF76DFDF8E75FFA81F9CAE7DE
:10A180000F4B1A78104B1B789A4202D0FFF73CFE17
:10A1900028E7FFF75FFD0022054B1A80FFF7AEFDB1
:10A1A00020E700BFDC0F002073160020721600208D
:10A1B000202200201D220020AC2100201E22002091
:10A1C000AA210020A2210020AB21002004207047FA
:10A1D0002223520003FB0121EE2303FB0010293050
:10A1E0007047032838B510D806290ED8102A0CD885
:10A1F000FFF7EEFF0546FCF715FA000284B2681C73
:10A20000FCF710FA204380B238BD0020FCE7032899
:10A2100070B51C460FD806290DD8102A0BD8FFF7A9
:10A22000D7FF0546210AFCF765FAE1B2681CBDE8D4
:10A230007040FCF75FBA70BD2DE9F843002400259B
:10A24000E7B212E05FFA86F94A4641463846FAF725
:10A250001DF9013603464A4641463846FFF7D7FF07
:10A26000112EEFD10135072D03D000265FFA85F8B6
:10A27000E8E70134042CE2D1BDE8F883F8B51446D0
:10A28000002700F129055618B44200D1F8BDA5F108
:10A290002903B3F56E7F06DA2846FCF7C3F9207070
:10A2A00001350134F0E72770FAE7F8B50E46174696
:10A2B000002400F12905B44200D1F8BDA5F129031D
:10A2C000B3F56E7F03DA395D2846FCF713FA0135E2
:10A2D0000134F0E7032810B406D8062904D8102A60
:10A2E00002D810BCFFF77DBF002010BC70471020C3
:10A2F000704740F21F4070472DE9F041144640F28C
:10A300001E474FF0000800F2E1355618B44201D163
:10A31000BDE8F0816FF47873EB18BB4206DC284689
:10A32000FCF780F9207001350134EFE784F80080F4
:10A33000F9E72DE9F0410E461746002440F21E4889
:10A3400000F2E135B44201D1BDE8F0816FF47873D9
:10A35000EB18434503DC395D2846FCF7CBF90135A2
:10A360000134EFE710B540F2E1342046002101341A
:10A37000FCF7C0F9B4F5006FF7D110BD0F28F7B5A1
:10A3800005464ED840F2FF70FCF74CF9002848D142
:10A3900040F2E1342DBBCDE900552046FCF742F9EF
:10A3A000661C8DF800008DF80150D0B3012812D141
:10A3B0003046FCF737F9A71C8DF8010088B3431E1F
:10A3C000022B19D83846FCF72DF9E61C8DF802004F
:10A3D00038B38DF8035001216846FFF7EBFB344694
:10A3E000DBE7B4F5006F1CD02046FCF71BF908B979
:10A3F000013DEDB20134CDE7042814D102243846E2
:10A40000FCF710F97E1C0DF8040050B17C2804D133
:10A4100002AB1C4404F8075CDDE70134072C374627
:10A42000EDD103B0F0BD3E46D5E7000047F6164338
:10A43000984210B50C461BD1FBF7A8F862790D4B7A
:10A4400072B100F0AA00002815BF012200223520B9
:10A4500029201A70FBF76CF8FBF70CF9002010BDEF
:10A460001B78002B14BF35202920FBF769F8F3E790
:10A470000120F4E722220020F8B5144642791D4657
:10A480009DF81870284B92B11C7000F0FBFA274B16
:10A49000188004F12003DBB2072B44D8012004F01C
:10A4A0000704A040C0B2BDE8F840F8F77BBB1E78B7
:10A4B000A6422ED11D4B188800F0E9FAC72828D8EB
:10A4C000AE4205F1200415D006F12003DBB2072BC4
:10A4D00006D8012006F00706B040C0B2F8F792FB9C
:10A4E000E3B2072B06D8012005F007039840C0B25D
:10A4F000F8F758FB3846E4B2FAF7D2F9072C12D82D
:10A50000012005F00705A840C0B2BDE8F840F8F703
:10A5100079BB04F12003DBB2072B04D8012004F03F
:10A520000704A040F0E7F8BD2322002024220020E9
:10A5300013B5A0F5F84018380C4606283BD8DFE8DC
:10A5400000F0171E0410252C330026230093E1236E
:10A5500047F61A411A462046FFF78EFF002002B048
:10A5600010BD27230093E52347F61B411A46F2E767
:10A570002623E022009347F61841E123EBE7272347
:10A58000E422009347F61941E523E4E72623E2227B
:10A59000009347F61C41E123DDE72723E6220093E1
:10A5A00047F61D41E523D6E72823E522009347F629
:10A5B0001E410123CFE7487918B10022024B1A70DF
:10A5C000CDE70120CBE700BF2322002047F67743E9
:10A5D000984270B506D047F67843984229D00124B6
:10A5E000204670BD4C7994B100F02CF8FAF70AFCC3
:10A5F00000F028F8044600F02BF8054600F02EF88D
:10A60000294602462046FAF7FFFC0024E8E700F05E
:10A6100019F8FAF703FC00F015F8054600F018F8F1
:10A62000064600F01BF8314602462846FAF7ECFCD5
:10A63000D6E74C7914B100F00BF8D7E700F008F832
:10A64000E7E70000014B1878704700BFDE0F0020DD
:10A65000014B1878704700BFDF0F0020014B1878BE
:10A66000704700BFDD0F0020014B1860704700BF2E
:10A6700028220020024B186808B103681847704769
:10A680002822002008B5FFF7F5FF08BD084B1B681E
:10A690006BB1084A127842B1074A92F90020002AA9
:10A6A000BFBF02784270062202705B68184770478D
:10A6B000282200201C110020782F0020034B1B684B
:10A6C0001BB1022101709B681847704728220020A7
:10A6D0000B4B07B51A8882420ED01880094B1B68B5
:10A6E00053B103228DF80500000A8DF806008DF89D
:10A6F0000420DB6801A8984703B05DF804FB00BFA5
:10A700002E220020282200200B4B07B51A888242F7
:10A710000FD01880094B1B685BB104228DF805002F
:10A72000000A8DF806008DF80420DB680DEB0200AE
:10A73000984703B05DF804FB2C220020282200205B
:10A740000C4B821C1B7863B10B4B93F90030002B30
:10A75000ACBF06231E230020013BDBB2FF2B02D13E
:10A7600070470623F7E712F8011B0029F4D00130E7
:10A77000C0B2F1E71C110020782F0020F1B1114B7D
:10A780001B789BB1104B93F90030002B0EDACA08EE
:10A790001D2A13D80123104401F0070103FA01F127
:10A7A0008378194214BF012000207047831C0830B1
:10A7B00013F8012B8A4203D08342F9D1002070475D
:10A7C000012070471C110020782F00204FF0FF332C
:10A7D000002230B5851C15F8014B8C420ED0B3F128
:10A7E000FF3F02D1002C08BF13460132D4B2062C21
:10A7F00062B2F0D15A1C01D01844817030BD0022E1
:10A8000010B5831C083013F8014B8C4208BF03F8C5
:10A81000012C8342F7D110BDCB081D2B07D818445B
:10A8200001F0070301219940837819438170704733
:10A83000CB081D2B08D81844012301F007018B40D9
:10A84000817821EA030181707047000010B4094C3F
:10A85000034624780A463CB1074C94F90040002C8A
:10A8600002DA10BCFFF7D8BF1146184610BCFFF73C
:10A87000ADBF00BF1C110020782F002010B4094C80
:10A88000034624780A463CB1074C94F90040002C5A
:10A8900002DA10BCFFF7CCBF1146184610BCFFF718
:10A8A000AEBF00BF1C110020782F0020074B0230E4
:10A8B0001B7843B1064B93F90030002B03DA1E22BC
:10A8C0000021F5F7C3BE0622FAE700BF1C110020E5
:10A8D000782F002042784B789A421DD190F90230AF
:10A8E0001BB191F902209A4216D190F903301BB1A5
:10A8F00091F903209A420FD190F905301BB191F9DB
:10A9000005209A4208D190F9040030B191F9043041
:10A91000181A18BF012070470120704770470000C7
:10A92000002814BF0220012008B5024B1870F9F767
:10A93000ABFA08BD30220020032008B5024B187086
:10A94000F9F7A2FA08BD00BF30220020FFF7E8BFE8
:10A95000012008B5024B1870F9F796FA08BD00BF40
:10A9600030220020FFF7F4BF7047704770477047F0
:10A9700010B5FFF7F9FF0024FBF774FBFFF7F5FFB5
:10A98000E0B2FBF7AFFA18B90134072CF8D110BDCB
:10A990000120FCE708B501F0CDF9BDE8084000F062
:10A9A00011BF08B5F9F7D8FEBDE8084040F2A46031
:10A9B00001F0F5B808B5FAF7FFFDFAF713FEFAF75C
:10A9C000C7FDFBF741FD0020FFF782FE0020FFF7E7
:10A9D0009BFEBDE80840F9F7CBBE0000302383F3AF
:10A9E0001188064BDA69064B1A600023054A13608A
:10A9F000054A136083F31188704700BF303100208F
:10AA00003C2200203422002038220020FFF7E6BF3D
:10AA1000D0B5302383F31188134B144C144AD969F1
:10AA200023681068C91A884212480AD9A3F58333EB
:10AA3000E03B23600468104B01F583312344E0318F
:10AA4000036011600468002383F311884FF47A7067
:10AA500000270A4E0A4AE0FB0167002330463946C8
:10AA6000F5F7C4FB2044D0BD303100203C2200204B
:10AA7000342200203822002088598F029F8601004E
:10AA8000A086010008B5FFF7C3FF80B208BD10B56E
:10AA90000446FFF7BDFF001B80B210BD10B5044691
:10AAA000FFF7B6FF001B10BDBFF34F8F0549064BE4
:10AAB000CA6802F4E0621343CB60BFF34F8F00BF5C
:10AAC000FDE700BF00ED00E00400FA0508B5024A0A
:10AAD000024B1A60FFF7E8FFEFBEADDEFC6F00200F
:10AAE0000A4A08B552F8041C094B99420DD10023BB
:10AAF00042F8043C83F31488064B1B6883F30888F0
:10AB000062B6054B1B689847FEE708BD0070002041
:10AB1000EFBEADDE00E0FF1F04E0FF1F08B5FFF74A
:10AB2000C3FF00000F4B10B51A78CAB901220E4CB2
:10AB30001A70206040F282324FF400714FF0804072
:10AB400002F08CF94FF480614FF0804040F2823285
:10AB500002F084F92146BDE81040044801F058BCD9
:10AB600010BD00BF40220020E00F002090310020E7
:10AB700008B54FF0FF31024801F02AFBC0B208BD12
:10AB80009C3100200A464FF0FF330146014801F096
:10AB9000C4BB00BFC03100200A464FF0FF3301465E
:10ABA000014801F03BBB00BF9C31002008B50348C1
:10ABB00001F053FC80F00100C0B208BD90310020CC
:10ABC000194B10B51C786CBB012208211A7017486C
:10ABD000224602F043F922462021144802F03EF9B1
:10ABE00022461021114802F039F94FF47A7000F032
:10ABF000D6FF41F6822208210C4802F02FF940F2DC
:10AC000082222021094802F029F940F282221021F3
:10AC1000064802F023F9064801F048FC4FF0FF32E5
:10AC2000044B1A6010BD00BF412200200004004008
:10AC3000EC320020E80F002001461A4810B50468E5
:10AC400001342BD14C1C29D053B3174C9B002382C9
:10AC50002346032A05D8DFE802F0021A1D1F00224E
:10AC6000DA600124016021F00F0001F00F0199600A
:10AC7000224604FA01F1586002F0F0F80A490B4844
:10AC800001F006FC094801F01FFC204610BD4FF4FE
:10AC90008002E5E78022E3E7054AE1E70020F5E7E7
:10ACA0001846F3E7E80F002044220020EC32002091
:10ACB000800040001FB501218DF807000DF10F0342
:10ACC0000DF10702034801F01AFC9DF80F0005B0D2
:10ACD0005DF804FBEC320020002307B501210DF1E3
:10ACE000070205488DF8073001F02BFC9DF807009E
:10ACF00003B05DF804FB00BFEC32002008B502464B
:10AD0000024801F00DFC002008BD00BFEC3200201D
:10AD100008B50246024801F014FC002008BD00BF3F
:10AD2000EC32002010B5074C2368013308D00648E8
:10AD300001F0D8FB044801F0B9FB4FF0FF3323606A
:10AD400010BD00BFE80F0020EC320020704700006B
:10AD500010B5084A084C117824784B1C03F00F03F7
:10AD60009C421DBF054C13706054002018BF012089
:10AD700010BD00BF1A3100201B3100200A31002015
:10AD8000F8B50B4C90F84B7090F84A601D460020C7
:10AD9000234643F8040F42EA012046EA07222946E7
:10ADA00000F0FCFA20606068002818BF2046F8BD5B
:10ADB0007823002090F84A10054B02291A7804D114
:10ADC000012A01D0062A02D15A78024B1A70704724
:10ADD000D8230020B023002008B5302383F3118846
:10ADE000034800F017FC002383F3118808BD00BF5F
:10ADF0009C10002038B5044605293DD8DFE801F055
:10AE0000303C0330303D302383F31188204D214AFC
:10AE1000012101F0F2FB204A0321204601F0EDFB65
:10AE200095F8901005F14402204601F0E6FB95F8F4
:10AE3000921021B105F16802204601F0DEFB1748AF
:10AE400000F0B1FB002383F31188154B1B7813B17D
:10AE50000520FFF77DFF0220BDE83840FFF778BFEF
:10AE60000846FFF775FF302383F311880B4800F085
:10AE700077FB002383F3118838BD302383F31188D7
:10AE8000064800F085FB002383F311880520E3E7E3
:10AE9000EC0F00201CEE000840EE00089C10002083
:10AEA000D123002070B5044606480D4603680BB157
:10AEB00000F0D8FC2B462146BDE87040024A01480C
:10AEC00000F0C8BC98230020CDAE000870B5302338
:10AED0000E4683F311880B78042B03D0002383F3F1
:10AEE000118870BD144B1B78DB09F7D1134C227805
:10AEF000002AF3D0124B1B78002BEFD00B899B0755
:10AF000005D408230F4A0121304601F0C8FB40F266
:10AF1000E73000210C4B24784FF47A72A4FB0345F0
:10AF200020184FF0000345EB0101F5F75FF93146BA
:10AF30008000FFF7B7FFD1E7782F0020942300208F
:10AF40001C110020B1230020A0860100F8B590F864
:10AF50004430044603F07F02212A40F0828013F03F
:10AF6000800334D0002B7CD090F84500022829D0F3
:10AF700003281ED0012874D194F848305BB1022B0D
:10AF800094F846200DD0494B1A70A36394F84A30C8
:10AF9000E36300232DE0464AA2630822E2632364B0
:10AFA000F8BD022AEFD1434BA3630623E3630023DA
:10AFB000F5E7B4F84830002B53D101203E4AE06356
:10AFC000A263ECE701203D4BE063A363EFE790F859
:10AFD00045300A2B3CD00B2B0ED0092B41D190F8D9
:10AFE00048300BB1022B3CD1354BA3630223E36302
:10AFF000344B23640120D3E7B0F8483023BB90F8EA
:10B0000046502D4B002D14BF012200221A701BD177
:10B010002A4B1A78C2B1302282F3118840F2E7300D
:10B0200000211E78284B4FF47A72A6FB0367301874
:10B030004FF0000347EB0101F5F7D8F821468000F7
:10B04000FFF730FF85F311880023A363E363D0E7A4
:10B050001E4990F847200D78184BED091A70F3D16E
:10B06000D8E740F28163B4F844209A4214D194F8AE
:10B070004920616894F848304D6843EA022394F807
:10B08000471094F846202046A84708B9002087E7D3
:10B090004368A36303687BE70D4B93F89230002B62
:10B0A000F4D02046BDE8F84000F094BAF023002028
:10B0B000B1230020D22300201C1100209423002063
:10B0C000D8230020B5AD0008A0860100782F00200D
:10B0D000EC0F002008B5102200210448F5F7B6FA5D
:10B0E0000023034A1370034A137008BD0A3100207D
:10B0F0001A3100201B310020F8B5294D294E2C466D
:10B10000002130782B78284F984230D101B120703F
:10B11000F8BD01222370254B1A70254B93F84F1070
:10B12000081C18BF0120FFF707FCE9E70022237085
:10B130001E4B1A70FFF73EFC1D4B93F84F10081C76
:10B1400018BF0120FFF702FCDAE72370184B93F8D1
:10B150004F10081C18BF0120FFF7E2FBD0E70021C9
:10B1600023700846F8E72370FFF7F2FBC8E71A469A
:10B17000BA5C013303F00F030121052AC4D80FF292
:10B18000080C5CF822F000BF67B1000809B10008A4
:10B190004BB100085FB1000813B100082DB10008E1
:10B1A0001B3100201A3100200A310020D123002059
:10B1B0002033002070B50546144C04F10803A36544
:10B1C00004F11C03E36504F13003E36704F18C062A
:10B1D000B0343146204600F081F93146204600F077
:10B1E000A7F9284601F0FAFD284601F0DCF941F202
:10B1F000883000F0D4FC0649284601F0C1F9284601
:10B2000001F0CAFD0022034B1A6070BDEC0F002054
:10B2100064EE000898230020014B1878704700BFA7
:10B22000B023002070B5302304460D46164683F344
:10B2300011880F490B78042B03D0002383F3118866
:10B2400070BD01200B89A04018420AD001EB840197
:10B25000CB684FF47A7158690C3000F0ADFC0130C6
:10B26000EBD033462A462146014801F018FAE4E7BC
:10B270002033002010B50D4B04461B7853B901460E
:10B2800008220120FFF7CEFF202221460848F5F7CB
:10B2900067F910BD074B014693F90030002BABBF97
:10B2A0000822202201200320ECE700BF1C1100200F
:10B2B000B1230020782F002010B504460146062255
:10B2C0000320FFF7AFFF062221460248F5F748F9B1
:10B2D00010BD00BFD2230020032201461046FFF715
:10B2E000A1BF0000202910B40A46044606D1044834
:10B2F000214650F8B03F10BC5B68184710BC70473F
:10B30000EC0F002070B50A4C88B004F1B005D4F8F9
:10B31000B03020221E6A694600232846B04720B17B
:10B32000C1B26846FEF72EFAF1E708B070BD00BF63
:10B33000EC0F0020FFF7D4BB7047704708B5FFF74C
:10B34000F9FF01F0A7FBFFF7F7FF08BD08B501F013
:10B35000BDFBFFF7F2FF08BDFFF704BB08B5FFF721
:10B36000B9FE0648FFF726FF054B064A41F2883032
:10B370001A60BDE8084000F012BC00BF2033002076
:10B380001024002020110020014B1868FFF76CB931
:10B3900010240020FFF7B0BEFFF7B4BF020A032A53
:10B3A00012D006D8012A20D0022A21D0002002463D
:10B3B00019E0212A11D0222AF8D10229F6D80E4A02
:10B3C0000E4852F8212006E0C0B20228EED80C4AFE
:10B3D0000C4952F82020405C05E00229E6D80920FB
:10B3E000094A52F821201A6070471220074AFAE7EA
:10B3F0005B20074AF7E700BF90EE00089CEE0008CC
:10B4000074EE000880EE000884EE0008FAEE0008F2
:10B410009FEE000813B5446BE36F1A681178042996
:10B4200015D1217A022912D11979012312898B4071
:10B4300013420CD101A904F1440000F078FD02464A
:10B4400028B1E46F019B2179206801F028F902B04E
:10B4500010BD0C3000F005BD4FF0FF330C3000F094
:10B4600000BD443000F0CCBD4FF0FF33443000F05D
:10B47000C7BD0C3000F0D8BC4FF0FF310C3000F0ED
:10B48000D3BC443000F09CBD4FF0FF32443000F09C
:10B4900097BDC26F70B5136805461978042901D0AD
:10B4A000012070BD017A0229FAD1012052795C890C
:10B4B00090400440F4D105F10C0000F070FC02460D
:10B4C0000028EDD0EE6FAB6A3068043B717901F073
:10B4D000D4F82046E5E7406BFFF7DBBF7FB50346B6
:10B4E00001260D4604460F4A43F8042B43600E4BD9
:10B4F000067202900193CB680C3000934B690A6A84
:10B50000314600F02AFC094B02940193AB68EA69CA
:10B51000009331462B6904F1440000F0E5FC04B0CF
:10B5200070BD00BF40F00008D7B4000815B4000893
:10B530000B68302282F311880A7903EB8202906152
:10B540004A79093243F822008A7912B103EB820367
:10B5500098610223C1670372002383F31188704747
:10B5600038B5044601250221043000F07FFB04F1C8
:10B570000C0025756FF0010100F051FB84F84C5070
:10B5800004F144006FF00101BDE8384000F047BB12
:10B5900010B501210446043000F068FB0023237538
:10B5A00084F84C3010BD38B5044600250C3000F04E
:10B5B000EBFB04F14400257500F0ADFC201D84F880
:10B5C0004C50012100F052FB2046BDE83840FFF707
:10B5D00060BF000090F8443003F06003202B09D1D5
:10B5E00090F84530202B05D3212B05D9222B4FF085
:10B5F000000309D000207047054B83630723C36312
:10B6000000230364012070478363C363F9E700BF2D
:10B6100030110020C36F73B51A68044611780429ED
:10B6200027D1017A022924D11979012315898B4068
:10B630001D401ED100F14406304600F026FDC0B189
:10B64000304601A900F073FCE36F06461A7E4AB14A
:10B6500001981A692946121A3044F4F7F7FFE36F8C
:10B660001B690193E06F019B01793246006801F08C
:10B6700016F802B070BD00EB81032DE9F3419E691D
:10B6800004460D46FEB1302383F311880821301D96
:10B6900004EB850700F0EAFAFB6806F144085B69F1
:10B6A0001B6813B1404600F050FC01A9404600F071
:10B6B0003EFC024650B1019B2946204600F0EFFFB8
:10B6C000002383F3118802B0BDE8F081FB685A695A
:10B6D0001268002AF4D01B8A013B1342F0D1F36FA9
:10B6E0001B7E002BECD104F14402E5E7093110B5D3
:10B6F00050F82140C4B1302383F31188042160182D
:10B7000000F0B4FAE26F04F10C001368527903EB15
:10B710008203DB689B69596800F04BFB2046FFF70A
:10B72000B8FE002383F3118810BD7047024B034A13
:10B730001A60034A5A6070471C310020A033002071
:10B7400000700020094B30B51C684D1E2244494250
:10B750002A440A4059681044884204D8A04202D3BF
:10B760001860104630BD0022FBE700BF1C310020EE
:10B7700008B5302383F31188FFF7E4FF002383F338
:10B78000118808BD70477047FEE7000070B50820BB
:10B7900000240B4B93E826000439954207D8D9685A
:10B7A000914209D8013803F11003F3D170BD51F86B
:10B7B000046F42F8046BF0E742F8044BF0E700BF77
:10B7C00068F0000838B501230025074C2370656038
:10B7D000FFF7ACFF0549064800F034F90223237057
:10B7E00085F3118838BD00BF28310020E8F000083B
:10B7F0003031002072B60322024BD865024B1A701A
:10B80000FEE700BF303100202831002000F03CB8B6
:10B81000034B59685A68521A9042FBD8704700BFD0
:10B82000001000E010B50A4A13699C68A1420CD8C8
:10B830005C68816003604460206058609868411AC9
:10B8400099604FF0FF33936110BD091B1B68ECE753
:10B85000303100200361002310B4C260436110BC8A
:10B86000FFF7E0BF036881689A680A449A604268FB
:10B8700013605A6000234FF0FF320360014B9A615E
:10B88000704700BF3031002070B5124D2946EA697B
:10B890000132EA6151F8102F8A4206D030269368AF
:10B8A000013B93602C69A36803B170BD2268616895
:10B8B0000A605160236083F31188E36821692046A0
:10B8C000984786F3118861690029EBD02046FFF77D
:10B8D000A9FFE7E730310020002382680375036980
:10B8E0001B6899689142FBD25A68036042601060FD
:10B8F0005860704700238268037503691B68996864
:10B900009142FBD85A6803604260106058607047EB
:10B9100008B5302383F311880A7D0023052A06D851
:10B92000DFE802F00C050503130F8A6913604FF07E
:10B93000FF3308468B61FFF7CFFF002383F31188A5
:10B9400008BD8A699368013393604A680B68136085
:10B950005A60ECE7FFF7C0BF054BD9680875186857
:10B96000026853601A6001220275D860F4F728BC9F
:10B970003031002030B50C4B87B0DC684B1C0546DD
:10B980000FD02346094A6846FFF764FF2846FFF7B1
:10B99000E3FF009B13B16846FFF764FFA06907B09F
:10B9A00030BDFFF7D9FFF9E73031002011B90008A9
:10B9B00038B50C4D8161EB6881689A680446914204
:10B9C00003D8BDE83840FFF787BF1846FFF792FF5E
:10B9D0000123EC60237501462046BDE83840F4F7AA
:10B9E000EFBB00BF30310020044B1A68DB68906861
:10B9F0009B68984294BF002001207047303100209E
:10BA0000084B10B51C68D868226853601A60012280
:10BA10002275DC60FFF76EFF01462046BDE810404E
:10BA2000F4F7CEBB30310020044B1A68DB68926813
:10BA30009B689A4201D9FFF7E3BF7047303100207D
:10BA400030BFFDE770B504460025194B86B085620E
:10BA500021630E46586000F027F904F110032361BA
:10BA600063614FF0FF33A361124BE561DA69002394
:10BA700004F13401C4E9082324606460A560E56230
:10BA8000E56580230C4A204600F01CF801230B4A90
:10BA9000E06003750092726868460192B268CDE971
:10BAA0000223074BCDE9043500F03EF806B070BD27
:10BAB000283100203031002009E700080EE7000897
:10BAC00041BA00088B6002224B62002308618A821F
:10BAD0000B62CB61084670478368C168A3F14C02D2
:10BAE00043F81C2C026943F84C2C42690C4843F87B
:10BAF000482C0C4A43F8180C43F82C2C022203F86B
:10BB0000142C002243F8201C03F8132C43F8041CC7
:10BB100043F8082C43F80C2CA3F12800704700BF11
:10BB200030310020D101000808B5FFF7D5FFBDE88E
:10BB30000840FFF70FBF000038B5302484F31188A8
:10BB40002839441844F8243C049B002544F8203C40
:10BB50000A4BA4F1240144F8043C0223A382084BBD
:10BB6000E160A260236162622562E56129462046A8
:10BB7000FFF71EFF85F31188204638BDD10100086C
:10BB800030310020024BDB6898610F20FFF7E4BEE4
:10BB900030310020302383F31188FFF7F3BF08B55D
:10BBA0000146302383F311880820FFF7E3FE0023CA
:10BBB00083F3118808BD0000054BDB6821B10360E9
:10BBC00098610320FFF7D6BE4FF0FF30704700BFEB
:10BBD0003031002003682BB10022026099611846C1
:10BBE000FFF7B8BE70470000064BDB6839B142680A
:10BBF00018605A60136043600420FFF7BBBE4FF02B
:10BC0000FF307047303100200368984206D01A6830
:10BC10000260506099611846FFF79CBE704738B5C6
:10BC200004460D462068844200D138BD0368236075
:10BC30005C608561FFF78EFEF4E7002300604060E2
:10BC400083607047C3691943037DC1610A2B03D127
:10BC50008369194205D170470B2B06D183698B4349
:10BC600003D100238361FFF775BE704770B50646A8
:10BC70000D460468B44200D170BDE3682B43E36015
:10BC800015B123691D4203D0A1686068FFF7DAFF90
:10BC90002468EFE7EFF30983203383F30988002357
:10BCA00083F3118870470000302080F3118862B65A
:10BCB0000B4B0C4AD96821F4E0610904090C0A43D2
:10BCC0000949DA60CA6842F08072CA6007490A68A6
:10BCD00042F001020A602022DA7783F822007047DE
:10BCE00000ED00E00003FA05F0ED00E0001000E0D8
:10BCF00010B5302383F311880B4B5B6813F400639A
:10BD00000FD0EFF309844FF08073203CE36184F39C
:10BD10000988FFF769FE10B1044BA36110BD044B05
:10BD2000FBE783F31188F9E700ED00E0E301000889
:10BD3000E601000808B500F077FF01F08EF800F08A
:10BD400044FB00F099FB00F00DFCFFF7FFFABDE8A3
:10BD5000084000F000B801F0A1B80172002130B530
:10BD6000039C043304FB0325C361049B006003634D
:10BD7000059B4060C160426102618561046242626C
:10BD80008162C162436330BD0022416AC260416189
:10BD900001618262C2626FF00101FFF740BF036977
:10BDA0004269934201D1C2680AB9181D7047002048
:10BDB000704703691960C26800210132C260C2691C
:10BDC000134482690361934224BF436A0361FFF70E
:10BDD0001BBF38B504460D46E3683BB162690020DD
:10BDE000131D1268A3621344E36207E0237A33B998
:10BDF00029462046FFF7F8FE0028EDDA38BD6FF03F
:10BE00000100FBE7C368C269013BC3604369134497
:10BE100082694361934224BF436A43610023836282
:10BE2000036B03B11847704770B53023044683F3A2
:10BE30001188866A3EB9FFF7CCFF054618B186F334
:10BE40001188284670BDA36AE26A13F8015B934229
:10BE5000A36202D32046FFF7D5FF002383F31188A6
:10BE6000EFE72DE9F84F04460F4691469A464FF00A
:10BE7000300888F311880025AB46A66A4EB95146B2
:10BE80002046FFF7A6FF20B186F311882846BDE8BB
:10BE9000F88FA16AE66AA9EB0503761A9E4228BFCD
:10BEA0001E46402E16D938464022F4F759FBA36AA5
:10BEB00040374033A3624035A26AE36A9A4202D314
:10BEC0002046FFF79FFF8BF311884D45DED288F3A4
:10BED0001188D2E738463246F4F742FBA36A37446A
:10BEE0003344A3623544E7E710B5029C0433017282
:10BEF000C36103FB042100238362C362039B0060D0
:10BF00000363049B4060C46042610261816104621A
:10BF10004262436310BD026A6FF00101C260426A6F
:10BF20004261026100228262C262FFF778BE436909
:10BF300002699A4201D1C26822B9184650F8043BFE
:10BF40000B60704700231846FAE7C368C2690133E3
:10BF5000C36043690021134482694361934224BF53
:10BF6000436A4361FFF750BE38B504460D46E368A7
:10BF70003BB1236900201A1DA262E2691344E36207
:10BF800007E0237A33B929462046FFF72DFE002823
:10BF9000EDDA38BD6FF00100FBE703691960C26894
:10BFA000013AC260C269134482690361934224BFAB
:10BFB000436A036100238362036B03B11847704730
:10BFC00070B5302304460E4683F31188856A35B96F
:10BFD0001146FFF7C9FF10B185F3118870BDA36A40
:10BFE0001E70A36AE26A01339342A36204D3E1693B
:10BFF00020460439FFF7D1FF002080F31188EDE7D8
:10C000002DE9F84F04460F4691469A464FF0300806
:10C0100088F311880025AB46A66A4EB951462046E2
:10C02000FFF7A2FF20B186F311882846BDE8F88FFC
:10C03000A06AE66AA9EB0503361A9E4228BF1E468F
:10C04000402E18D939464022F4F78AFAA36A4037BD
:10C050004033A3624035A26AE36A9A4204D3E1699D
:10C0600020460439FFF799FF8BF311884D45DCD248
:10C0700088F31188D0E739463246F4F771FAA36A9B
:10C0800037443344A3623544E5E7026943699A4281
:10C0900017D1C3689BB1836A8BB1043B9B1A0ED046
:10C0A0001360C368013BC360C3691A4483690261BA
:10C0B0009A4224BF436A0361002383620123184626
:10C0C00070470023FBE7F8B5154682680B46AA4285
:10C0D0008169066938BF8568761AB542044607D279
:10C0E00018462A46F4F73CFAA3692B44A3610DE0F5
:10C0F00011D932461846F4F733FAAF1B3A46E168D5
:10C100003044F4F72DFAE2683A44A261A368284665
:10C110005B1BA360F8BD18462A46F4F721FAE368D2
:10C12000E4E72DE9F0410446154683682669934209
:10C1300038BF856840690F46361AB54206D22A468E
:10C14000F4F70EFA63692B4463610DE012D93246AD
:10C15000A5EB0608F4F704FA4246B919E068F4F7CB
:10C16000FFF9E26842446261A36828465B1BA36052
:10C17000BDE8F0812A46F4F7F3F9E368E4E710B587
:10C180000024C361029B0A44006040608460C16077
:10C19000816141610261036210BD08B58269436932
:10C1A000934201D1826882B98268013282605A1C4E
:10C1B000426119700369426900219A4224BFC36831
:10C1C0004361FFF721FD002008BD4FF0FF30FBE782
:10C1D00070B5302304460E4683F31188A568A5B1D7
:10C1E000A368A269013BA360531CA361157822696F
:10C1F000934224BFE368A361E3690BB120469847EB
:10C20000002383F31188284607E031462046FFF7D4
:10C21000EBFC0028E2DA85F3118870BD2DE9F74FB9
:10C2200005460F4690469A46D0F81C90302686F375
:10C2300011884FF0000B144664B122463946284657
:10C24000FFF741FF034668B951462846FFF7CCFC8B
:10C250000028F1D0002383F31188A8EB040003B079
:10C26000BDE8F08FB9F1000F03D001902846C84710
:10C27000019B8BF31188E41A1F4486F31188DBE7D6
:10C28000C361009BC16081614161114400604060F5
:10C290008260016103627047F8B504460E46174696
:10C2A000302383F31188A568A5B1A368013BA3607F
:10C2B00063695A1C62611E70236962699A4224BFD5
:10C2C000E3686361E3690BB120469847002080F37F
:10C2D000118807E039462046FFF786FC0028E2DA9D
:10C2E00085F31188F8BD8369426910B59A4201D17E
:10C2F00082687AB982680021013282605A1C8261A8
:10C300001C7803699A4224BFC3688361FFF77CFCF1
:10C31000204610BD4FF0FF30FBE72DE9F74F0546F3
:10C320000F4690469A46D0F81C90302686F3118826
:10C330004FF0000B144664B1224639462846FFF7F9
:10C34000F0FE034668B951462846FFF74DFC002829
:10C35000F1D0002383F31188A8EB040003B0BDE8FB
:10C36000F08FB9F1000F03D001902846C847019B18
:10C370008BF31188E41A1F4486F31188DBE70C3035
:10C38000FFF74CBF4FF0FF330C30FFF747BF3030A3
:10C39000FFF7C3BF4FF0FF333030FFF7BEBF0C30A5
:10C3A000FFF716BF4FF0FF310C30FFF711BF3030F1
:10C3B000FFF772BF4FF0FF323030FFF76DBF01293A
:10C3C00014BF6FF013000020704700F009BE00009A
:10C3D000034637B515460D4A044643F8042B43601F
:10C3E00001238022037200900B4600F154010C30AF
:10C3F000FFF7C5FE00942B46802204F1D40104F11E
:10C400003000FFF73DFF03B030BD00BFF4F000087F
:10C4100010B53023044683F3118800F0F3FD0223A6
:10C420000020237280F3118810BD38B5436904469B
:10C430000D461BB904210844FFF718FC294604F1F6
:10C440000C00FFF7AAFE002806DA201D4FF4006159
:10C45000BDE83840FFF70ABC38BD302383F31188AC
:10C460000023406983F31188B0FA80F040097047D7
:10C470004FF0FF31FFF7A0BB00F08CBE012303702B
:10C4800000230C3040F8083C40F8043CFFF7D5BBD3
:10C4900010B53023044683F31188416000F086FE16
:10C4A00002230020237080F3118810BD10B53023C3
:10C4B000044683F3118800F0C7FE00230122636065
:10C4C000227083F3118810BD302383F311884368F1
:10C4D00099685A684FF480338B409361002383F34B
:10C4E00011887047302383F31188436899685A682C
:10C4F00001238B409361002383F31188704738B583
:10C500000446302585F31188032504F8085B00F004
:10C51000B9FE2046FFF7ACFF002383F3118838BD36
:10C5200010B53023044683F31188032304F8083B35
:10C5300000F0BDFE2046FFF79BFF002383F3118828
:10C5400010BD10B53023044683F31188032304F88B
:10C55000083B00F0C2FE2046FFF78AFF002383F36A
:10C56000118810BD01F0DEB8012303700023C36100
:10C5700083620362C3624362036343608360704704
:10C5800038B50546302383F3118800244160C46028
:10C5900004614461846101F0CBF802232B7084F3C1
:10C5A0001188204638BD70B53023064683F31188C4
:10C5B00001F0D6F8344600250123756004F80C3BE1
:10C5C0001C3654F8043B7BB1586920B16FF001016F
:10C5D0000C30FFF7FFFA54F8043C986920B16FF073
:10C5E00001010C30FFF7F6FAB44244F8045CE8D1DC
:10C5F000FFF71AFA85F3118870BD70B500EB81035F
:10C60000054650690E461446DA6018B1142200211E
:10C61000F4F71CF8A06918B114220021F4F716F8F9
:10C6200031462846BDE8704001F0B8B8F8B5044678
:10C630000027836800F1100503F00113836000F107
:10C640001C0655F8043B7BB1586920B16FF001011D
:10C650000C30FFF7BFFA55F8043C986920B16FF031
:10C6600001010C30FFF7B6FAB54245F8047CE8D179
:10C670002046BDE8F84001F01DB9F0B4012500EBFB
:10C680008104E4684789A4698D403D434581236066
:10C690000023A2606360E360F0BC01F07DB9F0B4F8
:10C6A000012500EB8104E468078964698D403D43FE
:10C6B000058123600023A2606360E360F0BC01F0A9
:10C6C0008BB90000037810B5052B10D1084C4FF43E
:10C6D0007A70E37A43F00803E372637843F004036B
:10C6E0006370FFF75CFA637803F0FB03637010BDBF
:10C6F000004001402DE9F0410223002504464FF09F
:10C7000030080370C564856000F10C0600F11C0759
:10C7100056F8043BABB188F3118856F8043C5869CD
:10C7200020B16FF001010C30FFF754FA56F8043CC9
:10C73000986920B16FF001010C30FFF74BFA85F3D7
:10C740001188BE4246F8045CE2D184F83450204699
:10C7500001F092F863681B6823B12046BDE8F04100
:10C7600000211847BDE8F081F8B503780446052B91
:10C7700029D080F850300523037043681B680BB143
:10C780000421984700263027A66004F10C051C34CC
:10C7900055F8043BABB187F3118855F8043C586950
:10C7A00020B16FF001010C30FFF714FA55F8043C8A
:10C7B000986920B16FF001010C30FFF70BFA86F396
:10C7C0001188A542E4D1F8BD0178052906D1436856
:10C7D00090F850201B68027003B1184770470000A2
:10C7E000F8B590F8343004460E4613B1002380F8B3
:10C7F000343004F144023146204601F0B1F8636858
:10C800009B68B3B994F8443013F0600538D0002128
:10C81000204601F021F90021204601F00FF963685C
:10C820001B6813B1062120469847062384F834304C
:10C83000F8BD204698470028E4D094F84B2094F89F
:10C840004A3043EA0223E26B9A4294F9442088BFBB
:10C85000E363002AE36B80F20781002B00F0FB808A
:10C86000092384F83430302383F311880021E36BEB
:10C87000A26B2046FFF713FF002383F31188D7E74D
:10C8800094F8452003F07F0343EA022340F202328A
:10C89000934200F0CC8025D8022B00F0A08009D86C
:10C8A000002B51D0012BB2D1774BA3630223E3635A
:10C8B00000234EE0B3F5817F00F0A680B3F5407F02
:10C8C00049D0B3F5807FA2D194F84630012B9ED198
:10C8D000B4F84C3023F00203A4F84C30A563E563B0
:10C8E0002564AAE740F2016293421DD8B3F5C06FF8
:10C8F0003BD2B3F5A06F8AD1B4F84430B3F5A06F42
:10C900000ED194F84630204684F84E3000F03EFFB9
:10C9100063681B6813B101212046984703232370E5
:10C920000023A363E36314E0B3F5106F33D040F644
:10C9300002429342B8D0B3F5006F7FF468AF04F1C0
:10C940004F03A363012324E004F14C02A2630222FB
:10C95000E263236471E794F84630012B7FF457AF0C
:10C96000B4F84C3043F00203B6E794F8492061680C
:10C9700094F848304F6843EA022394F8471094F83B
:10C9800046202046B84700283FF441AF4368A363E0
:10C990000368E363A4E72378042B10D1302383F3E7
:10C9A00011882046FFF742FE85F311880321636852
:10C9B00084F84F501B6821700BB12046984794F8BB
:10C9C0004630002BACD084F84F30042323706368CA
:10C9D0001B68002BA4D0022120469847A0E794F8BA
:10C9E000483020461D0603F00F010AD500F09CFFD9
:10C9F000012804D002287FF40AAF244B55E7244BCA
:10CA000053E700F075FFF3E794F84630002B7FF40E
:10CA1000FEAE94F8483013F00F0181D01A0620467C
:10CA200002D501F031F87BE701F022F878E794F8BD
:10CA30004630002B7FF4EBAE94F8483013F00F0132
:10CA40003FF46EAF1B06204602D501F005F867E7FC
:10CA500000F0F4FF64E7142384F8343031462046B4
:10CA6000BDE8F84000F08CBF63B1152384F8343082
:10CA7000302383F311880021E36BA26B2046FFF77C
:10CA8000FCFDF9E60B23E7E720F100081CF10008A4
:10CA90001EF1000808B500F0C9F80B4B9A6C42F083
:10CAA00020029A649A6C9A6C42F040029A649A6CE2
:10CAB0009A6C42F080029A649A6C9A6C42F480728A
:10CAC0009A649B6C08BD00BF000C014070471623A0
:10CAD00003604FF0FF3070470020704718467047E2
:10CAE0000020704710B50022044608460121FEF7D9
:10CAF0003FFE18B90C234FF0FF30236010BD08B57E
:10CB00001346002158221846F3F7A0FD4FF40052B7
:10CB10004260002008BD01207047000008B50248AF
:10CB2000FEF768FEF3F7E4FC13E7000808B50248D7
:10CB3000FEF760FEF3F7DCFC18E700080120704701
:10CB4000704700F16043090103F56143C9B283F8FE
:10CB50000013012300F01F024009800000F1604033
:10CB6000934000F56140C0F88031036070470122B6
:10CB700000F01F039A4043099B0003F1604303F553
:10CB80006143C3F88020C3F88021002300F1604096
:10CB900000F5614080F800337047090100F1604002
:10CBA000C9B200F56D4001767047000017498A68E8
:10CBB000022A12D0032A26D0154B1649012A18BF83
:10CBC0000B46124A926902F07F020132520801328A
:10CBD000B3FBF2F3104A13607047104A0B68526FB0
:10CBE00049686FEA9212012902F003020CBF08495A
:10CBF0000B49033203F01F034A4301335B0801333F
:10CC0000B2FBF3F3DDE7074BDBE700BF000C0140AD
:10CC1000006CDC0200127A00381100200004014090
:10CC20000048E801001BB700FFF7C0BF13B50C2098
:10CC3000032440F2BE71314B314A9C62D862C2F883
:10CC4000941000219962D9629C62D8628020C3F856
:10CC50001C0CD3F81C0CC3F81C0C009101914FF470
:10CC60000141C3F8481C4FF6FC71A3F574431963E6
:10CC70000F2119600223136501234BF68031D36421
:10CC8000936D03F001030193009B01330093019B1B
:10CC900013B9009B8B42F3D1019B03B9FEE7194BFB
:10CCA0001949012019600021A3F590439961802161
:10CCB0001962196A1962202158601960196819608F
:10CCC000196801431960C02151679067D16F03292A
:10CCD000FCD102229A6001220021DA60074A9162A7
:10CCE000D1629A6C42F400429A649A6CDA6C42F413
:10CCF0000062DA64DB6C02B010BD00BF00000140CE
:10CD0000000401400054014012000003144B834210
:10CD100025D1144B02201A6C134942F480721A6414
:10CD20001A6C42F002021A64D3F8882042F0020220
:10CD3000C3F88820D3F8882022F00202C3F88820A4
:10CD400001225A63DA670864DA6608225A615A696E
:10CD500042F004025A615A6942F001025A61704776
:10CD600020330020000C0140004C0140084B83425E
:10CD70000CD1084B5A6902F008025A6100225A612C
:10CD8000DA66DA671A6C22F002021A64704700BF92
:10CD900020330020000C01400F4A936C43F4004301
:10CDA00043F0200393644FF080436FF4C0521A6342
:10CDB0004FF07072DA624FF020721A6000225A60EF
:10CDC0009A60DA604FF44C325A62012203F5A033C4
:10CDD0005A700722DA727047000C01400E4A6FF455
:10CDE0008051936C43F4004343F0200393644FF06D
:10CDF00080436FF4C0521A6300221A609A60DA60AE
:10CE000019634FF0807119604FF4805159605A6274
:10CE10004FF080529A617047000C0140062108B51E
:10CE20000846FFF78EFE06210720FFF78AFE06213F
:10CE30000820FFF786FE06210920FFF782FE062163
:10CE40000A20FFF77EFE06211020FFF77AFEBDE8DC
:10CE5000084006212120FFF774BE7047C9434FF0F8
:10CE60005533016302F003015943016042F380012D
:10CE70004160C2F3C10159438160C2F3411159437A
:10CE8000C160C2F3C1214B43C3624FF01133C2F3FF
:10CE9000C3125A43026242627047000040F2CF223E
:10CEA000044B08215A6000229A6007220B201A6066
:10CEB000FFF773BE10E000E008B5302383F311885C
:10CEC000FEF7A4FC002383F3118808BD08B5FFF723
:10CED000F3FFBDE80840FEF70BBF0000024A5368AD
:10CEE00043F0020353607047003800402DE9F041E1
:10CEF000384DD5F854717B69D806DCB20AD5302399
:10CF000083F311884FF48061281DFEF7AFFE0023E4
:10CF100083F31188302383F311882F4EA6F1040880
:10CF200014F00F0332D183F311887B68980714D56E
:10CF3000A10612D5302383F311882848FFF7D3F9CF
:10CF4000002844DA08212448FEF790FE7B6823F08D
:10CF500002037B60002383F311887B689A0711D555
:10CF600063060FD5302383F311886A6CAB6C9A4249
:10CF700005D1AB6B1BB110211748FEF777FE0023DC
:10CF800083F31188BDE8F041FEF7B2BE14F0020F42
:10CF900014BF4FF480710021620748BF41F02001A7
:10CFA000230748BF41F0400114F0010418BF41F0CD
:10CFB00080013046FEF75AFE3B682CB195F85811B7
:10CFC00040461940FFF731FA7C69E4B2A8E73860BF
:10CFD000C0E700BF9031002094310020C031002014
:10CFE00010B5054C054A00212046FFF7F1F9044B26
:10CFF000C4F8543110BD00BF90310020DDCE0008D0
:10D000000038004038B5294C037A002918BF0C4677
:10D01000012B05461AD1264B984217D1254B0C21DE
:10D020009A6C1E2042F480429A649A6CD3F8902045
:10D0300042F48042C3F89020D3F8902022F480423A
:10D04000C3F89020D3F89030FFF77BFDD5F854312A
:10D05000E1791A6902F050020A431A612168164AFE
:10D0600002EB5102B2FBF1F202F00F01C3F8C01063
:10D070008021D960C2F3071119600021C2F3073281
:10D080005A60D960607922790243A0790243DA605C
:10D090000122C3F89C10C3F898205A6842F0050298
:10D0A0005A60FF2385F8583138BD00BF24F10008CD
:10D0B00090310020000C014000A24A0470B5334CAE
:10D0C000E5692E6BE26A6B6A9A4234BFE36A6B6A67
:10D0D00013F1FF3338D2E36A002B41D1EB6263686E
:10D0E0001B6833B104222948227098472378042B07
:10D0F00001D102232370302383F3118800212448B7
:10D10000FEF768FD002383F31188F30718D5286A1A
:10D11000228E666AE36A616AD31A3344121A934212
:10D1200028BF134699424FF6FF7138BF636A13F167
:10D13000FF331ED2636A1BB9EB6A23F00103EB6273
:10D14000BDE87040FEF7D4BD296EE26A013AE262A2
:10D15000A26A002ABCD01170A26A0132A262B7E7AB
:10D16000E26AEB699A429EBFE36A03F1FF33EB6127
:10D17000CBE7626A013A6262226A0AB92966D6E797
:10D1800012F8010B28662262D1E700BFEC320020C2
:10D19000F432002010B5034C2046FFF76FF9024B24
:10D1A000E36110BDEC32002000300040037810B580
:10D1B000012B044622D1224B98421FD1214B0A2138
:10D1C0009A6C1A2042F480529A649A6CD3F8902098
:10D1D00042F48052C3F89020D3F8902022F4805279
:10D1E000C3F89020D3F89030FFF7ABFC6268E36996
:10D1F000128A5A611A6942F001021A616168E36990
:10D20000CA8989890A4342F00702218E92B21A60C4
:10D2100069B901229A619869904205D10132B2F54B
:10D22000807FF7D191B201E0012AFBD12186002253
:10D230009A61DA61DA6A22F0FF02DA629B6C10BD51
:10D24000EC320020000C014008B50378022B13D10A
:10D250000022C3699A60DA6A22F0FF02DA629B6CEC
:10D26000064B984208D11A20FFF781FC044B9A6CB8
:10D2700022F480529A649B6C08BD00BFEC320020FF
:10D28000000C014091B18362038E41625B089942B8
:10D29000C16228BF1946C369026299610139D96127
:10D2A000DA6A42F01102DA6201229A60704799B19B
:10D2B00000238362038E41625B089942C16228BFEA
:10D2C0001946C369026299610139D961DA6A42F08B
:10D2D0001102DA6201229A60704799B10023036259
:10D2E000038E41625B089942C16228BF1946C36937
:10D2F000826299610139D961DA6A42F01102DA6217
:10D3000001229A60704700000A4A0B4B10B502EBED
:10D310008002987338B1DC7D987D40EA04200B18B8
:10D32000994203D110BD987DC0B2F8E7147801F896
:10D33000014BF5E7204001400040014090F83420C7
:10D3400010B5152A04460CD8012393400C4A134209
:10D3500008D19B0205D5036C03B19847002384F8DC
:10D36000343010BD00216022064B99735A749973B2
:10D370005A7443681B680BB1062198470623EEE7F1
:10D38000410E1000004001402DE9F843244C00F10B
:10D39000020804EB8803D3F80490224ED9F8185001
:10D3A000B073337D0746DB0733D5A968FFF7ACFFC1
:10D3B000AB68B9F812200344AB606B689042034439
:10D3C0006B602B68A3EB00032B602B8A03F1FF3308
:10D3D0009BB22B8200D3F3B9012303FA07F26389CE
:10D3E00023EA0203638104EB88035B68DB6813B103
:10D3F00039460B489847302383F3118804EB88049F
:10D400006368986941680C30FEF7E4FB002383F3FE
:10D410001188BDE8F883337D03F0FE033375F8E728
:10D420002033002000400140F8B5214C871C04EB5C
:10D4300087035E680146726950681568A84219D36F
:10D44000012303FA01F2238923EA02032381B3684B
:10D450000BB120469847302383F3118804EB8704EF
:10D460006368002158690C30FEF7B4FB002383F396
:10D47000118817E00F4B9973136918445060281AEC
:10D48000DED0348A844228BF044690681461034485
:10D490000948936000EB81011C449C4203D10122A6
:10D4A000044B5A74F8BD13F8012B0A70F5E700BF5E
:10D4B00020330020004001402040014090F83420FB
:10D4C00010B5152A04460CD8012393400C4A134288
:10D4D00008D19B0505D5036C03B19847002384F858
:10D4E000343010BD00216022064B99735A74997331
:10D4F0005A7443681B680BB1062198470623EEE770
:10D50000410C3000004001402DE9F047824B9E79EC
:10D51000F6B2B70702D58148FFF756F9750702D56D
:10D520007E48FFF7E7F8340713D57C4C6368DB6867
:10D5300023B9794AD37A03F0F703D3722378052B02
:10D5400002D17648FFF740F96368DB680BB1734896
:10D550009847714A9378177903F0FF08FFB253B9DF
:10D56000002F3DD1F30702D56C48FFF7FDF8BDE869
:10D57000F047FEF7BDBB18F0010F1FD00021674C2C
:10D58000D4F80C909173537CDBB2580744BF5174AC
:10D5900084F83410DA0605D580215F4A51740022E0
:10D5A00084F8342094F834200AB1062A28D1DB0705
:10D5B00004D5D9F8043000215848984718F0020FD4
:10D5C00002D00120FFF730FF18F0040F02D0022034
:10D5D000FFF72AFF18F0080F02D00320FFF724FFFF
:10D5E000B80702D50120FFF7CFFE790702D5022048
:10D5F000FFF7CAFE3A07B5D50320FFF7C5FEB1E72E
:10D60000092A49D1444D6B7CDBB213F00201D5D11C
:10D6100003F01103112BD1D0D9F81420A97351684C
:10D620001369106819445160411AB9F810E017D015
:10D63000714528BF71469068116103443848936072
:10D640005A18934208D1B9F810308B4294BF022186
:10D650000A21314B5974B1E713F8014B0470F0E71C
:10D66000734503D10A236B741161A7E7238923F063
:10D6700001032381D9F808300BB12848984730239B
:10D6800083F311880021E36858690C30FEF7A2FA91
:10D69000002383F3118891E7152A8FD1DFF878A052
:10D6A0009AF81130DD0789D5D9F818500020A968FB
:10D6B000FFF72AFEAB68B9F812200344AB606B6831
:10D6C000904203446B602B684FF00002A3EB000311
:10D6D0002B602B8A03F1FF339BB22B8200D3A3B9BB
:10D6E0000D4B9A7348225A74638923F001036381B6
:10D6F000E368DB6813B1002108489847302383F3BF
:10D700001188E36898694168BFE740238AF80E20D2
:10D710008AF8113052E700BF00400140203300205A
:10D72000204001400148FEF71FBF00BF203300200A
:10D7300010B50478012C0ED1074AC260FFF7E6FA53
:10D740000022064B0D21DA72DC715A720E20BDE800
:10D750001040FFF7F6B910BD2CF100080040014061
:10D76000037810B5012B04460CD00E20FFF7FFF90B
:10D770000022054B2046DA72DA715A72BDE8104079
:10D78000FFF7F4BA10BD00BF0040014090F84E20F2
:10D79000014B1A70704700BF0040014000EB810050
:10D7A000344BC26801F00F0110B59973106800F096
:10D7B0000300002956D002282CD003282AD00128A3
:10D7C00027D153690BB993691BB3E020294B987497
:10D7D000108AC0F3C7001874402058740820587489
:10D7E00058740120DC7900FA01F149B241EA0400E1
:10D7F000C0B2D871C0205875528AC2F3C702DA7419
:10D8000080221A7510221A751A755A7A1143C9B2F4
:10D81000597210BD506980B100209874108AC0F30D
:10D82000C700187440205874082058745874012098
:10D83000DC7988402043C0B2D8719369002BE8D0CE
:10D8400000200C4B5875528AC2F3C702DA7480224A
:10D850001A7510221A751A750122587A02FA01F106
:10D860000143D4E70028D4D1DA7942F00102DA7119
:10D87000CFE700BF00400140002208B50B4BDA7132
:10D880005A724268D2681AB1DA7A42F00802DA7241
:10D89000074B0021C360FFF781FF0122034B5A7041
:10D8A000DA7A42F00102DA7208BD00BF004001409E
:10D8B0002CF1000870B50D4B0021DA79402602F0FA
:10D8C0000102DA71082401228025102059729A730E
:10D8D0000132D2B2042A99745E745C745C74597516
:10D8E0001D7518751875F2D170BD00BF004001405C
:10D8F0000C4B01F00F029A7341B95A7C52070ED4B7
:10D90000D87910F0010018BF02207047187D10F080
:10D91000200004D15B7A134113F0010FF3E70120DB
:10D92000704700BF004001400C4B01F00F029A739A
:10D9300041B95A7C52070ED4D87910F0010018BFB3
:10D9400002207047587C10F0100004D1DB7913419D
:10D9500013F0010FF3E70120704700BF00400140C2
:10D96000064B01F00F0103EB810302F10801187867
:10D9700002F8010B9142FAD1704700BF20400140EC
:10D980004822044B01F00F0199735A74002380F868
:10D99000343070470040014010B501F00F0400EB37
:10D9A0008101CB6899690A6872B1588A1318013BE2
:10D9B000B3FBF0F39BB20B82064B9C7334B11A7D20
:10D9C00002F0FE021A7510BD0123F4E740225A74DA
:10D9D000F9E700BF0040014000EB810311F00F01A7
:10D9E00070B508BF4025DC6808BF124A636904BFF0
:10D9F00091735574228A1D680F4CAA4228BF2A468B
:10DA00001A619B6804EB81049D189D4205D1094B66
:10DA1000997331B101225A7470BD13F8016B2670ED
:10DA2000F3E7597CC168098A914294BF02220A2215
:10DA3000F1E700BF0040014020400140054B01F0EC
:10DA40000F01997311B120221A75704760225A7420
:10DA5000704700BF00400140044B01F00F01997373
:10DA600011B110225A7470476022FBE70040014058
:10DA7000044B01F00F01997311B180221A757047A0
:10DA80005974704700400140044B01F00F01997335
:10DA900011B140225A7470475974704700400140D8
:10DAA000074BD3E902128A4208D0596801F59C70ED
:10DAB000824201D1D96070470832DA60704700BFF6
:10DAC000AC2D00200023074930B51A460C4683428E
:10DAD00001D1E25430BD11F8015B01332A44D2B2C6
:10DAE000F5E700BF782500202DE9F84303461646E8
:10DAF0001A481B4C00F8013BF2F732FDD4E90187CC
:10DB000008F59C794F4506F10106E36804D1984574
:10DB100006D10020BDE8F88307F108029342F7E739
:10DB2000104A216902F2CF735B1A312B98BF226130
:10DB3000322EEED82569324628460849F2F710FD04
:10DB40004F453D6035447D6018BF083725610CBFE7
:10DB5000C4F80880A7600120DCE700BF342F002054
:10DB6000AC2D0020DC2500200368044905220B6051
:10DB7000037907200B71FFF7B7BF00BFC025002056
:10DB800070B505461F4C003044F0010418BF012059
:10DB9000A047286A1C4E003018BF0120A047012072
:10DBA000A047686B003018BF0120A0470024174B26
:10DBB000174A18495A601961C2E90011C3E90222E3
:10DBC0001C704FF4E1302B6A3560984701223368AE
:10DBD0002146C3E90544DA751A766422DC619A7736
:10DBE0000D4B0E221C700D4B0D481C605C60F2F753
:10DBF0002DFD0C4B1C800C4B1C601C710B4B1C70C6
:10DC000070BD00BF8CF10008B0250020AC2D0020B5
:10DC1000F42D0020DC250020B6250020B8250020AA
:10DC2000C5250020B4250020C02500206C2F002031
:10DC3000004870471DE70008034BD8689B68C01A6E
:10DC400018BF0120704700BFAC2D002038B5184C1C
:10DC500000252378032B29D8DFE803F0020C1620D7
:10DC60000A23144843708570FFF77EFF08B1012333
:10DC7000237038BDF6230F4845708370FFF774FF9B
:10DC80000028F6D00223F3E7F6230A484370857094
:10DC9000FFF76AFF0028ECD00323E9E70A230548D1
:10DCA00045708370FFF760FF0028E2D02570E0E741
:10DCB000B7250020C025002007B501228DF80700F8
:10DCC0000DF107010620FFF70FFF03B05DF804FB1D
:10DCD00038B504460E4D0F4B286843F00103003061
:10DCE00018BF01209847601EC0B204280ED80A4A07
:10DCF0002B68125C53F822402046F2F72FFE214693
:10DD0000BDE8384002460820FFF7EEBE002038BDCF
:10DD1000B02500208CF1000886F1000808B1FFF75B
:10DD200023BF7047082202490120FFF7DDBE00BF74
:10DD3000B82500200E2202490220FFF7D5BE00BF01
:10DD4000C52500202DE9F74F984C80462068984E55
:10DD5000003046F0010618BF01200F46B04720688A
:10DD6000944D003018BF0120B0472368DFF860925F
:10DD7000186B003018BF0120B0472368586A003084
:10DD800018BF0120B04723681B6B984700283FD07D
:10DD900023685B6A984795F83220012A52D0002AFE
:10DDA00047D0022A57D099F80030002B6FD0A854E2
:10DDB000013B0132D2B2DBB285F8322089F8003063
:10DDC000002BE0D119467B48013A914261D3AA5C0D
:10DDD0009A425CD14AF66623ADF80430BB238DF835
:10DDE0000630236803219B6A01A8984700226B78BC
:10DDF00085F832205B2B52D05C2B00F089805A2BA7
:10DE000040F08A80EB7813F0F80F01D12268D377C5
:10DE10002068003018BF0120B047674A1378914648
:10DE2000032B00F29080DFE813F0DC007B00B100F0
:10DE3000D500662801D0AC28A5D10123287085F82B
:10DE40003230A0E75A2822D35C2801D9AA281ED153
:10DE500068700223F3E7BB284FF0030310D12A7840
:10DE60002168662AA87085F832308CD16A78AA2A8F
:10DE700089D1002285F832200A754F4A137082E753
:10DE8000A870013085F8323089F800007BE7002364
:10DE9000D5E710F801CB01316344DBB295E7E978AF
:10DEA0002368322927D00FD822291DD004D8212950
:10DEB000AED101225A75ABE7232918D03129A7D159
:10DEC00001211983DA77A3E735291AD006D8332937
:10DED00015D034299CD101221A7799E7362914D01C
:10DEE000422995D11A7593E70122DA8290E75A7593
:10DEF0004FF48072F9E74FF480721A8388E71A832F
:10DF0000E0E7012199765A76DCE70121D976FAE734
:10DF10002368EA789A777BE70322274B1A7077E722
:10DF20002368264D5B6B98472B68984223685B6B90
:10DF300027D398472B68C01A214B1B78834202D203
:10DF4000022389F80030B8F1000F00F06881B8F1C1
:10DF5000060F40F06C81002F00F05381194C23789C
:10DF6000D90704D523F001032370FFF7DBFE2378E4
:10DF70009A0740F1548123F002032370FFF7DAFE81
:10DF80004DE198472B68DB431844D5E70E4A0F490B
:10DF9000137809780133DBB29942137003D200235E
:10DFA0001370FFF77DFD0023CBE700BFB0250020F5
:10DFB0008CF1000844250020AC2D0020682F0020A3
:10DFC0003C110020B6250020D42500203D11002062
:10DFD000D3250020FFF764FD0023A24A89F8003012
:10DFE0001370D9E902239342ADD0D3E900159E4BBB
:10DFF0006D1A2A461846F2F7B3FA8246002DA2D0CF
:10E00000206805F1FF3B003018BF0120B0471E22F9
:10E010009649974B0A701A709AF800200C2A1DD85E
:10E02000DFE812F00D00140044005C006C007A0080
:10E0300082009300A500BC00C400CC00DB000522D8
:10E040008C4B5A638C4A1A6004201BE023681B7DAA
:10E0500033B1002211461046FFF746FD032370E757
:10E0600003230C220B70834B0B205A6345F2AC1236
:10E070001A80082281499A700A68C3F803204A6806
:10E08000C3F80720FFF71EFD2368986A003018BF09
:10E090000120B04777482368818E9B6A98472368A0
:10E0A0005B6B9847764B186001234AE703231222E3
:10E0B0000B70704B5A6345F2AC221A800E229A7094
:10E0C0006E4A033302F10C0152F8040B8A4243F802
:10E0D000040BF9D1128811201A80D3E703230622FA
:10E0E0000B70644B05205A6345F2AC321A80022251
:10E0F0009A70BAF80120A3F80320C3E7032305228E
:10E100000B705C4B5A6345F2AC421A8001229A7044
:10E110009AF80120DA7097E7032305220B70554B1C
:10E120005A6345F2AC52F0E70521524A9AF80100D1
:10E13000516345F2AC611180012153289170D07078
:10E1400016BF102219701A707EE7032309220B7084
:10E15000484B08205A6345F6AC021A8005229A7093
:10E16000464A11681279C3F80310DA718AE745F656
:10E17000AC12DFF800A10335CAF83450AAF8002029
:10E1800010221A705A463D498AF802B00AF103007B
:10E19000F2F7E6F9DAF83400013873E7DFF8D4A0D3
:10E1A0000335CAF8345045F6AC32E7E7DFF8C4A0CF
:10E1B0000335CAF8345045F6AC42DFE7DFF8B4A0C7
:10E1C00045F6AC52504620F8022B102202351A7048
:10E1D000CAF834505A462949DAE70323254D6B63C0
:10E1E0004AF666232B80BB23AB702368986A003005
:10E1F00018BF0120B0472368A98E9B6A284698471C
:10E200002CE723681F4D5B6B98472B689842236867
:10E210005B6B07D398472B6898427FF49FAE03B09F
:10E22000BDE8F08F98472B68C01A0128F5E7154D17
:10E2300027B123685B6B984728608FE623685B6B88
:10E2400098472B68984223685B6B05D398472B68E7
:10E25000C01A0728EDD8E2E798472B68DB43034450
:10E26000072BF7E7D4250020C02D00203C1100200B
:10E270003D11002078250020AC560100C12D002062
:10E28000682F0020D8250020022202490320FFF732
:10E290002BBC00BFB4250020012202490420FFF757
:10E2A00023BC00BF6C2F0020244B08201A4610B559
:10E2B00013F8011B91B3002313605360FFF732FD85
:10E2C000012000231E4A12F8011B61B30E22002117
:10E2D0001B48F2F7BBF9FFF72DFD0120194B197808
:10E2E0005A780A4304D000221A80FFF7CDFF01209C
:10E2F000154A0023114612F8014BCCB100231248F5
:10E300000B600B71FFF70AFD0120104B1A7822B148
:10E3100000221A70FFF7C0FF012010BD013810F075
:10E32000FF00C5D1CDE70133DBB20E2BCBD1D5E752
:10E330000133DBB2052BDED1E7E700BFB8250020B3
:10E34000C5250020B4250020C02500206C2F00200A
:10E35000F8B504461F464A4B4A4A186842F0010283
:10E36000003018BF01200D469DF818609047231F0C
:10E37000A02B43D8444A022315B3D55CA5421AD03A
:10E380003DB9D454414A137843F001031370284631
:10E39000F8BD0133082BF0D16EB1E30804F007019A
:10E3A00001243B4A8C40D15C0C43D454374A137847
:10E3B00043F0020313700025E9E70133082B09D06D
:10E3C000D15CA142F9D10021D154304A137843F0F5
:10E3D000010313702E48E108435C04F0070443FA7C
:10E3E00004F2D207E7D5012202FA04F4274A23EA0D
:10E3F00004034354137843F00203C7E7A4F1E00297
:10E4000093B2072B16D86DB10FB1E32C05D00123C1
:10E410001D4993400A7813430B701C4A137843F04C
:10E420000103C7E70123184903FA02F20B7823EA34
:10E430000203F1E7A4F1A50083B2022B0FD8012259
:10E440001449824091F9003052B22DB11343DBB22E
:10E450000B70FFF721FFAEE723EA0203F7E7A4F111
:10E46000A8031A2B0AD825B158340B4BE4B233F861
:10E4700014500A4B1D80FFF707FF9CE7012586E734
:10E48000B02500208CF10008B8250020B62500201A
:10E49000C52500206C2F002050F10008B425002075
:10E4A0004B4A494847464544434200FF4400000068
:10E4B0000020202020202020202028282828282054
:10E4C000202020202020202020202020202020204C
:10E4D00020881010101010101010101010101010B4
:10E4E00010040404040404040404041010101010A4
:10E4F000101041414141414101010101010101016E
:10E5000001010101010101010101010110101010BF
:10E51000101042424242424202020202020202023F
:10E520000202020202020202020202021010101093
:10E5300020000000000000000000000000000000BB
:10E5400000000000000000000000000000000000CB
:10E5500000000000000000000000000000000000BB
:10E5600000000000000000000000000000000000AB
:10E57000000000000000000000000000000000009B
:10E58000000000000000000000000000000000008B
:10E59000000000000000000000000000000000007B
:10E5A000000000000000000000000000000000006B
:10E5B00000000000040C002000000000000000002B
:10E5C000000000000000000000000000000000004B
:10E5D000000000000000000000000000000000003B
:10E5E000000000000000000000000000000000002B
:10E5F000000000000000000000000000000000001B
:10E60000000000000000000000000000000000000A
:10E61000000000000000000081828300E200E900A9
:10E62000EA00B500B600B700CD008301CC008A0136
:10E6300092019401210223022402250226022702CC
:10E640002A02B300B4006F0070009F01CB019F024B
:10E65000A002000000000000C0D40100E09304000C
:10E66000C0270900804F120040771B0080EE360063
:10E6700060EA00000D0A6B6579626F617264207652
:10E6800065723A204B425F56455253494F4E000D3A
:10E690000A636F7265207665723A20302E32322E10
:10E6A00031342D31372D676231326662662D6469EF
:10E6B0007274790D0A000D0A6275696C64206461D8
:10E6C00074653A20323032362D30312D31322D31D1
:10E6D000323A30393A3535004A616E652042542D60
:10E6E00031004A616E652042542D32004A616E65E8
:10E6F0002042542D33005742204B422034005742D1
:10E70000204B422035006330006D61696E00696402
:10E710006C650065786974006B696C6C0062747379
:10E72000206C69622078746B2076657273696F6EF5
:10E730003A2076312E352E340000000000080040CB
:10E7400001080040020800400308004005000040A6
:10E750000408004005080040000400400104004097
:10E760000A0400400B0400400C0400400D0400406B
:10E770000E04004007080040080800400908004057
:10E780000948032181620C21C162084890F81003F6
:10E79000074900F00F000A68824200D0086000209C
:10E7A000401C2328FCDB70470000014000F0FF1FE5
:10E7B000040401400748032181620C21C16206481C
:10E7C000016801F00F01082901D90821016000BF8B
:10E7D00000BF7047000001400404014003000040F6
:10E7E000000000400100004004000040020C004016
:10E7F0000F0000400608004021522C00E2000000FB
:10E8000029003A003B003C003D003E003F00400034
:10E8100041004200430044004500137E460047008B
:10E82000480035001E001F002000210022002300A8
:10E8300024002500260027002D002E002A00490074
:10E840004A004B002B0014001A00080015001700A6
:10E850001C0018000C00120013002F0030003100C3
:10E860004C004D004E00390004001600070009005E
:10E870000A000B000D000E000F00330034003200C0
:10E880002800000000000000E10064001D001B00E3
:10E89000060019000500110010003600370038008E
:10E8A000E5008700000052000000E000E300E20005
:10E8B000000000002C002C0000000000E400E70035
:10E8C000E60021520000500051004F0000000000FF
:10E8D0000000000000000000000000000000000038
:10E8E0000000000089002800000000000000037CF8
:10E8F000BD00BE00B100B300B500B200AC00AE0078
:10E90000AB00A800AA00A90001000100010001005D
:10E910000100007E017E027E057E067E0100010070
:10E920000100010001000100010001000100237845
:10E9300001000100010001000100010001000100CF
:10E94000010049000100460001000100217801009A
:10E9500001000100010001000100010001000100AF
:10E960000100010001002078010001000100010008
:10E970000000000000000100010001000100010092
:10E98000010001000100147E0100010001000100EE
:10E99000010000002778000001000B70010000005A
:10E9A0000000077E077E000000000100010001005A
:10E9B000010000002A782878297800000000000073
:10E9C0000000000000000000000000000000000047
:10E9D0000000010001000000000000002900BD004F
:10E9E000BE0052012C082C085101AC00AE00AB0057
:10E9F000A800AA00A900137E460047004800350081
:10EA00001E001F00200021002200230024002500FA
:10EA1000260027002D002E002A0049004A004B0046
:10EA20002B0014001A000800150017001C00180025
:10EA30000C00120013002F00300031004C004D007C
:10EA40004E00390004001600070009000A000B0000
:10EA50000D000E000F0033003400320028000000CB
:10EA600000000000E10064001D001B00060019000A
:10EA7000050011001000360037003800E50087005F
:10EA8000000052000000E000E200E300000000008F
:10EA90002C002C0000000000E400E700E6002352F8
:10EAA0000000500051004F00000000000000000076
:10EAB0000000000000000000000000000000000056
:10EAC00089002800000000000000037C3A003B00A1
:10EAD0003C003D003E003F0040004100420043003A
:10EAE0004400450001000100010001000100007E1A
:10EAF000017E027E057E067E01000100010001000C
:10EB00000100010001000100010023780100010063
:10EB10000100157E01000100010001000100490013
:10EB20000100460001000100217801000100010000
:10EB300001000100010001000100010001000100CD
:10EB40000100207801000100010001000000000028
:10EB500000000100010001000100010001000100AE
:10EB6000010000000100010001000100010000009F
:10EB70002778000001000100010000000000077E6E
:10EB8000077E0000000001000100010001000000FC
:10EB90002A78287829780000000000000000000092
:10EBA0000000000000000000000000000000010064
:10EBB000010000000000000081828300E200E90003
:10EBC000EA00B500B600B700CD008301CC008A0191
:10EBD0009201940121022302240225022602270227
:10EBE0002A02B300B4006F0070009F01CB019F02A6
:10EBF000A002000000080040010800400208004098
:10EC000003080040050000400408004005080040DB
:10EC100000040040010400400A0400400B040040CE
:10EC20000C0400400D0400400E04004007080040A2
:10EC300008080040090800400300004000000040B0
:10EC40000100004004000040020C00400F000040A2
:10EC500006080040003131295A1B750A81930008CB
:10EC60008D930008C5930008E59300080001010199
:10EC70000101010101010202020202020202020379
:10EC80000303030303030304040404040404050549
:10EC9000050505060606060607070707070808080C
:10ECA00008090909090A0A0A0B0B0B0C0C0C0D0DBB
:10ECB0000D0E0E0E0F0F0F10101111111212131353
:10ECC0001414151516161717181819191A1A1B1BCC
:10ECD0001C1D1D1E1E1F2020212222232424252628
:10ECE00026272829292A2B2C2D2D2E2F3031323260
:10ECF000333435363738393A3B3C3D3E3F4041426C
:10ED0000434445464748494A4C4D4E4F5051535451
:10ED1000555658595A5B5D5E5F6162646566686905
:10ED20006B6C6D6F7072737577787A7B7D7E808285
:10ED3000838587888A8C8E8F91939596989A9C9ECE
:10ED4000A0A2A3A5A7A9ABADAFB1B3B5B7BABCBEDE
:10ED5000C0C2C4C6C9CBCDCFD1D4D6D8DBDDDFE2AB
:10ED6000E4E7E9EBEEF0F3F5F8FAFDFF0000000050
:10ED70000000000000000000000000000000000093
:10ED80000000000000000000000000000000000083
:10ED9000000000002A2B28000000000000000000F6
:10EDA0000000000000000029000000002C1E34209C
:10EDB000212224342627252E362D3738271E1F20C2
:10EDC0002122232425263333362E37381F04050607
:10EDD0000708090A0B0C0D0E0F101112131415164B
:10EDE0001718191A1B1C1D2F3130232D3504050649
:10EDF0000708090A0B0C0D0E0F101112131415162B
:10EE00001718191A1B1C1D2F3130354C000000003B
:10EE10007E0F00D4FFFFFFC7000000780300000052
:10EE2000000000004DAD00080000000008000000D8
:10EE3000802300200000000002000000000000000D
:10EE400003000000000000004DAD000800000000BD
:10EE500020000000DC230020000000000200000071
:10EE600000000000F5AD000881AD00084DAF0008BE
:10EE7000D9AD000850EF000854EF00085AEF000821
:10EE800004040A00B1EE0008CAEE0008EAEE000829
:10EE90000CEF000866EF000888EF00084422B6096E
:10EEA000025B00030100A0FA090400000103010154
:10EEB0000009211101000122440007058103080017
:10EEC00001090401000203000000092111010001F1
:10EED000222200070582032000010705020320000B
:10EEE00001090402000103000000092111010001D1
:10EEF00022B6000705830320000112010002000072
:10EF00000040136101100001010200010501090622
:10EF1000A101050719E029E71500250195087501EC
:10EF200081029501750881010507190029FF150067
:10EF300026FF0095067508810005081901290515A9
:10EF4000002501950575019102950175039101C098
:10EF5000040309040403200000000A034A006100BE
:10EF60006E00650000000660FF0961A101096215DD
:10EF70000026FF009520750881020963150026FF11
:10EF800000952075089102C005010902A1018502C2
:10EF90000901A10005091901290815002501950895
:10EFA000750181020501093009311581257F95021E
:10EFB0007508810609381581257F95017508810638
:10EFC000050C0A38021581257F950175088106C058
:10EFD000C005010980A101850319012AB7001501A7
:10EFE00026B700950175108100C0050C0901A1012B
:10EFF000850419012AA002150126A00295017510A9
:10F000008100C005010906A1018506050719E0294F
:10F01000E7150025019508750181020507190029EA
:10F02000EF1500250195F0750181020508190129E8
:10F0300005950575019102950175039101C00000C8
:10F040000000000069B4000859B4000889B4000841
:10F0500079B4000883B4000873B4000863B40008EE
:10F0600053B4000800000000C0F700089C330020E3
:10F070009C3300209C330020C0F7000800000000F3
:10F080000000000000000000C0F7000800000000C1
:10F090000000000000000000C0F7000800000000B1
:10F0A0000000000000000000C0F7000800000000A1
:10F0B0000000000000000000C0F700080000000091
:10F0C0000000000000000000C0F700080000000081
:10F0D0000000000000000000C0F700080000000071
:10F0E000000000000000000006E7000818240020CF
:10F0F000282500200000000095C3000885C30008F3
:10F10000B5C30008A5C30008AFC300089FC300082B
:10F110008FC300087FC30008BFC3000800000100C0
:10F120000000000000960000030000000000000046
:10F13000E1C70008BDD400083DD3000840004000EE
:10F140002825002028250020010000003C25002063
:10F15000E200E900EA00B500B600B700CD00830187
:10F16000CC008A019201940121022302240225028B
:10F17000260227022A02B300B4006F0070009F012C
:10F18000CB019F02A0020001020304000549D1F84F
:10F190000012054A114010B10448814200D0FEE738
:10F1A0007047000000F0FF1FFF3F00F08029003093
:10F1B0005245454E54206D616C6C6F6320737563CE
:10F1C00063656564656400002E2E2F2E2E2F2E2E73
:10F1D0002F2E2E2F2E2E2F2E2E2F2E2E2F2E2E2F49
:10F1E0006E65776C69622F6C6962632F7374646CEF
:10F1F00069622F72616E642E630000002C206675B8
:10F200006E6374696F6E3A2000000000617373656D
:10F210007274696F6E2022257322206661696C65A5
:10F22000643A2066696C6520222573222C206C6963
:10F230006E65202564257325730A0000232D302B6D
:10F2400020000000686C4C0065666745464700007A
:10F25000303132333435363738394142434445460C
:10F2600000000000303132333435363738396162CE
:08F27000636465660000000004
:08F27800A40FFF7F010000005C
:10F28000040C002000000000F8E50008D8E50008A4
:10F29000B8E50008000000000000000000000000C9
:10F2A000000000000000000000000000000000005E
:10F2B000000000000000000000000000000000004E
:10F2C000000000000000000000000000000000003E
:10F2D000000000000000000000000000000000002E
:10F2E00000000000D8E60008E2E60008ECE60008AE
:10F2F000F6E60008FEE6000800000000000000003E
:10F300000000000025AB000871AB000885AB0008C9
:10F3100099AB0008ADAB000811AA0008000000007E
:10F320000000000000000000CD2600086133000846
:10F3300085330008F92300083D27000869220008EA
:10F3400000000000B80B0000007E0000000000007C
:10F35000B80B0000017E000000000000B80B0000A8
:10F36000027E000000000000B80B0000037E0000D9
:10F3700000000000B80B0000047E00000000000048
:10F38000B80B0000057E000000000000B80B000074
:10F39000437E000000000000B80B0000037C00006A
:10F3A00000000000B80B0000117E0000000000000B
:10F3B000B80B0000127E000000000000B80B000037
:10F3C000137E00004D4E4F505152535455565758CE
:10F3D000595A5B5C5D4C4B4A494847464544434259
:10F3E00041403E3D3C3B292A2B2C2D2E2F303132E3
:10F3F0003334353638393A2827262524232221204C
:10F400001F1E1D1C1BFFFFFF0D0E0F1011121314EA
:10F4100015161718191AFF00FF0C0B0AFFFF090831
:10F42000FFFF07060504FF030201FFFFFFFFFFFFC9
:10F43000FFFFFFFFFFFF3F37FFFFFFC734D440C789
:10F4400040BB40AA409B408C407C4050403C402008
:10F450004011400240083410341C34283434344005
:10F46000344D345934653472347E348A34A134A432
:10F4700034A4289E289028842878286B285F285355
:10F480002847283A282E28222815280528031B1249
:10F490001B1F1B2B1B371B441B501B5C1B681B7546
:10F4A0001B811B8D1B991BA91BA91BBB1BC71BD435
:10F4B0001BD40FC70FBB0FA60F9E0F930F870F7B99
:10F4C0000F6E0F620F560F4A0F3D0F310F250F19A8
:10F4D0000F0C0F000F00000F001C00280034004428
:10F4E0000050005C0068007800840090009C00AC34
:10F4F00000BB00C700D400D40004040404010401CC
:10F5000001040401010101010404040404040404CD
:10F5100004040101040404040404040404040404B1
:10F52000040404040404040404040404040404049B
:10F53000040404040404040404040404040404048B
:10F54000040404040404040404040404040404047B
:10F550000404040404040404FA0000000000000091
:10F5600001000000000000004B0000003D3C0008CE
:10F57000FF000000FA000000000000000100000091
:10F58000000000004A0000003D3C0008FF000000B1
:10F59000FA00000000000000010000000000000070
:10F5A000490000003D3C0008FF000000FA00000098
:10F5B0000000000001000000000000004800000002
:10F5C0003D3C0008FF000000FA00000000000000C1
:10F5D0000100000000000000470000003D3C000862
:10F5E000FF000000FA000000000000000100000021
:10F5F000000000005E000000A53E0008FF000000C3
:10F60000FA00000000000000FF0000000000000001
:10F61000FF000000000000000000000000000000EB
:10F6200000000000000000000000000000000000DA
:10F630000000000000000000F8E70008007C000067
:10F6400000000000FE1600204D5E000801140A1E96
:10F650000150082800FF00FFFF03390501030102E4
:10F660000096000003000000FFFFFFFF0400000001
:10F670000400000000000000000000000000000086
:10F68000000000000000000000000000000000007A
:10F69000000000000000000000000000000000006A
:10F6A000000000000000000000000000000000005A
:10F6B000030000000000000077B60008EDB6000867
:10F6C00020002000000000000000000002000000F8
:10F6D0000000000003000000000000002BB700083D
:10F6E0000000000008000000000000000000000012
:10F6F0000200000000000000203300200202000091
:10F7000004000000040000002000000020000000B1
:10F710000000000058220020E82200200000000025
:10F7200000000000000000000000000000000000D9
:10F7300000000000000000000000000000000000C9
:10F7400000000000000000000000000000000000B9
:10F7500000000000000000000000000000000000A9
:10F760000000000000000000000000000000000099
:10F770000000000000000000000000000000000089
:10F780000000000000000000000000000000000079
:10F790000000000000000000000000000100000068
:10F7A00019B2000875B20008B9B20008D9B2000851
:10F7B000009600000000080000A24A041E1E00007F
:04000005080001B935
:00000001FF
